:020000040801F1
:1000000000000220B5D501088919010891190108DD
:1000100099190108A1190108A91901080000000097
:10002000000000000000000000000000B1190108FD
:10003000BF19010800000000CD190108DB190108F3
:1000400005D6010805D6010805D6010805D6010820
:1000500005D6010805D6010805D6010805D6010810
:1000600005D6010805D6010805D60108E9190108D9
:10007000FD19010805D6010805D6010805D60108B5
:1000800005D6010805D6010805D6010805D60108E0
:10009000111A010805D6010805D6010805D6010880
:1000A00005D6010805D6010805D6010805D60108C0
:1000B00005D6010805D6010805D6010805D60108B0
:1000C00005D6010805D6010805D6010805D60108A0
:1000D00005D6010805D6010805D6010805D6010890
:1000E00005D6010805D6010805D6010805D6010880
:1000F00005D6010805D6010805D6010805D6010870
:1001000005D6010805D6010805D6010805D601085F
:1001100005D6010805D6010805D6010805D601084F
:1001200005D6010805D6010805D6010805D601083F
:1001300005D6010805D6010805D6010805D601082F
:1001400005D6010805D6010805D601080000000003
:10015000000000000000000000000000000000009F
:1001600000000000000000000000000005D60108AB
:1001700005D6010805D6010805D6010805D60108EF
:1001800005D6010805D6010805D6010805D60108DF
:1001900005D601080000000005D6010805D60108B3
:1001A00005D6010805D6010805D6010805D60108BF
:1001B00005D6010805D6010805D6010805D60108AF
:1001C00005D6010805D6010805D6010805D601089F
:0801D00005D6010805D601085F
:1001D80010B5054C237833B9044B13B10448AFF379
:1001E80000800123237010BD84010020000000005E
:1001F80008D6010808B5034B1BB103490348AFF300
:10020800008008BD000000008801002008D6010811
:1002180053B94AB9002908BF00281CBF4FF0FF3165
:100228004FF0FF3000F06AB9ADF1080C6DE904CE6B
:1002380000F006F8DDF804E0DDE9022304B07047B9
:100248002DE9F047089D0C46002B4ED194468C456D
:100258008646B2FA82F262D94AB1C2F120039140CD
:1002680020FA03F30CFA02FC194300FA02FE4FEAE3
:100278001C471FFA8CF6B1FBF7F44FEA1E4307FB45
:10028800141143EA014304FB06F199420AD91CEB15
:10029800030304F1FF3080F01281994240F20F818C
:1002A800023C6344591A1FFA8EF3B1FBF7F007FBBF
:1002B800101143EA014300FB06F69E420AD91CEBE3
:1002C800030300F1FF3180F0FC809E4240F2F98088
:1002D800634402389B1B40EA044000211DB1D3400F
:1002E8000022C5E90032BDE8F0878B4205D90DB17F
:1002F800C5E9000100210846F5E7B3FA83F10029B2
:1003080046D1A34202D39042C0F0F080861A64EB33
:1003180003030120002DE6D0C5E90063E3E7002AC6
:1003280040F09080A1EB0C044FEA1C481FFA8CF7B0
:100338000121B4FBF8F64FEA1E4308FB164443EAD2
:10034800044307FB06F0984208D91CEB030306F1A7
:10035800FF3402D2984200F2CD8026461C1A1FFABA
:100368008EF3B4FBF8F008FB104443EA044300FBA7
:1003780007F79F4208D91CEB030300F1FF3402D2B0
:100388009F4200F2B0802046DB1B40EA0640A5E70A
:10039800C1F120068B4022FA06F71F4320FA06FC1B
:1003A80004FA01F343EA0C03F44000FA01F8380CAC
:1003B8004FEA1349B4FBF0FE1FFA87FC00FB1E440A
:1003C80049EA04440EFB0CF9A14502FA01F20AD9E4
:1003D8003C190EF1FF3A80F08480A14540F28180FB
:1003E800AEF1020E3C44A4EB09041FFA83F9B4FBF6
:1003F800F0F300FB134449EA044403FB0CFCA44556
:1004080007D93C1903F1FF3067D2A44565D9023BEF
:100418003C4443EA0E40A0FB0293A4EB0C049C422C
:10042800CE469C4651D34ED055B1B8EB0E0364EB83
:100438000C0404FA06F6CB401E43CC40C5E9006420
:10044800002150E7C2F1200320FA03F10CFA02FC64
:1004580024FA03F394400C434FEA1C4800FA02FEC6
:100468001FFA8CF7B3FBF8F008FB1031230C43EAB2
:10047800014300FB07F1994208D91CEB030300F183
:10048800FF362CD299422AD9023863445B1AA4B2A7
:10049800B3FBF8F108FB113344EA034401FB07F30B
:1004A800A34208D91CEB040401F1FF3613D2A3427E
:1004B80011D902396444E41A41EA004139E7044693
:1004C800F0E6084606E7C845AED2B9EB020E63EB84
:1004D800070C0138A8E73146EDE7034699E73046AF
:1004E800D4E7D6467FE7634402384DE706462346FD
:1004F80008460FE7023E634430E700BF704700BF7D
:1005080002440346934200D1704703F8011BF9E700
:1005180070B50D4D0D4C641BA4100026A64209D1E0
:100528000B4D0C4C0DF06CF8641BA4100026A64271
:1005380005D170BD55F8043B98470136EEE755F8EC
:10054800043B98470136F2E7B0D60108B0D6010857
:10055800B0D60108B4D6010890B587B000AF4FF403
:100568007A737B6064237B6106F00CF800F0B2F9C3
:1005780000F0B0FB00F032FE00F062FE00F0FAFE80
:1005880000F0C0FF01F04AF800F002FC00F0AAFCFD
:1005980001F052F901F06AFD00233B6116E0484979
:1005A8003A6913465B0013449B000B440433002252
:1005B8001A6043493A6913465B0013449B000B4495
:1005C8000833404A1A603B6901333B613B69052B9C
:1005D800E5D97F213C4809F091F87F213B4809F093
:1005E8008DF804223A49384808F084F9022239493A
:1005F800364808F07FF9384B1B6800225A63364B9F
:100608001B6800229A63344B1B680022DA63334B61
:100618001B6800225A63314B1B6800229A632F4BD8
:100628001B680022DA6300212B4809F02DFC042105
:10063800294809F029FC0821274809F025FC002150
:10064800264809F021FC0421244809F01DFC082152
:10065800224809F019FC224809F044FB214B1B7879
:10066800002B76D0204B1B78002B72D00023FB6028
:100678001FE01349FA6813465B0013449B000B44C0
:10068800D3ED007A9FED192ADFED191A9FED191A9B
:10069800DFED160AB0EE670A00F0CCFAF0EE407A09
:1006A800154AFB689B001344C3ED007AFB680133CD
:1006B800FB60FB68052BDCD90123BB603EE000BF73
:1006C800B00100209A99993E14020020800200206F
:1006D800A0010020A80100200404002050040020EC
:1006E8009C040020AC010020AD0100200000C8429D
:1006F8000000000000C07345F80100206D4ABB6887
:100708009B001344D3ED007A6A4B93ED007AB0EE68
:10071800472ADFED691A9FED691ADFED670AB0EE27
:10072800670A00F087FAF0EE407A624ABB689B00DD
:100738001344C3ED007ABB680133BB60BB68052B6B
:10074800DCD900F0FBF95E4B00221A705D4B0022E9
:100758001A7005F07BFF02467B69D31A632B7FF67C
:100768007DAF05F073FF7861574B1B7823F00104C8
:100778004FF40061554807F06FF8034623435AB217
:10078800514B1B785BB213435BB2DAB24E4B1A7013
:100798004D4B1B7823F002044FF480514B4807F06F
:1007A8005BF803465B0023435AB2474B1B785BB2A6
:1007B80013435BB2DAB2444B1A70434B1B7823F0F5
:1007C80004044FF40051414807F046F803469B00E3
:1007D80023435AB23C4B1B785BB213435BB2DAB289
:1007E800394B1A70384B1B7823F008044FF48041BA
:1007F800364807F031F80346DB0023435AB2324B40
:100808001B785BB213435BB2DAB22F4B1A702E4BD4
:100818001B7823F010044FF400412C4807F01CF813
:1008280003461B0123435AB2274B1B785BB2134381
:100838005BB2DAB2244B1A70234B1B7823F02004E6
:100848004021234807F008F803465B0123435AB2C6
:100858001D4B1B785BB213435BB2DAB21A4B1A70AA
:10086800194B1B7823F040042021184806F0F4FFA8
:1008780003469B0123435AB2134B1B785BB21343C5
:100888005BB2DAB2104B1A700F4B1B7823F080045E
:1008980010210E4806F0E0FF0346DB0123435AB25D
:1008A800094B1B785BB213435BB2DAB2064B1A7082
:1008B800D4E600BFF8010020000000000000C84294
:1008C800AC010020AD010020100200200004004807
:1008D8000008004880B594B000AF07F1180338222B
:1008E80000211846FFF70CFE3B1D00221A605A60D3
:1008F8009A60DA601A61002007F038FA2123BB6198
:100908004FF48033FB6101233B6302237B630323A2
:10091800BB630423FB6355233B6402237B640423EA
:10092800BB640223FB6407F11803184605F09AFE1E
:100938000346002B01D000F0C7F90F237B60032387
:10094800BB600023FB6000233B6100237B613B1DF0
:100958000421184606F098F90346002B01D000F050
:10096800B3F900BF5037BD4680BD000080B582B0E6
:1009780000AF78607B681B68B3F1A04F02D100F02C
:100988000FF806E07B681B68044A934201D100F027
:100998006DF800BF0837BD4680BD00BF000100509C
:1009A80080B483B000AF00237B604FE02C4A7B68A3
:1009B80032F8133007EE903AB8EEE77A29497A68A8
:1009C80013465B0013449B000B440833D3ED007AB5
:1009D80027EE277A23497A6813465B0013449B0065
:1009E8000B440833D3ED007AF7EE006A76EEE76A37
:1009F8001C497A6813465B0013449B000B4404337C
:100A08001B6807EE903AF8EE677A66EEA77A77EEFB
:100A1800277A14497A6813465B0013449B000B44F9
:100A2800C3ED007A0E4A7B6832F8133018460D4938
:100A38007A6813465B0013449B000B440433186028
:100A4800094B01221A707B6801337B607B68032B9A
:100A5800ACD900BF00BF0C37BD465DF8047B7047BA
:100A6800A0010020B0010020AC01002080B483B0B8
:100A780000AF04237B6051E07B68043B2C4A32F8CA
:100A8800133007EE903AB8EEE77A2A497A681346A7
:100A98005B0013449B000B440833D3ED007A27EE28
:100AA800277A24497A6813465B0013449B000B4459
:100AB8000833D3ED007AF7EE006A76EEE76A1D494F
:100AC8007A6813465B0013449B000B4404331B688D
:100AD80007EE903AF8EE677A66EEA77A77EE277A0D
:100AE80014497A6813465B0013449B000B44C3ED1A
:100AF800007A7B68043B0E4A32F8133018460D49D9
:100B08007A6813465B0013449B000B440433186057
:100B1800094B01221A707B6801337B607B68052BC7
:100B2800AAD900BF00BF0C37BD465DF8047B7047EB
:100B3800A8010020B0010020AD01002080B584B0DC
:100B480000AF364BD3ED017A9FED352ADFED351A2C
:100B58009FED351ADFED330AB0EE670A00F06AF848
:100B680087ED030A2D4BD3ED027A9FED2D2ADFED99
:100B78002D1A9FED2D1ADFED2B0AB0EE670A00F053
:100B880059F887ED020A254BD3ED037A9FED242A05
:100B9800DFED241A9FED241ADFED220AB0EE670A72
:100BA80000F048F887ED010A1C4BD3ED047A9FED5D
:100BB8001C2ADFED1C1A9FED1C1ADFED1A0AB0EE95
:100BC800670A00F037F887ED000A184B1B68D7ED65
:100BD800037AFCEEE77A17EE902A5A63134B1B68E8
:100BE800D7ED027AFCEEE77A17EE902A9A630F4B5C
:100BF8001B68D7ED017AFCEEE77A17EE902ADA63E4
:100C08000B4B1B68D7ED007AFCEEE77A17EE902ABB
:100C18005A6300BF1037BD4680BD00BFF8010020F1
:100C280000409C45000000000000C8420404002069
:100C38005004002080B489B000AF87ED050AC7EDE5
:100C4800040A87ED031AC7ED021A87ED012A97ED0A
:100C5800057AD7ED047A37EE677AD7ED016AD7EDD2
:100C6800027A76EEE77A67EE276A97ED037AD7ED90
:100C7800047A37EE677AC6EE877A97ED027A77EECE
:100C8800277AC7ED077A97ED027AD7ED077AB4EE9F
:100C9800E77AF1EE10FA02DDBB68FB610AE097ED36
:100CA800017AD7ED077AB4EEE77AF1EE10FA01D5BA
:100CB8007B68FB61FB6907EE903AB0EE670A243760
:100CC800BD465DF8047B704780B400AF72B600BFC4
:100CD80000BFFDE780B58AB000AF07F1140300221A
:100CE8001A605A609A60DA601A61264BDB6C254AF2
:100CF80043F02003D364234BDB6C03F020033B61F8
:100D08003B69204BDB6C1F4A43F00103D3641D4B46
:100D1800DB6C03F00103FB60FB681A4BDB6C194AC0
:100D280043F00203D364174BDB6C03F00203BB6090
:100D3800BB68144BDB6C134A43F00403D364114BB8
:100D4800DB6C03F004037B607B684FF630037B6148
:100D58000023BB610223FB6107F1140319460A480B
:100D680006F0F8FB40237B610023BB610223FB6193
:100D780007F114031946054806F0ECFB00BF2837B5
:100D8800BD4680BD0010024000040048000800482D
:100D980080B58CB000AF07F1240300221A605A60B6
:100DA8009A603B1D202200211846FFF7A9FB484BFB
:100DB8004FF0A0421A60464B4FF440325A60444B01
:100DC80000229A60424B0022DA60414B00221A61ED
:100DD8003F4B01225A613E4B04229A613C4B002250
:100DE8001A773B4B00225A77394B04221A62384B48
:100DF800002283F82420364B4FF49062DA62344B99
:100E08004FF480621A63324B012283F83820304B4A
:100E18000022DA632E4B002283F840202C4807F08A
:100E2800ADFB0346002B01D0FFF74EFF00237B628A
:100E380007F124031946264808F0C2FC0346002B94
:100E480001D0FFF741FF234B7B600623BB600223E1
:100E5800FB607F233B6104237B610023BB613B1D57
:100E680019461B4807F02EFE0346002B01D0FFF75A
:100E78002BFF194B7B600C23BB603B1D19461448A4
:100E880007F020FE0346002B01D0FFF71DFF134B90
:100E98007B601223BB603B1D19460D4807F012FE0C
:100EA8000346002B01D0FFF70FFF0D4B7B60182383
:100EB800BB603B1D1946064807F004FE0346002B9D
:100EC80001D0FFF701FF00BF3037BD4680BD00BF2E
:100ED8001402002002003004040060080800900C8E
:100EE8001000C01080B588B000AF3B46202200211A
:100EF8001846FFF705FB334B334A1A60314B4FF462
:100F080040325A602F4B00229A602E4B0022DA6042
:100F18002C4B00221A612B4B01225A61294B0422C7
:100F28009A61284B00221A77264B00225A77254BC4
:100F380002221A62234B002283F82420214B4FF40B
:100F48009062DA621F4B4FF480621A631D4B0122D4
:100F580083F838201B4B0022DA631A4B002283F8EF
:100F68004020184807F00AFB0346002B01D0FFF782
:100F7800ABFE164B3B6006237B600223BB607F23DE
:100F8800FB6004233B6100237B613B4619460D4807
:100F980007F098FD0346002B01D0FFF795FE0C4B98
:100FA8003B600C237B603B461946064807F08AFDE8
:100FB8000346002B01D0FFF787FE00BF2037BD4650
:100FC80080BD00BF80020020000100500000524791
:100FD8000020903680B5A0B000AF786007F16C03B0
:100FE80000221A605A609A60DA601A6107F11803E1
:100FF800542200211846FFF783FA7B681B68B3F177
:10100800A04F6AD14FF40043BB614FF00053FB651A
:1010180007F11803184606F04FF80346002B01D0D5
:10102800FFF752FE664B1B680133654A1360644B39
:101038001B68012B0BD1634BDB6C624A43F40053F2
:10104800D364604BDB6C03F400537B617B695D4BBD
:10105800DB6C5C4A43F00103D3645A4BDB6C03F04E
:1010680001033B613B690F23FB6603233B670023B6
:101078007B6707F16C0319464FF0904006F06AFA57
:10108800514B524A1A60504B05225A604E4B00226F
:101098009A604D4B0022DA604B4B80221A614A4B12
:1010A8004FF480725A61484B4FF480629A61464B04
:1010B8002022DA61444B4FF480521A62424806F00B
:1010C800E3FB0346002B01D0FFF7FEFD7B683E4A99
:1010D8005A653D4A7B6893626EE07B681B683C4AB0
:1010E800934269D14FF40043BB614FF00053FB6555
:1010F80007F11803184605F0DFFF0346002B01D05F
:10110800FFF7E2FD2E4B1B6801332D4A13602C4B71
:101118001B68012B0BD12B4BDB6C2A4A43F4005381
:10112800D364284BDB6C03F40053FB60FB68254B4E
:10113800DB6C244A43F00103D364224BDB6C03F0DD
:101148000103BB60BB683023FB6603233B670023B6
:101158007B6707F16C0319464FF0904006F0FAF9E7
:101168001C4B1D4A1A601B4B24225A60194B002243
:101178009A60184B0022DA60164B80221A61154BD0
:101188004FF480725A61134B4FF480629A61114B8D
:101198002022DA610F4B4FF480521A620D4806F094
:1011A80073FB0346002B01D0FFF78EFD7B68094ACD
:1011B8005A65084A7B68936200BF8037BD4680BD88
:1011C800AC03002000100240EC020020080002409E
:1011D800000100504C0300201C00024080B582B082
:1011E80000AF164B9B6C154A43F004039364134BF2
:1011F8009B6C03F004037B607B68104B9B6C0F4A6D
:1012080043F0010393640D4B9B6C03F001033B60B7
:101218003B68002200210B2006F037FF0B2006F068
:101228004EFF002200210C2006F02FFF0C2006F0B4
:1012380046FF00BF0837BD4680BD00BF0010024012
:1012480080B500AF1B4B1C4A1A601A4B1B4A5A60E8
:10125800184B00229A60174B0122DA60154B0022C6
:101268001A61144B00225A61124B00229A61114BE9
:101278000022DA610F4B00221A620E4808F0A8FB20
:101288000346002B01D0FFF71FFD0021094808F095
:101298003AFC0346002B01D0FFF716FD0021054854
:1012A80008F07CFC0346002B01D0FFF70DFD00BFC2
:1012B80080BD00BFB003002000540040FBA7A03051
:1012C80080B59EB000AF786007F1640300221A6011
:1012D8005A609A60DA601A6107F1100354220021FB
:1012E8001846FFF70DF97B681B681F4A934236D1F1
:1012F80040233B610023FB6207F11003184605F009
:10130800DBFE0346002B01D0FFF7DEFC174BDB6C3E
:10131800164A43F00203D364144BDB6C03F0020358
:10132800FB60FB684FF440737B661223BB660023A7
:10133800FB6600233B6704237B6707F164031946B8
:101348000B4806F007F9094B9B6D084A43F4001354
:101358009365064B9B6D03F40013BB60BB6800BF2D
:101368007837BD4680BD00BF0054004000100240E1
:101378000004004880B59CB000AF07F1600300226C
:101388001A605A609A60DA6007F1540300221A6002
:101398005A609A6007F1380300221A605A609A600E
:1013A800DA601A615A619A613B1D3422002118469D
:1013B800FFF7A6F8514B524A1A60504B10225A6058
:1013C8004E4B00229A604D4B42F20F72DA604B4B43
:1013D80000221A61494B00225A61484B80229A61C7
:1013E800464808F027FC0346002B01D0FFF76CFCA9
:1013F8004FF480533B6607F1600319463F4808F0F5
:1014080069FF0346002B01D0FFF75EFC3B4808F05C
:10141800D9FC0346002B01D0FFF756FC00237B655F
:101428000023BB650023FB6507F1540319463348C5
:1014380009F0FCFC0346002B01D0FFF745FC6023B4
:10144800BB630023FB6300233B6400237B6400230E
:10145800BB640023FB6400233B6507F138030022CB
:101468001946264808F022FE0346002B01D0FFF754
:101478002BFC07F1380304221946204808F016FE11
:101488000346002B01D0FFF71FFC07F138030822A1
:1014980019461A4808F00AFE0346002B01D0FFF748
:1014A80013FC00237B600023BB600023FB60002348
:1014B8003B6100237B614FF40053BB610023FB6158
:1014C80000233B6200237B624FF00073BB62002362
:1014D800FB6200233B6300237B633B1D19460748DF
:1014E80009F03AFD0346002B01D0FFF7EDFB034856
:1014F80000F028F900BF7037BD4680BD0404002005
:10150800002C014080B58EB000AF07F128030022FF
:101518001A605A609A60DA6007F11C0300221A60A8
:101528005A609A603B4600221A605A609A60DA60F4
:101538001A615A619A61384B4FF080421A60364BF3
:1015480010225A60344B00229A60334B42F20F72D9
:10155800DA60314B00221A612F4B80229A612E48A3
:1015680008F068FB0346002B01D0FFF7ADFB4FF4F2
:101578008053BB6207F128031946274808F0AAFEE2
:101588000346002B01D0FFF79FFB234808F01AFC05
:101598000346002B01D0FFF797FB0023FB610023D4
:1015A8007B6207F11C0319461B4809F03FFC034600
:1015B800002B01D0FFF788FB60233B6000237B6092
:1015C8000023BB6000233B613B46002219461248BA
:1015D80008F06CFD0346002B01D0FFF775FB3B4676
:1015E800042219460C4808F061FD0346002B01D07F
:1015F800FFF76AFB3B4608221946074808F056FDE4
:101608000346002B01D0FFF75FFB034800F09AF870
:1016180000BF3837BD4680BD5004002080B588B073
:1016280000AF07F1100300221A605A609A60DA606E
:101638003B1D00221A605A609A601D4B1D4A1A60B1
:101648001B4BA9225A601A4B00229A60184B40F291
:10165800E732DA60164B00221A61154B80229A6134
:10166800134808F0E7FA0346002B01D0FFF72CFBDC
:101678004FF480533B6107F1100319460C4808F0FA
:1016880029FE0346002B01D0FFF71EFB20237B60B9
:101698000023FB603B1D1946054809F0C7FB0346BC
:1016A800002B01D0FFF710FB00BF2037BD4680BDDF
:1016B8009C0400200004004080B487B000AF78602C
:1016C8007B681B681C4A93420CD11C4B1B6E1B4A3F
:1016D80043F400631366194B1B6E03F400637B61CC
:1016E8007B6922E07B681B68B3F1804F0CD1134BF8
:1016F8009B6D124A43F001039365104B9B6D03F0F9
:1017080001033B613B6910E07B681B680C4A93420C
:101718000BD10A4B9B6D094A43F002039365074BB3
:101728009B6D03F00203FB60FB6800BF1C37BD46DE
:101738005DF8047B704700BF002C01400010024098
:101748000004004080B58AB000AF786007F1140348
:1017580000221A605A609A60DA601A617B681B6816
:10176800324A93421ED1324BDB6C314A43F00103BB
:10177800D3642F4BDB6C03F001033B613B694FF4EF
:10178800E0637B610223BB610023FB6100233B62B2
:1017980006237B6207F1140319464FF0904005F0C9
:1017A800D9FE3FE07B681B68B3F1804F3AD1204BEC
:1017B800DB6C1F4A43F00203D3641D4BDB6C03F060
:1017C8000203FB60FB681A4BDB6C194A43F0010308
:1017D800D364174BDB6C03F00103BB60BB684FF4A9
:1017E80081637B610223BB610023FB6100233B62B1
:1017F80001237B6207F1140319460E4805F0AAFE7F
:101808004FF400437B610223BB610023FB6100238B
:101818003B6201237B6207F1140319464FF09040A5
:1018280005F098FE00BF2837BD4680BD002C01405A
:10183800001002400004004880B500AF224B234A44
:101848001A60214B4FF4E1325A601F4B00229A6014
:101858001D4B0022DA601C4B00221A611A4B0C2225
:101868005A61194B00229A61174B0022DA61164B14
:1018780000221A62144B00225A62134B00229A6209
:10188800114809F0FDFB0346002B01D0FFF71CFAB5
:1018980000210D480AF098F90346002B01D0FFF704
:1018A80013FA002108480AF0CDF90346002B01D0AD
:1018B800FFF70AFA04480AF04EF90346002B01D054
:1018C800FFF702FA00BF80BDE8040020003801409D
:1018D80080B59EB000AF786007F1640300221A60FB
:1018E8005A609A60DA601A6107F1100354220021E5
:1018F8001846FEF705FE7B681B681E4A934235D1E1
:1019080001233B6100237B6107F11003184605F0B2
:10191800D3FB0346002B01D0FFF7D6F9164B1B6EFD
:10192800154A43F480431366134B1B6E03F480433C
:10193800FB60FB68104BDB6C0F4A43F00203D36477
:101948000D4BDB6C03F00203BB60BB68C0237B66F6
:101958000223BB660023FB6600233B6707237B67E4
:1019680007F164031946054805F0F4FD00BF783710
:10197800BD4680BD00380140001002400004004808
:1019880080B400AF00BFFDE780B400AF00BFFDE743
:1019980080B400AF00BFFDE780B400AF00BFFDE733
:1019A80080B400AF00BFFDE780B400AF00BFBD4604
:1019B8005DF8047B704780B400AF00BFBD465DF89A
:1019C800047B704780B400AF00BFBD465DF8047B60
:1019D800704780B500AF04F027FE00BF80BD00004F
:1019E80080B500AF024806F072F800BF80BD00BFA6
:1019F800EC02002080B500AF024806F068F800BF8E
:101A080080BD00BF4C03002080B500AF024800F045
:101A1800FCFD00BF80BD00BF7C05002080B582B002
:101A280000AF0F4B1B6E0E4A43F0010313660C4BBD
:101A38001B6E03F001037B607B68094B9B6D084AB2
:101A480043F080539365064B9B6D03F080533B60D6
:101A58003B6806F02FFA00BF0837BD4680BD00BFBF
:101A68000010024080B598B000AF786007F10C0311
:101A7800542200211846FEF743FD7B681B68154A6F
:101A8800934222D14FF40053FB600023BB6407F15B
:101A98000C03184605F010FB0346002B01D0FFF796
:101AA80013F90D4B9B6D0C4A43F4000393650A4BE5
:101AB8009B6D03F40003BB60BB6800220021142067
:101AC80006F0E3FA142006F0FAFA00BF6037BD46C4
:101AD80080BD00BF005C00400010024080B582B0AD
:101AE80000AF78607B68D3F8D8227B6803F526734B
:101AF800194610460AF0EAF900BF0837BD4680BD0E
:101B080080B582B000AF78600B46FB707B68D3F875
:101B1800D802FA78796813469B001344DB000B441B
:101B280003F5B2731A68FB7819460AF024FA00BF65
:101B38000837BD4680BD80B582B000AF78600B46DF
:101B4800FB707B68D3F8D802FA78796813469B0053
:101B58001344DB000B4424331A68FB7819460AF057
:101B68006DFA00BF0837BD4680BD80B582B000AFB2
:101B780078607B68D3F8D83218460AF081FB00BF3A
:101B88000837BD4680BD80B584B000AF78600123BA
:101B9800FB737B685B79022B01D0FFF795F87B68B4
:101BA800D3F8D832FA7B114618460AF02BFB7B682B
:101BB800D3F8D83218460AF0D7FA00BF1037BD4616
:101BC80080BD000080B582B000AF78607B68D3F834
:101BD800D83218460AF026FB7B685B7A002B05D0C2
:101BE800044B1B69034A43F00603136100BF08371F
:101BF800BD4680BD00ED00E080B582B000AF7860E2
:101C08007B685B7A002B07D0084B1B69074A23F0D7
:101C18000603136100F0F8F97B68D3F8D832184648
:101C28000AF016FB00BF0837BD4680BD00ED00E096
:101C380080B582B000AF78602B4A7B68C2F8D83292
:101C48007B68294AC3F8C422274B284A1A60264BC6
:101C580008221A71244B02225A71234B0222DA718C
:101C6800214B00221A72204B00225A721E4B00226E
:101C78009A721D4B0022DA721B4800F0D6FB03460D
:101C8800002B01D0FFF720F87B68D3F8C402182393
:101C98000022002102F08FF87B68D3F8C402582391
:101CA8000022802102F087F87B68D3F8C402C023A1
:101CB8000022812102F07FF87B68D3F8C4024FF438
:101CC80088730022012102F076F87B68D3F8C402F9
:101CD8004FF480730022822102F06DF80023184629
:101CE8000837BD4680BD00BF7C050020005C004071
:101CF80080B584B000AF78600023FB730023BB730A
:101D08007B68D3F8C432184600F05DFC0346FB73C9
:101D1800FB7B184600F07EF90346BB73BB7B184675
:101D28001037BD4680BD80B584B000AF78600846E6
:101D380011461A460346FB700B46BB7013463B80A0
:101D48000023FB730023BB737B68D3F8C402BB7802
:101D58003A88F97800F0A4FD0346FB73FB7B18462C
:101D680000F058F90346BB73BB7B18461037BD46D5
:101D780080BD80B584B000AF78600B46FB7000234F
:101D8800FB730023BB737B68D3F8C432FA7811461F
:101D9800184600F0E2FD0346FB73FB7B184600F093
:101DA80039F90346BB73BB7B18461037BD4680BD67
:101DB80080B584B000AF78600B46FB700023FB73DE
:101DC8000023BB737B68D3F8C432FA7811461846EF
:101DD80000F08BFE0346FB73FB7B184600F01AF9F4
:101DE8000346BB73BB7B18461037BD4680BD80B524
:101DF80084B000AF78600B46FB700023FB730023B0
:101E0800BB737B68D3F8C432FA781146184600F0E1
:101E1800BEFE0346FB73FB7B184600F0FBF8034647
:101E2800BB73BB7B18461037BD4680BD80B485B0F8
:101E380000AF78600B46FB707B68D3F8C432FB6058
:101E480097F90330002B0BDAFB7803F07F02F9686F
:101E580013469B001344DB000B4412331B780BE042
:101E6800FB7803F07F02F96813469B001344DB00FC
:101E78000B4403F5A9731B7818461437BD465DF863
:101E8800047B704780B584B000AF78600B46FB7068
:101E98000023FB730023BB737B68D3F8C432FA7842
:101EA8001146184600F0D8FC0346FB73FB7B184626
:101EB80000F0B0F80346BB73BB7B18461037BD462D
:101EC80080BD80B586B000AFF8607A603B600B4695
:101ED800FB720023FB750023BB75FB68D3F8C402B3
:101EE800F97A3B687A6800F0C9FD0346FB75FB7D0B
:101EF800184600F08FF80346BB75BB7D18461837A7
:101F0800BD4680BD80B586B000AFF8607A603B60A2
:101F18000B46FB720023FB750023BB75FB68D3F8E7
:101F2800C402F97A3B687A6800F05FFD0346FB75E6
:101F3800FB7D184600F06EF80346BB75BB7D18465E
:101F48001837BD4680BD80B582B000AF78600B46BB
:101F5800FB707B68D3F8C432FA781146184600F053
:101F680075FD034618460837BD4680BD80B582B06A
:101F780000AF78600B46FB70FB78002B02D0012B7A
:101F880013D023E07B685B7A002B07D000F03CF885
:101F9800104B1B690F4A23F0060313617B68D3F8C3
:101FA800D83218460AF054F910E07B68D3F8D832D2
:101FB80018460AF037F97B685B7A002B05D0054B89
:101FC8001B69044A43F00603136100BF00BF0837CA
:101FD800BD4680BD00ED00E080B483B000AF7860FE
:101FE800034B18460C37BD465DF8047B704700BFAD
:101FF8005808002080B483B000AF786000BF0C3769
:10200800BD465DF8047B704780B500AFFEF762FC03
:1020180000BF80BD80B485B000AF0346FB710023CC
:10202800FB73FB79032B17D801A252F823F000BFEA
:10203800492001084F200108552001085B200108AC
:102048000023FB730BE00323FB7308E00123FB73FE
:1020580005E00323FB7302E00323FB7300BFFB7B54
:1020680018461437BD465DF8047B704780B500AF4D
:1020780000221249124809F087FE0346002B01D0BE
:10208800FEF722FE0F490E4809F0AEFE0346002B6C
:1020980001D0FEF719FE0C4909480BF011FA034666
:1020A800002B01D0FEF710FE054809F0C4FE0346D8
:1020B800002B01D0FEF708FE00BF80BD0000002005
:1020C800780A0020800000205400002080B483B0EB
:1020D80000AF03463960FB713B6812221A80034B3C
:1020E80018460C37BD465DF8047B70472000002079
:1020F80080B483B000AF03463960FB713B680422AB
:102108001A80034B18460C37BD465DF8047B7047B0
:102118003400002080B582B000AF03463960FB71FF
:10212800FB79002B05D13A68074908480AF06BFE8D
:1021380004E03A68044905480AF065FE024B18466F
:102148000837BD4680BD00BF480D002020D60108D5
:1021580080B582B000AF03463960FB713A68044924
:1021680004480AF050FE024B18460837BD4680BDA9
:10217800480D002038D6010880B582B000AF03466C
:102188003960FB713B681A221A8000F043F8024B51
:1021980018460837BD4680BD3800002080B582B09B
:1021A80000AF03463960FB71FB79002B05D13A6813
:1021B800074908480AF027FE04E03A680449054838
:1021C8000AF021FE024B18460837BD4680BD00BF05
:1021D800480D00204CD6010880B582B000AF0346F8
:1021E8003960FB71FB79002B05D13A68074908482B
:1021F8000AF009FE04E03A68044905480AF003FEBB
:10220800024B18460837BD4680BD00BF480D002068
:1022180058D6010880B584B000AF0F4B1B68FB602F
:102228000E4B1B68BB600E4B1B687B60FA687B68B3
:102238001344FB60FB68002B09D008220949F868A1
:1022480000F014F804220849B86800F00FF800BF3D
:102258001037BD4680BD00BF9075FF1F9475FF1FE6
:102268009875FF1F3A0000204A00002080B487B00C
:1022780000AFF860B9601346FB710023FB750023BB
:10228800FB7527E0FB681B0F092B0BD8FB681B0F9E
:10229800DAB2FB7D5B001946BB680B443032D2B220
:1022A8001A700AE0FB681B0FDAB2FB7D5B00194667
:1022B800BB680B443732D2B21A70FB681B01FB6053
:1022C800FB7D5B000133BA68134400221A70FB7D62
:1022D8000133FB75FA7DFB799A42D3D300BF00BF67
:1022E8001C37BD465DF8047B7047000080B500AF21
:1022F8000022054905480BF0F8F8054903480BF09A
:1023080012F90023184680BD48170020780A0020DB
:10231800480F002080B400AF00231846BD465DF882
:10232800047B704780B483B000AF03463960FB710B
:102338001346BB80FB79232B4AD801A252F823F01D
:10234800D9230108D9230108D9230108D923010871
:10235800D9230108D9230108D9230108D923010861
:10236800D9230108D9230108D9230108D923010851
:10237800D9230108D9230108D9230108D923010841
:10238800D9230108D9230108D9230108D923010831
:10239800D9230108D9230108D9230108D923010821
:1023A800D9230108D9230108D9230108D923010811
:1023B800D9230108D9230108D9230108D923010801
:1023C800D9230108D9230108D9230108D9230108F1
:1023D80000BF002318460C37BD465DF8047B7047E4
:1023E80080B582B000AF78603960796805480BF035
:1023F8009AF804480BF0B0F8002318460837BD4691
:1024080080BD00BF780A002080B487B000AFF860B4
:10241800B9601346FB710023FB7597F9173018460E
:102428001C37BD465DF8047B704780B584B000AFAB
:1024380078607B68002B01D10123C0E07B6893F8AA
:102448009132DBB2002B06D17B68002283F8902200
:102458007868FFF707FB7B68032283F891227B6883
:102468001B68184601F02BFD0023FB733EE0FA7B46
:10247800796813469B001344DB000B441133012297
:102488001A70FA7B796813469B001344DB000B44EF
:102498001033FA7B1A70FA7B796813469B00134451
:1024A800DB000B44133300221A70FA7B7968134659
:1024B8009B001344DB000B44203300221A60FA7B94
:1024C800796813469B001344DB000B442433002235
:1024D8001A60FB7B79685A1C13469B001344DB0087
:1024E8000B4400221A60FB7B0133FB737B681B796A
:1024F800FA7B9A42BBD30023FB7344E0FA7B7968EA
:1025080013469B001344DB000B4403F251130022D3
:102518001A70FA7B796813469B001344DB000B445E
:1025280003F5A873FA7B1A70FA7B796813469B0047
:102538001344DB000B4403F2531300221A70FA7B96
:10254800796813469B001344DB000B4403F5B07312
:1025580000221A60FA7B796813469B001344DB005B
:102568000B4403F5B27300221A60FA7B79681346AC
:102578009B001344DB000B4403F5B47300221A607C
:10258800FB7B0133FB737B681B79FA7B9A42B5D3DB
:102598007B6818687B68043393E8060001F0AAFC9E
:1025A8007B6800221A737B68012283F891227B687A
:1025B8009B7A012B02D1786801F040FC0023184671
:1025C8001037BD4680BD80B582B000AF78607B68AB
:1025D80093F89032012B01D1022312E07B6801228B
:1025E80083F890227B681B68184601F051FC7B68D1
:1025F8001B68184603F011FF7B68002283F89022BD
:10260800002318460837BD4680BD80B584B000AFAA
:1026180078607B681B68184603F016FFF860FB6853
:1026280003F40043002B03D0786800F004FB10E1AA
:10263800FB6803F48063002B13D07B681B68B3F836
:1026480044309AB27B681B6822F4806292B2A3F885
:1026580044207868FFF797FA0021786800F0FCF8C2
:10266800F7E0FB6803F48043002B0CD07B681B6801
:10267800B3F844309AB27B681B6822F4804292B265
:10268800A3F84420E5E0FB6803F40053002B0CD0CA
:102698007B681B68B3F844309AB27B681B6822F4E5
:1026A800005292B2A3F84420D3E0FB6803F48053AD
:1026B800002B34D07B681B68B3F840309AB27B6833
:1026C8001B6822F0040292B2A3F840207B681B68C2
:1026D800B3F840309AB27B681B6822F0080292B2C5
:1026E800A3F840207B6893F8C832012B07D17B6898
:1026F800002283F8C82200217868FFF737FC786841
:10270800FFF77AFA7B681B68B3F844309AB27B68A3
:102718001B6822F4805292B2A3F8442099E0FB6827
:1027280003F40063002B27D07B681B68B3F84030A4
:102738009AB27B681B6842F0080292B2A3F8402064
:102748007B681B68B3F844309AB27B681B6822F434
:10275800006292B2A3F844207B681B68B3F840304B
:102768009AB27B681B6842F0040292B2A3F8402038
:102778007868FFF727FA6CE0FB6803F08003002B0A
:1027880040D07B681B68B3F844309AB27B681B68FA
:1027980022F0800292B2A3F844207B6893F8C832F2
:1027A800002B2BD17B681B68B3F840309AB27B684A
:1027B8001B6842F0040292B2A3F840207B681B68B1
:1027C800B3F840309AB27B681B6842F0080292B2B4
:1027D800A3F840207B68012283F8C8227B681B6825
:1027E800B3F854309BB29B0803F03C027B68C3F8F3
:1027F800CC2201217868FFF7B9FB2AE07868FFF757
:10280800E1F926E0FB6803F40073002B0FD07B6826
:102818001B68B3F844309AB27B681B6822F40072D4
:1028280092B2A3F844207868FFF79FF911E0FB689B
:1028380003F48073002B0CD07B681B68B3F844301A
:102848009AB27B681B6822F4807292B2A3F8442083
:1028580000BF1037BD4680BD80B582B000AF78603C
:102868000B46FB707B6893F89032012B01D1022351
:1028780012E07B68012283F890227B68FA781A7349
:102888007B681B68FA781146184603F0B2FD7B682E
:10289800002283F89022002318460837BD4680BDE1
:1028A80080B584B000AF7860084611461A460346E2
:1028B800FB700B463B801346BB700023FB7297F9F5
:1028C8000330002B0EDAFB7803F0070213469B0057
:1028D8001344DB0010337A681344FB60FB68012261
:1028E8005A700EE0FB7803F0070213469B0013446E
:1028F800DB0003F5A8737A681344FB60FB680022C9
:102908005A70FB7803F00703DAB2FB681A703A884A
:10291800FB681A61FB68BA78DA70BB78022B02D1BF
:10292800FB6800221A717B6893F89032012B01D161
:1029380002230EE07B68012283F890227B681B68E3
:10294800F968184601F0F4FA7B68002283F89022AF
:10295800FB7A18461037BD4680BD80B584B000AFFD
:1029680078600B46FB7097F90330002B0EDAFB7882
:1029780003F0070213469B001344DB0010337A6808
:102988001344FB60FB6801225A700EE0FB7803F0E9
:10299800070213469B001344DB0003F5A8737A680B
:1029A8001344FB60FB6800225A70FB7803F00703AE
:1029B800DAB2FB681A707B6893F89032012B01D168
:1029C80002230EE07B68012283F890227B681B6853
:1029D800F968184601F070FE7B68002283F890229F
:1029E800002318461037BD4680BD80B586B000AFBD
:1029F800F8607A603B600B46FB72FB7A03F00702D3
:102A080013469B001344DB0003F5A873FA681344CC
:102A18007B617B697A685A617B693A689A617B69EC
:102A28000022DA617B6900225A70FB7A03F00703FF
:102A3800DAB27B691A70FB681B687969184602F07C
:102A480028F8002318461837BD4680BD80B483B0E7
:102A580000AF78600B46FB70FB7803F007027968DB
:102A680013469B001344DB000B4403F5B6731B6845
:102A780018460C37BD465DF8047B704780B586B0B4
:102A880000AFF8607A603B600B46FB72FB7A03F09C
:102A9800070213469B001344DB001033FA68134403
:102AA8007B617B697A685A617B693A689A617B695C
:102AB800012283F824207B693A681A627B69002224
:102AC800DA617B6901225A70FB7A03F00703DAB2F4
:102AD8007B691A70FB681B687969184601F0D9FF91
:102AE800002318461837BD4680BD80B584B000AFB6
:102AF80078600B46FB70FB7803F007037A6812795D
:102B0800934201D901233EE097F90330002B0EDAF6
:102B1800FB7803F0070213469B001344DB001033D5
:102B28007A681344FB60FB6801225A700CE0FA785B
:102B380013469B001344DB0003F5A8737A6813441B
:102B4800FB60FB6800225A70FB6801229A70FB78D0
:102B580003F00703DAB2FB681A707B6893F89032C7
:102B6800012B01D102230EE07B68012283F8902219
:102B78007B681B68F968184603F03CFB7B680022F9
:102B880083F89022002318461037BD4680BD80B5D3
:102B980084B000AF78600B46FB70FB7803F00F033E
:102BA8007A681279934201D9012340E097F90330FA
:102BB800002B0EDAFB7803F0070213469B00134440
:102BC800DB0010337A681344FB60FB6801225A70FB
:102BD8000EE0FB7803F0070213469B001344DB006A
:102BE80003F5A8737A681344FB60FB6800225A70E7
:102BF800FB6800229A70FB7803F00703DAB2FB68DF
:102C08001A707B6893F89032012B01D102230EE0F1
:102C18007B68012283F890227B681B68F968184654
:102C280003F039FB7B68002283F8902200231846C2
:102C38001037BD4680BD80B596B000AF7860ADE373
:102C48007B681B68B3F84430A7F84E30B7F84E30AD
:102C5800DBB203F00F0387F84D3097F84D30002BA7
:102C680040F06F81B7F84E3003F01003002B4CD1C1
:102C78007B681B681B889BB223F4E14323F0700335
:102C8800FB817B681A68FB896FEA43436FEA534309
:102C98009BB213807B6810337B657B681B68B3F835
:102CA80050309BB21A467B6D1B78DB0013447A6860
:102CB8001268134403F202431B88C3F309027B6DB5
:102CC800DA617B6D5A697B6DDB691A447B6D5A61E9
:102CD80000217868FEF72FFF7B681B7BDBB2002B97
:102CE80000F05C837B6D9B69002B40F057837B6809
:102CF8001B7BDBB263F07F03DAB27B681B68A3F847
:102D08004C207B6800221A7348E37B6803F5A8739C
:102D18007B657B681B681B88A7F84A30B7F84A3080
:102D280003F40063002B32D07B681B68B3F8503083
:102D38009BB21A467B6D1B78DB0013447A681268D5
:102D4800134403F206431B88C3F309027B6DDA615F
:102D58007B6818687B6803F526717B6DDA887B6D64
:102D6800DB699BB203F0C2FB7B681B681B889AB2C5
:102D780040F68F7313403B827B681B683A8A42F0A7
:102D8800800292B21A807868FEF7A8FE06E3B7F9C7
:102D98004A30002B80F202837B681B681B889AB23A
:102DA80040F68F731340FB837B681B68FA8B42F0F5
:102DB800800292B21A807B681B68B3F850309BB2CD
:102DC8001A467B6D1B78DB0013447A68126813443B
:102DD80003F206431B88C3F309027B6DDA617B6D3E
:102DE800DB69002B19D07B6D5B69002B15D07B68E4
:102DF80018687B6D59697B6DDA887B6DDB699BB2DE
:102E080003F074FB7B6D5A697B6DDB691A447B6D3B
:102E18005A6100217868FEF773FE7B681B681B887F
:102E2800A7F84A30B7F84A3003F40063002B40F0A3
:102E3800B582B7F84A3003F44053B3F5405F00F069
:102E4800AD827B681B68BB617B681B68B3F8503038
:102E58009BB21A46BB691344BB61BB6903F20643C4
:102E68007B617B691B889BB2C3F309039AB27B69B8
:102E78001A807B6D1B693E2B1DD97B6D1B695B0915
:102E88007B647B6D1B6903F01F03002B02D17B6CF5
:102E9800013B7B647B691B889AB27B6C9BB29B026B
:102EA8009BB213439BB26FEA43436FEA53439AB210
:102EB8007B691A8026E07B6D1B69002B0AD17B6930
:102EC8001B889BB26FEA43436FEA53439AB27B690C
:102ED8001A8017E07B6D1B695B087B647B6D1B693F
:102EE80003F00103002B02D07B6C01337B647B6908
:102EF8001B889AB27B6C9BB29B029BB213439AB21B
:102F08007B691A807B681B681B889BB223F480430B
:102F180023F070037B827B8A83F480537B827B8AD5
:102F280083F400537B827B681A687B8A43F07F4373
:102F380043F47F0343F4004343F080039BB21380C0
:102F48002CE27B681B681A4697F84D309B001344A7
:102F58001B88A7F84A30B7F94A30002B80F2F68070
:102F68007B681B681A4697F84D309B0013441B88F2
:102F78009AB240F68F731340A7F848307B681B68F5
:102F88001A4697F84D309B001344B7F8482042F092
:102F9800800292B21A8097F84D2013469B00134482
:102FA800DB0003F5A8737A6813447B657B6D1B7B94
:102FB800002B23D17B681B68B3F850309BB21A46AC
:102FC8007B6D1B78DB0013447A681268134403F2A4
:102FD80006431B88C3F30903A7F85030B7F85030ED
:102FE800002B00F08E807B6818687B6D59697B6DBB
:102FF800DA88B7F8503003F079FA82E07B6DDB7835
:10300800022B0AD1B7F84A301A46796D786800F071
:10301800D3F90346A7F8503073E07B681B681A465B
:103028007B6D1B789B0013441B889BB223F4E04301
:1030380023F07003A7F852307B681B681A467B6D33
:103048001B789B001A44B7F8523043F07F4343F48F
:103058007F0343F4004343F0C0039BB213807B68B3
:103068001B681A467B6D1B789B0013441B889BB218
:1030780003F48043002B22D07B681B68B3F85030E0
:103088009BB21A467B6D1B78DB0013447A68126882
:10309800134403F202431B88C3F30903A7F8503013
:1030A800B7F85030002B2CD07B6818687B6D5969B5
:1030B8007B6D1A89B7F8503003F018FA21E07B6865
:1030C8001B68B3F850309BB21A467B6D1B78DB0047
:1030D80013447A681268134403F206431B88C3F347
:1030E8000903A7F85030B7F85030002B09D07B6897
:1030F80018687B6D59697B6D5A89B7F8503003F0B1
:10310800F5F97B6DDA69B7F850301A447B6DDA61EE
:103118007B6D5A69B7F850301A447B6D5A617B6DE4
:103128009B69002B05D0B7F850207B6D1B699A422C
:1031380006D27B6D1B7819467868FEF7E1FC05E03E
:103148007B681B68796D184601F0A3FCB7F84A3014
:1031580003F08003002B00F0218197F84D201346DF
:103168009B001344DB0010337A6813447B657B684B
:103178001B681A4697F84D309B0013441B889BB276
:1031880023F4E14323F07003A7F842307B681B68FF
:103198001A4697F84D309B001A44B7F842306FEA48
:1031A80043436FEA53439BB213807B6DDB78012B5B
:1031B80040F0A2807B6D00229A617B6D1B7B002B07
:1031C80000F09380B7F84A3003F04003002B46D054
:1031D8007B6D5B78002B26D17B681B687B627B68E4
:1031E8001B68B3F850309BB21A467B6A13447B6263
:1031F8007B6D1B78DA007B6A134403F202433B625F
:103208003B6A1B889BB2C3F309039AB23B6A1A80D4
:103218003B6A1B889BB26FEA43436FEA53439AB2F7
:103228003B6A1A8061E07B6D5B78012B5DD17B681E
:103238001B68FB627B681B68B3F850309BB21A4668
:10324800FB6A1344FB627B6D1B78DA00FB6A13444C
:1032580003F20243BB62BB6A00221A8045E07B6826
:103268001B68FB637B6D5B78002B26D17B681B6832
:103278007B637B681B68B3F850309BB21A467B6B44
:1032880013447B637B6D1B78DA007B6B134403F27A
:1032980006433B633B6B1B889BB2C3F309039AB29B
:1032A8003B6B1A803B6B1B889BB26FEA43436FEA08
:1032B80053439AB23B6B1A8017E07B6D5B78012B06
:1032C80013D17B681B68B3F850309BB21A46FB6B6E
:1032D8001344FB637B6D1B78DA00FB6B134403F22A
:1032E8000643BB63BB6B00221A807B6D1B781946B3
:1032F8007868FEF720FC51E0B7F84A3003F4807391
:10330800002B44D17B681B68B3F850309BB21A4637
:103318007B6D1B78DB0013447A681268134403F250
:1033280002431B88C3F30903A7F840307B6D9A69F1
:10333800B7F840309A4207D97B6D9A69B7F84030A0
:10334800D21A7B6D9A6102E07B6D00229A617B6DD7
:103358009B69002B06D17B6D1B7819467868FEF7B0
:10336800EAFB1BE07B6D5A69B7F840301A447B6D65
:103378005A617B6DDA69B7F840301A447B6DDA61BF
:103388007B681B68796D184601F083FB06E0B7F887
:103398004A301A46796D786800F017F97B681B681F
:1033A800B3F844309BB21BB2002BFFF649AC0023A4
:1033B80018465837BD4680BD80B588B000AFF86064
:1033C800B9601346FB80FB8803F48043002B7CD054
:1033D800FB681B68B3F850309BB21A46BB681B7871
:1033E800DB001344FA681268134403F202431B8893
:1033F800C3F309037B83BB689A697B8B9A4206D324
:10340800BB689A697B8BD21ABB689A6102E0BB6879
:1034180000229A61BB689B69002B23D1FB681B685B
:103428001A46BB681B789B0013441B889BB223F485
:10343800804323F070033B833B8B83F400533B832F
:10344800FB681B681A46BB681B789B001A443B8BB9
:1034580043F07F4343F47F0343F4004343F0800386
:103468009BB21380FB8803F04003002B1FD0FB683E
:103478001B681A46BB681B789B0013441B889BB2C9
:1034880023F4E04323F07003FB82FB681B681A46B1
:10349800BB681B789B001A44FB8A43F07F4343F4C4
:1034A8007F0343F4004343F0C0039BB213807B8B3C
:1034B800002B00F08580FB681868BB685969BB68F9
:1034C8001A897B8B03F012F87AE0FB681B68B3F863
:1034D80050309BB21A46BB681B78DB001344FA686D
:1034E8001268134403F206431B88C3F309037B8362
:1034F800BB689A697B8B9A4206D3BB689A697B8BB7
:10350800D21ABB689A6102E0BB6800229A61BB6864
:103518009B69002B23D1FB681B681A46BB681B7884
:103528009B0013441B889BB223F4804323F0700351
:10353800FB83FB8B83F40053FB83FB681B681A46F1
:10354800BB681B789B001A44FB8B43F07F4343F412
:103558007F0343F4004343F080039BB21380FB884E
:1035680003F04003002B1FD1FB681B681A46BB6899
:103578001B789B0013441B889BB223F4E04323F081
:103588007003BB83FB681B681A46BB681B789B00EB
:103598001A44BB8B43F07F4343F47F0343F4004357
:1035A80043F0C0039BB213807B8B002B08D0FB68D1
:1035B8001868BB685969BB685A897B8B02F096FF0B
:1035C8007B8B18462037BD4680BD80B5A4B000AFC0
:1035D800F860B9601346FB80FB8803F04003002BBA
:1035E80000F0DB81FB681B68B3F850309BB21A46C9
:1035F800BB681B78DB001344FA681268134403F2B3
:1036080002431B88C3F30903A7F88630BB689A698D
:10361800B7F886309A4207D9BB689A69B7F88630F6
:10362800D21ABB689A6102E0BB6800229A61BB6843
:103638009B69002B40F0B980BB685B78002B26D1D2
:10364800FB681B68FB62FB681B68B3F850309BB2D1
:103658001A46FB6A1344FB62BB681B78DA00FB6AF4
:10366800134403F20243BB62BB6A1B889BB2C3F3D9
:1036780009039AB2BB6A1A80BB6A1B889BB26FEABD
:1036880043436FEA53439AB2BB6A1A801AE0BB6895
:103698005B78012B16D1FB681B687B63FB681B6892
:1036A800B3F850309BB21A467B6B13447B63BB68FC
:1036B8001B78DA007B6B134403F202433B633B6BDA
:1036C80000221A80FB681B687B62BB685B78002B52
:1036D80026D1FB681B68FB61FB681B68B3F8503098
:1036E8009BB21A46FB691344FB61BB681B78DA007E
:1036F800FB69134403F20643BB61BB691B889BB299
:10370800C3F309039AB2BB691A80BB691B889BB2D1
:103718006FEA43436FEA53439AB2BB691A8017E0D2
:10372800BB685B78012B13D1FB681B68B3F850307A
:103738009BB21A467B6A13447B62BB681B78DA002B
:103748007B6A134403F206433B623B6A00221A80F9
:10375800BB681B781946F868FEF7EDF9FB8803F497
:103768008043002B00F0FA82FB681B681A46BB688E
:103778001B789B0013441B889BB223F4E04323F07F
:103788007003FB82FB681B681A46BB681B789B00AA
:103798001A44FB8A43F07F4343F47F0343F44043D6
:1037A80043F080039BB21380D8E2FB8803F4804384
:1037B800002B21D0FB681B681A46BB681B789B004E
:1037C80013441B889BB223F4E04323F07003A7F84B
:1037D8008A30FB681B681A46BB681B789B001A4432
:1037E800B7F88A3043F07F4343F47F0343F4404300
:1037F80043F080039BB21380BB6893F82430012BFD
:1038080040F0AC82BB685A69B7F886301A44BB6886
:103818005A61BB68DA69B7F886301A44BB68DA615E
:10382800BB681A6ABB681B699A420BD3BB681B69E1
:10383800C7F88C30BB681A6AD7F88C30D21ABB68C4
:103848001A6217E0BB681B6A002B08D1B7F88630EC
:10385800C7F88C30BB68002283F824200AE0BB68D4
:10386800002283F82420BB681B6AC7F88C30BB6829
:1038780000221A62BB685B78002B65D1FB681B6865
:10388800FB63FB681B68B3F850309BB21A46FB6BAE
:103898001344FB63BB681B78DA00FB6B134403F229
:1038A8000243BB63BB6B1B889BB2C3F309039AB289
:1038B800BB6B1A80D7F88C303E2B1DD9D7F88C30CB
:1038C8005B09BB64D7F88C3003F01F03002B02D1CF
:1038D800BB6C013BBB64BB6B1B889AB2BB6C9BB2D5
:1038E8009B029BB213439BB26FEA43436FEA534375
:1038F8009AB2BB6B1A8044E0D7F88C30002B0AD1FF
:10390800BB6B1B889BB26FEA43436FEA53439AB27F
:10391800BB6B1A8035E0D7F88C305B08BB64D7F8EE
:103928008C3003F00103002B02D0BB6C0133BB6465
:10393800BB6B1B889AB2BB6C9BB29B029BB21343B6
:103948009AB2BB6B1A801CE0BB685B78012B18D15C
:10395800FB681B687B64FB681B68B3F850309BB23C
:103968001A467B6C13447B64BB681B78DA007B6C5B
:10397800134403F202433B64D7F88C309AB23B6C91
:103988001A80FB681868BB685969BB681A89D7F838
:103998008C309BB202F068FDE0E1FB681B68B3F86D
:1039A80050309BB21A46BB681B78DB001344FA6898
:1039B8001268134403F206431B88C3F30903A7F8EC
:1039C8008630BB689A69B7F886309A4207D3BB68D5
:1039D8009A69B7F88630D21ABB689A6102E0BB6868
:1039E80000229A61BB689B69002B40F0C080BB68CD
:1039F8005B78002B26D1FB681B68FB67FB681B689C
:103A0800B3F850309BB21A46FB6F1344FB67BB6890
:103A18001B78DA00FB6F134403F20243BB67BB6FEA
:103A28001B889BB2C3F309039AB2BB6F1A80BB6FA2
:103A38001B889BB26FEA43436FEA53439AB2BB6F4A
:103A48001A801AE0BB685B78012B16D1FB681B68EB
:103A58007B66FB681B68B3F850309BB21A467B6ED6
:103A680013447B66BB681B78DA007B6E134403F251
:103A780002433B663B6E00221A80FB681B687B672B
:103A8800BB685B78002B2BD1FB681B68FB66FB6867
:103A98001B68B3F850309BB21A46FB6E1344FB66A2
:103AA800BB681B78DA00FB6E134403F20643C7F8C1
:103AB8008030D7F880301B889BB2C3F309039AB2D1
:103AC800D7F880301A80D7F880301B889BB26FEA0D
:103AD80043436FEA53439AB2D7F880301A8017E00D
:103AE800BB685B78012B13D1FB681B68B3F85030B7
:103AF8009BB21A467B6F13447B67BB681B78DA005E
:103B08007B6F134403F206433B673B6F00221A8026
:103B1800BB681B781946F868FEF70DF8FB8803F4B4
:103B28008043002B40F01A81FB681B681A46BB686B
:103B38001B789B0013441B889BB223F4E04323F0BB
:103B48007003A7F88830FB681B681A46BB681B78A7
:103B58009B001A44B7F8883043F07F4343F47F034F
:103B680043F4404343F080039BB21380F6E0FB88A4
:103B780003F48043002B21D1FB681B681A46BB68FD
:103B88001B789B0013441B889BB223F4E04323F06B
:103B98007003A7F84E30FB681B681A46BB681B7891
:103BA8009B001A44B7F84E3043F07F4343F47F0339
:103BB80043F4404343F080039BB21380BB6893F8FF
:103BC8002430012B40F0CA80BB685A69B7F88630A8
:103BD8001A44BB685A61BB68DA69B7F886301A4478
:103BE800BB68DA61BB681A6ABB681B699A420BD367
:103BF800BB681B69C7F88C30BB681A6AD7F88C3069
:103C0800D21ABB681A6217E0BB681B6A002B08D17E
:103C1800B7F88630C7F88C30BB68002283F82420B8
:103C28000AE0BB681B6AC7F88C30BB6800221A62BE
:103C3800BB68002283F82420FB681B687B65BB688F
:103C48005B78002B65D1FB681B68FB65FB681B680C
:103C5800B3F850309BB21A46FB6D1344FB65BB6842
:103C68001B78DA00FB6D134403F20643BB65BB6D9A
:103C78001B889BB2C3F309039AB2BB6D1A80D7F8AD
:103C88008C303E2B1DD9D7F88C305B09BB66D7F832
:103C98008C3003F01F03002B02D1BB6E013BBB66C7
:103CA800BB6D1B889AB2BB6E9BB29B029BB213433F
:103CB8009BB26FEA43436FEA53439AB2BB6D1A80D3
:103CC80041E0D7F88C30002B0AD1BB6D1B889BB222
:103CD8006FEA43436FEA53439AB2BB6D1A8032E0EE
:103CE800D7F88C305B08BB66D7F88C3003F001033B
:103CF800002B02D0BB6E0133BB66BB6D1B889AB22A
:103D0800BB6E9BB29B029BB213439AB2BB6D1A80E7
:103D180019E0BB685B78012B15D1FB681B68B3F809
:103D280050309BB21A467B6D13447B65BB681B7889
:103D3800DA007B6D134403F206433B65D7F88C30F9
:103D48009AB23B6D1A80FB681868BB685969BB68F2
:103D58005A89D7F88C309BB202F086FBFB681B6847
:103D68001A46BB681B789B0013441B889BB223F43C
:103D7800E04323F04003BB82BB8A83F01003BB827D
:103D8800BB8A83F02003BB82FB681B681A46BB68AA
:103D98001B789B001A44BB8A43F07F4343F47F039C
:103DA80043F4004343F080039BB21380002318467A
:103DB8009037BD4680BD80B487B000AFF8607B60A7
:103DC8000B467B8113463B817B8903F080039BB2C2
:103DD800002B0BD07B8903F0070213469B0013448A
:103DE800DB001033FA6813447B6109E07A891346D3
:103DF8009B001344DB0003F5A873FA6813447B6146
:103E08003B89002B07D17B6900221A737B689AB221
:103E18007B69DA800BE07B6901221A737B689AB2AE
:103E28007B691A817B681B0C9AB27B695A810023D3
:103E380018461C37BD465DF8047B704780B485B0D2
:103E480000AF78607B681B68FB607B680122C3F861
:103E5800D0227B68002283F8C822FB68B3F854306C
:103E68009BB243F001039AB2FB68A3F85420FB68A5
:103E7800B3F854309BB243F002039AB2FB68A3F83C
:103E88005420002318461437BD465DF8047B70475C
:103E980080B485B000AF78607B680022A3F8442026
:103EA8004BF68073FB60FB689AB27B68A3F84020EE
:103EB800002318461437BD465DF8047B704780B46C
:103EC80085B000AF78604BF68073FB607B68B3F811
:103ED80040309AB2FB689BB2DB439BB213409AB264
:103EE8007B68A3F84020002318461437BD465DF8C8
:103EF800047B704780B485B000AFF8603B1D83E851
:103F08000600FB680122A3F84020FB680022A3F802
:103F18004020FB680022A3F84420FB680022A3F895
:103F28005020002318461437BD465DF8047B7047BF
:103F380080B49DB000AF78603960002387F86F3097
:103F48007A683B681B789B0013441B889BB223F458
:103F5800EC4323F07003A7F86C303B68DB78032B45
:103F68001FD801A252F823F0813F01089D3F0108A4
:103F7800B33F01088F3F0108B7F86C3043F4007372
:103F8800A7F86C3012E0B7F86C3043F4C063A7F8B8
:103F98006C300BE0B7F86C3043F48063A7F86C30F2
:103FA80004E0012387F86F3000E000BF7A683B68BF
:103FB8001B789B001A44B7F86C3043F07F4343F4F6
:103FC8007F0343F4004343F080039BB213807A6875
:103FD8003B681B789B0013441B889BB21BB223F4DD
:103FE800E04323F070031AB23B681B781BB21343FB
:103FF8001BB2A7F866307A683B681B789B001A44A6
:10400800B7F8663043F07F4343F47F0343F400433B
:1040180043F080039BB213803B681B7B002B40F06E
:1040280078813B685B78002B00F084807B68BB61FB
:104038007B68B3F850309BB21A46BB691344BB6126
:104048003B681B78DA00BB69134403F580637B6126
:104058003B68DB885B089BB25B009AB27B691A807D
:104068007A683B681B789B0013441B887B827B8A99
:1040780003F04003002B1BD07A683B681B789B0039
:1040880013441B889BB223F4E04323F070033B8264
:104098007A683B681B789B001A443B8A43F07F434D
:1040A80043F47F0343F4004343F0C0039BB21380FF
:1040B8003B68DB78012B20D07A683B681B789B0033
:1040C80013441B889BB223F4E04323F04003BB81D5
:1040D800BB8983F02003BB817A683B681B789B000F
:1040E8001A44BB8943F07F4343F47F0343F40043FE
:1040F80043F080039BB21380D5E27A683B681B7853
:104108009B0013441B889BB223F4E04323F0400335
:10411800FB817A683B681B789B001A44FB8943F053
:104128007F4343F47F0343F4004343F080039BB28F
:104138001380B8E27B683B637B68B3F850309BB26E
:104148001A463B6B13443B633B681B78DA003B6BB6
:10415800134403F20443FB623B68DB885B089BB2B1
:104168005B009AB2FB6A1A807B68BB627B68B3F813
:1041780050309BB21A46BB6A1344BB623B681B783B
:10418800DA00BB6A134403F206437B627B6A1B882E
:104198009BB2C3F309039AB27B6A1A803B681B6916
:1041A8003E2B1DD93B681B695B09BB663B681B69D5
:1041B80003F01F03002B02D1BB6E013BBB667B6A79
:1041C8001B889AB2BB6E9BB29B029BB213439BB2F5
:1041D8006FEA43436FEA53439AB27B6A1A8026E038
:1041E8003B681B69002B0AD17B6A1B889BB26FEA6C
:1041F80043436FEA53439AB27B6A1A8017E03B68DD
:104208001B695B08BB663B681B6903F00103002B55
:1042180002D0BB6E0133BB667B6A1B889AB2BB6E49
:104228009BB29B029BB213439AB27B6A1A807A684C
:104238003B681B789B0013441B887B847B8C03F4AE
:104248008043002B1BD07A683B681B789B00134483
:104258001B889BB223F4E04323F070033B847A6805
:104268003B681B789B001A443B8C43F07F4343F424
:104278007F0343F4404343F080039BB213803B68C1
:104288001B78002B24D17A683B681B789B00134469
:104298001B889BB223F4804323F07003BB83BB8B42
:1042A80083F48053BB83BB8B83F40053BB837A684E
:1042B8003B681B789B001A44BB8B43F07F4343F455
:1042C8007F0343F4004343F080039BB21380EAE189
:1042D8007A683B681B789B0013441B889BB223F4C5
:1042E800804323F07003FB83FB8B83F40053FB8331
:1042F8007A683B681B789B001A44FB8B43F07F432A
:1043080043F47F0343F4004343F080039BB21380DC
:10431800C9E13B68DB78022B1ED17A683B681B78C1
:104328009B0013441B889BB223F4E04323F07003E3
:10433800A7F862307A683B681B789B001A44B7F884
:10434800623043F07F4343F47F0343F4014343F077
:1043580080039BB213801DE07A683B681B789B0042
:1043680013441B889BB223F4E24323F07003A7F89D
:1043780064307A683B681B789B001A44B7F864304D
:1043880043F07F4343F47F0343F4004343F0800347
:104398009BB213807B68FB657B68B3F850309BB297
:1043A8001A46FB6D1344FB653B681B78DA00FB6D0E
:1043B800134403F58063BB653B681B895B089BB2AC
:1043C8005B009AB2BB6D1A807B687B657B68B3F82B
:1043D80050309BB21A467B6D13447B653B681B7853
:1043E800DA007B6D134403F204433B653B685B8949
:1043F8005B089BB25B009AB23B6D1A803B685B78A6
:10440800002B40F093807A683B681B789B0013442C
:104418001B88A7F84030B7F8403003F48043002BDE
:104428001BD07A683B681B789B0013441B889BB29F
:1044380023F4E04323F07003FB877A683B681B781A
:104448009B001A44FB8F43F07F4343F47F0343F4FC
:10445800404343F080039BB213807A683B681B7823
:104468009B0013441B88BB87BB8F03F04003002BC2
:104478001BD07A683B681B789B0013441B889BB24F
:1044880023F4E04323F070037B877A683B681B784A
:104498009B001A447B8F43F07F4343F47F0343F42C
:1044A800004343F0C0039BB213807A683B681B78D3
:1044B8009B0013441B889BB223F4804323F07003B2
:1044C8003B873B8F83F480533B873B8F83F40053B8
:1044D8003B877A683B681B789B001A443B8F43F004
:1044E8007F4343F47F0343F4004343F080039BB2CC
:1044F80013807A683B681B789B0013441B889BB227
:1045080023F4E04323F04003FB867A683B681B787A
:104518009B001A44FB8E43F07F4343F47F0343F42C
:10452800004343F080039BB21380BCE07A683B6889
:104538001B789B0013441B88A7F84E30B7F84E3001
:1045480003F48043002B1DD07A683B681B789B00DE
:1045580013441B889BB223F4E04323F07003A7F8AD
:104568004C307A683B681B789B001A44B7F84C308B
:1045780043F07F4343F47F0343F4404343F0800315
:104588009BB213807A683B681B789B0013441B8896
:10459800A7F84A30B7F84A3003F04003002B1DD083
:1045A8007A683B681B789B0013441B889BB223F4F2
:1045B800E04323F07003A7F848307A683B681B781B
:1045C8009B001A44B7F8483043F07F4343F47F0315
:1045D80043F4004343F0C0039BB213803B68DB788D
:1045E800012B24D07A683B681B789B0013441B88F6
:1045F8009BB223F4E04323F04003A7F84430B7F814
:10460800443083F02003A7F844307A683B681B786D
:104618009B001A44B7F8443043F07F4343F47F03C8
:1046280043F4004343F080039BB213801DE07A6893
:104638003B681B789B0013441B889BB223F4E04320
:1046480023F04003A7F846307A683B681B789B0044
:104658001A44B7F8463043F07F4343F47F0343F4EA
:10466800004343F080039BB213807A683B681B7851
:104678009B0013441B889BB223F4804323F07003F0
:10468800A7F842307A683B681B789B001A44B7F851
:10469800423043F07F4343F47F0343F4004343F045
:1046A80080039BB2138097F86F3018467437BD4665
:1046B8005DF8047B704700BF80B48DB000AF7860B0
:1046C80039603B681B7B002B40F08E803B685B7831
:1046D800002B44D07A683B681B789B0013441B88E6
:1046E800BB81BB8903F04003002B1BD07A683B6871
:1046F8001B789B0013441B889BB223F4E04323F0F0
:1047080070037B817A683B681B789B001A447B891D
:1047180043F07F4343F47F0343F4004343F0C00373
:104728009BB213807A683B681B789B0013441B88F4
:104738009BB223F4E04323F040033B817A683B6853
:104748001B789B001A443B8943F07F4343F47F0363
:1047580043F4004343F080039BB2138092E17A68EC
:104768003B681B789B0013441B887B827B8A03F47D
:104778008043002B1BD07A683B681B789B0013444E
:104788001B889BB223F4E04323F070033B827A68D2
:104798003B681B789B001A443B8A43F07F4343F4F1
:1047A8007F0343F4404343F080039BB213807A684D
:1047B8003B681B789B0013441B889BB223F48043FF
:1047C80023F07003FB817A683B681B789B001A44CE
:1047D800FB8943F07F4343F47F0343F4004343F0F2
:1047E80080039BB213804DE13B685B78002B40F05F
:1047F800A5807A683B681B789B0013441B883B8420
:104808003B8C03F48043002B1BD07A683B681B78F1
:104818009B0013441B889BB223F4E04323F07003EE
:10482800FB837A683B681B789B001A44FB8B43F038
:104838007F4343F47F0343F4404343F080039BB238
:1048480013807A683B681B789B0013441B88BB83E2
:10485800BB8B03F04003002B1BD07A683B681B78A6
:104868009B0013441B889BB223F4E04323F070039E
:104878007B837A683B681B789B001A447B8B43F0E8
:104888007F4343F47F0343F4004343F0C0039BB2E8
:1048980013807A683B681B789B0013441B889BB283
:1048A80023F4E04323F070033B837A683B681B786A
:1048B8009B001A443B8B43F07F4343F47F0343F44C
:1048C800004343F0C0039BB213807A683B681B78AF
:1048D8009B0013441B889BB223F4804323F070038E
:1048E800FB827A683B681B789B001A44FB8A43F07A
:1048F8007F4343F47F0343F4004343F080039BB2B8
:1049080013807A683B681B789B0013441B889BB212
:1049180023F4E04323F04003BB827A683B681B78AA
:104928009B001A44BB8A43F07F4343F47F0343F45C
:10493800004343F080039BB21380A3E07A683B688E
:104948001B789B0013441B88FB85FB8D03F4804375
:10495800002B1BD07A683B681B789B0013441B888C
:104968009BB223F4E04323F07003BB857A683B686D
:104978001B789B001A44BB8D43F07F4343F47F03AD
:1049880043F4404343F080039BB213807A683B684A
:104998001B789B0013441B887B857B8D03F04003A9
:1049A800002B1BD07A683B681B789B0013441B883C
:1049B8009BB223F4E04323F070033B857A683B689D
:1049C8001B789B001A443B8D43F07F4343F47F03DD
:1049D80043F4004343F0C0039BB213807A683B68FA
:1049E8001B789B0013441B889BB223F4E04323F0FD
:1049F8007003FB847A683B681B789B001A44FB8C25
:104A080043F07F4343F47F0343F4404343F0800380
:104A18009BB213807A683B681B789B0013441B8801
:104A28009BB223F4E04323F04003BB847A683B68DD
:104A38001B789B001A44BB8C43F07F4343F47F03ED
:104A480043F4004343F080039BB213807A683B68C9
:104A58001B789B0013441B889BB223F4804323F0EC
:104A680070037B847A683B681B789B001A447B8CB4
:104A780043F07F4343F47F0343F4004343F0800350
:104A88009BB21380002318463437BD465DF8047B7B
:104A9800704780B5C2B000AF07F58473A3F5827381
:104AA800186007F58473A3F58473196007F5847398
:104AB800A3F584731B685B78012B40F0B78607F574
:104AC8008473A3F584731B689A6907F58473A3F547
:104AD80084731B681B699A4208D907F58473A3F588
:104AE80084731B681B69C7F8043107E007F58473F2
:104AF800A3F584731B689B69C7F8043107F58473B1
:104B0800A3F584731B681B7B002B3AD107F58473CC
:104B1800A3F584731B68596907F58473A3F5847337
:104B28001B68DA88D7F804319BB207F58470A0F5C2
:104B38008270006801F098FC07F58473A3F582730E
:104B48001B683B6107F58473A3F582731B68B3F890
:104B580050309BB21A463B6913443B6107F5847396
:104B6800A3F584731B681B78DA003B69134403F2CE
:104B78000243FB60D7F804319AB2FB681A8000F050
:104B88001FBE07F58473A3F584731B68DB78022BBB
:104B980040F0628407F58473A3F584731B681A6A6E
:104BA80007F58473A3F584731B681B699A4240F266
:104BB800DF8307F58473A3F582731A6807F5847396
:104BC800A3F584731B681B789B0013441B889BB256
:104BD80023F4E04323F07003A7F8563007F58473F5
:104BE800A3F582731A6807F58473A3F584731B68A9
:104BF8001B789B001A44B7F8563043F07F4343F4C0
:104C08007F0343F4014343F080039BB2138007F50D
:104C18008473A3F584731B681A6AD7F80431D21A0F
:104C280007F58473A3F584731B681A6207F5847308
:104C3800A3F582731A6807F58473A3F584731B6858
:104C48001B789B0013441B889BB203F04003002B86
:104C580000F0C78107F58473A3F582731B683B6373
:104C680007F58473A3F584731B685B78002B77D1F1
:104C780007F58473A3F582731B68BB6207F5847319
:104C8800A3F582731B68B3F850309BB21A46BB6A0F
:104C98001344BB6207F58473A3F584731B681B7800
:104CA800DA00BB6A134403F206437B627B6A1B8803
:104CB8009BB2C3F309039AB27B6A1A80D7F804310E
:104CC8003E2B21D9D7F804315B09C7F80031D7F852
:104CD800043103F01F03002B04D1D7F80031013B46
:104CE800C7F800317B6A1B889AB2D7F800319BB2AB
:104CF8009B029BB213439BB26FEA43436FEA534351
:104D08009AB27B6A1A8050E0D7F80431002B0AD196
:104D18007B6A1B889BB26FEA43436FEA53439AB29C
:104D28007B6A1A8041E0D7F804315B08C7F8003184
:104D3800D7F8043103F00103002B04D0D7F8003171
:104D48000133C7F800317B6A1B889AB2D7F8003163
:104D58009BB29B029BB213439AB27B6A1A8024E0EF
:104D680007F58473A3F584731B685B78012B1CD14A
:104D780007F58473A3F582731B68B3F850309BB2B0
:104D88001A463B6B13443B6307F58473A3F584739E
:104D98001B681B78DA003B6B134403F20643FB6283
:104DA800D7F804319AB2FB6A1A8007F58473A3F521
:104DB80084731B685B89A7F8763007F58473A3F5BD
:104DC80084731B685969D7F804319BB2B7F8762009
:104DD80007F58470A0F58270006801F045FB07F5BF
:104DE8008473A3F584731B685A69D7F804311A448D
:104DF80007F58473A3F584731B685A6107F58473F8
:104E0800A3F584731B681A6A07F58473A3F5847382
:104E18001B681B699A420FD907F58473A3F584733D
:104E28001B681A6AD7F80431D21A07F58473A3F5F8
:104E380084731B681A620EE007F58473A3F5847304
:104E48001B681B6AC7F8043107F58473A3F58473DC
:104E58001B6800221A6207F58473A3F584731B6824
:104E68005B78002B77D107F58473A3F582731B68F1
:104E7800BB6107F58473A3F582731B68B3F85030E0
:104E88009BB21A46BB691344BB6107F58473A3F54B
:104E980084731B681B78DA00BB69134403F202436E
:104EA8007B617B691B889BB2C3F309039AB27B6958
:104EB8001A80D7F804313E2B21D9D7F804315B0981
:104EC800C7F8FC30D7F8043103F01F03002B04D1D6
:104ED800D7F8FC30013BC7F8FC307B691B889AB2D5
:104EE800D7F8FC309BB29B029BB213439BB26FEA8C
:104EF80043436FEA53439AB27B691A8056E0D7F866
:104F08000431002B0AD17B691B889BB26FEA4343AB
:104F18006FEA53439AB27B691A8047E0D7F80431A5
:104F28005B08C7F8FC30D7F8043103F00103002B05
:104F380004D0D7F8FC300133C7F8FC307B691B88F4
:104F48009AB2D7F8FC309BB29B029BB213439AB239
:104F58007B691A802AE007F58473A3F584731B68BC
:104F68005B78012B22D107F58473A3F582731B6844
:104F78003B6207F58473A3F582731B68B3F850305E
:104F88009BB21A463B6A13443B6207F58473A3F548
:104F980084731B681B78DA003B6A134403F20243EC
:104FA800FB61D7F804319AB2FB691A8007F584735C
:104FB800A3F584731B681B89A7F8763007F58473FB
:104FC800A3F584731B685969D7F804319BB2B7F805
:104FD800762007F58470A0F58270006801F044FA25
:104FE800EEE307F58473A3F584731B685B78002BE5
:104FF80077D107F58473A3F582731B68BB6407F543
:105008008473A3F582731B68B3F850309BB21A46B9
:10501800BB6C1344BB6407F58473A3F584731B68E6
:105028001B78DA00BB6C134403F202437B647B6C8D
:105038001B889BB2C3F309039AB27B6C1A80D7F81A
:1050480004313E2B21D9D7F804315B09C7F8F83071
:10505800D7F8043103F01F03002B04D1D7F8F83038
:10506800013BC7F8F8307B6C1B889AB2D7F8F83048
:105078009BB29B029BB213439BB26FEA43436FEA16
:1050880053439AB27B6C1A8056E0D7F80431002B50
:105098000AD17B6C1B889BB26FEA43436FEA534388
:1050A8009AB27B6C1A8047E0D7F804315B08C7F8DE
:1050B800F830D7F8043103F00103002B04D0D7F8F7
:1050C800F8300133C7F8F8307B6C1B889AB2D7F8F0
:1050D800F8309BB29B029BB213439AB27B6C1A8046
:1050E8002AE007F58473A3F584731B685B78012BAA
:1050F80022D107F58473A3F582731B683B6507F516
:105108008473A3F582731B68B3F850309BB21A46B8
:105118003B6D13443B6507F58473A3F584731B68E3
:105128001B78DA003B6D134403F20243FB64D7F8A3
:1051380004319AB2FB6C1A8007F58473A3F5847363
:105148001B681B89A7F8763007F58473A3F5847369
:105158001B685969D7F804319BB2B7F8762007F570
:105168008470A0F58270006801F07EF907F58473F9
:10517800A3F584731B685A69D7F804311A4407F5F4
:105188008473A3F584731B685A6107F58473A3F5C8
:1051980084731B681A6A07F58473A3F584731B6804
:1051A8001B699A420FD907F58473A3F584731B68AA
:1051B8001A6AD7F80431D21A07F58473A3F58473F1
:1051C8001B681A620EE007F58473A3F584731B68E5
:1051D8001B6AC7F8043107F58473A3F584731B6849
:1051E80000221A6207F58473A3F582731B683B6477
:1051F80007F58473A3F584731B685B78002B77D15C
:1052080007F58473A3F582731B68BB6307F5847382
:10521800A3F582731B68B3F850309BB21A46BB6B78
:105228001344BB6307F58473A3F584731B681B7869
:10523800DA00BB6B134403F206437B637B6B1B886A
:105248009BB2C3F309039AB27B6B1A80D7F8043177
:105258003E2B21D9D7F804315B09C7F8F430D7F8C9
:10526800043103F01F03002B04D1D7F8F430013BBD
:10527800C7F8F4307B6B1B889AB2D7F8F4309BB22E
:105288009B029BB213439BB26FEA43436FEA5343BB
:105298009AB27B6B1A8050E0D7F80431002B0AD100
:1052A8007B6B1B889BB26FEA43436FEA53439AB206
:1052B8007B6B1A8041E0D7F804315B08C7F8F430FB
:1052C800D7F8043103F00103002B04D0D7F8F430E9
:1052D8000133C7F8F4307B6B1B889AB2D7F8F430E7
:1052E8009BB29B029BB213439AB27B6B1A8024E059
:1052F80007F58473A3F584731B685B78012B1CD1B5
:1053080007F58473A3F582731B68B3F850309BB21A
:105318001A463B6C13443B6407F58473A3F5847306
:105328001B681B78DA003B6C134403F20643FB63EB
:10533800D7F804319AB2FB6B1A8007F58473A3F58A
:1053480084731B685B89A7F8763007F58473A3F527
:1053580084731B685969D7F804319BB2B7F8762073
:1053680007F58470A0F58270006801F07DF827E2E7
:1053780007F58473A3F584731B681B6AC7F80431A7
:1053880007F58473A3F582731A6807F58473A3F588
:1053980084731B681B789B0013441B889BB223F4FF
:1053A800E24323F07003A7F8623007F58473A3F58E
:1053B80082731A6807F58473A3F584731B681B78D6
:1053C8009B001A44B7F8623043F07F4343F47F03ED
:1053D80043F4004343F080039BB2138007F58473C2
:1053E800A3F582731B68FB6507F58473A3F58273C5
:1053F8001B68B3F850309BB21A46FB6D1344FB652B
:1054080007F58473A3F584731B681B78DA00FB6DBA
:10541800134403F20243BB65D7F804319AB2BB6D5B
:105428001A8007F58473A3F584731B681B89A7F892
:10543800763007F58473A3F584731B685969D7F828
:1054480004319BB2B7F8762007F58470A0F5827016
:10545800006801F009F8B3E107F58473A3F58473D4
:105468001B681A6AD7F80431D21A07F58473A3F5B2
:1054780084731B681A6207F58473A3F582731A682C
:1054880007F58473A3F584731B681B789B0013448A
:105498001B889BB203F04003002B00F0C68007F581
:1054A8008473A3F582731B683B6707F58473A3F5C0
:1054B80084731B685B78002B77D107F58473A3F599
:1054C80082731B68BB6607F58473A3F582731B6838
:1054D800B3F850309BB21A46BB6E1344BB6607F54F
:1054E8008473A3F584731B681B78DA00BB6E1344BE
:1054F80003F206437B667B6E1B889BB2C3F30903EA
:105508009AB27B6E1A80D7F804313E2B21D9D7F88E
:1055180004315B09C7F8F030D7F8043103F01F03F2
:10552800002B04D1D7F8F030013BC7F8F0307B6E80
:105538001B889AB2D7F8F0309BB29B029BB21343F8
:105548009BB26FEA43436FEA53439AB27B6E1A8069
:1055580050E0D7F80431002B0AD17B6E1B889BB230
:105568006FEA43436FEA53439AB27B6E1A8041E075
:10557800D7F804315B08C7F8F030D7F8043103F0E6
:105588000103002B04D0D7F8F0300133C7F8F0300E
:105598007B6E1B889AB2D7F8F0309BB29B029BB205
:1055A80013439AB27B6E1A8024E007F58473A3F53F
:1055B80084731B685B78012B1CD107F58473A3F5F2
:1055C80082731B68B3F850309BB21A463B6F134482
:1055D8003B6707F58473A3F584731B681B78DA00AF
:1055E8003B6F134403F20643FB66D7F804319AB2C3
:1055F800FB6E1A8007F58473A3F584731B685B89B7
:10560800A7F8763007F58473A3F584731B68596986
:10561800D7F804319BB2B7F8762007F58470A0F567
:105628008270006800F020FFCAE007F58473A3F5D4
:1056380084731B685B78002B77D107F58473A3F517
:1056480082731B68FB6707F58473A3F582731B6875
:10565800B3F850309BB21A46FB6F1344FB6707F54B
:105668008473A3F584731B681B78DA00FB6F1344FB
:1056780003F20243BB67BB6F1B889BB2C3F30903EA
:105688009AB2BB6F1A80D7F804313E2B21D9D7F8CC
:1056980004315B09C7F8EC30D7F8043103F01F0375
:1056A800002B04D1D7F8EC30013BC7F8EC30BB6FC6
:1056B8001B889AB2D7F8EC309BB29B029BB213437B
:1056C8009BB26FEA43436FEA53439AB2BB6F1A80A7
:1056D8005CE0D7F80431002B0AD1BB6F1B889BB262
:1056E8006FEA43436FEA53439AB2BB6F1A804DE0A7
:1056F800D7F804315B08C7F8EC30D7F8043103F069
:105708000103002B04D0D7F8EC300133C7F8EC3094
:10571800BB6F1B889AB2D7F8EC309BB29B029BB246
:1057280013439AB2BB6F1A8030E007F58473A3F570
:1057380084731B685B78012B28D107F58473A3F564
:1057480082731B68C7F8843007F58473A3F58273E6
:105758001B68B3F850309BB21A46D7F8843013440C
:10576800C7F8843007F58473A3F584731B681B7826
:10577800DA00D7F88430134403F20243C7F88030C4
:10578800D7F804319AB2D7F880301A8007F58473B5
:10579800A3F584731B681B89A7F8763007F5847313
:1057A800A3F584731B685969D7F804319BB2B7F81D
:1057B800762007F58470A0F58270006800F054FE2A
:1057C80007F58473A3F582731A6807F58473A3F544
:1057D80084731B681B789B0013441B889BB223F4BB
:1057E800E04323F040037B817B8983F010037B81B6
:1057F8007B8983F020037B8107F58473A3F582738B
:105808001A6807F58473A3F584731B681B789B00DB
:105818001A447B8943F07F4343F47F0343F40043F6
:1058280043F080039BB2138000F0DEBC07F584735D
:10583800A3F584731B681B7B002B40F0BB8007F526
:105848008473A3F584731B689A6907F58473A3F5B9
:1058580084731B681B699A4217D907F58473A3F5EB
:1058680084731B681B69C7F8043107F58473A3F5B3
:1058780084731B689A69D7F80431D21A07F58473C0
:10588800A3F584731B689A610EE007F58473A3F58A
:1058980084731B689B69C7F8043107F58473A3F503
:1058A80084731B6800229A6107F58473A3F58273D9
:1058B8001B68C7F8903007F58473A3F582731B68DB
:1058C800B3F850309BB21A46D7F890301344C7F853
:1058D800903007F58473A3F584731B681B78DA008E
:1058E800D7F89030134403F20643C7F88C30D7F842
:1058F8008C301B889BB2C3F309039AB2D7F88C305B
:105908001A80D7F804313E2B24D9D7F804315B0923
:10591800C7F8E830D7F8043103F01F03002B04D18F
:10592800D7F8E830013BC7F8E830D7F88C301B8847
:105938009AB2D7F8E8309BB29B029BB213439BB252
:105948006FEA43436FEA53439AB2D7F88C301A8010
:1059580000F010BCD7F80431002B0CD1D7F88C30EC
:105968001B889BB26FEA43436FEA53439AB2D7F856
:105978008C301A80FEE3D7F804315B08C7F8E830AA
:10598800D7F8043103F00103002B04D0D7F8E8302E
:105998000133C7F8E830D7F88C301B889AB2D7F8AB
:1059A800E8309BB29B029BB213439AB2D7F88C3073
:1059B8001A80DFE307F58473A3F584731B68DB782B
:1059C800022B40F0188207F58473A3F584731B68D3
:1059D8005B78002B40F09D8007F58473A3F58273F4
:1059E8001B68C7F8AC3007F58473A3F582731B688E
:1059F800B3F850309BB21A46D7F8AC301344C7F806
:105A0800AC3007F58473A3F584731B681B78DA0040
:105A1800D7F8AC30134403F20243C7F8A830D7F8DC
:105A2800A8301B889BB2C3F309039AB2D7F8A830F1
:105A38001A8007F58473A3F584731B681B693E2BD2
:105A48002BD907F58473A3F584731B681B695B095D
:105A5800C7F8E43007F58473A3F584731B681B69E2
:105A680003F01F03002B04D1D7F8E430013BC7F83B
:105A7800E430D7F8A8301B889AB2D7F8E4309BB244
:105A88009B029BB213439BB26FEA43436FEA5343B3
:105A98009AB2D7F8A8301A8070E007F58473A3F596
:105AA80084731B681B69002B0CD1D7F8A8301B889E
:105AB8009BB26FEA43436FEA53439AB2D7F8A830D0
:105AC8001A805BE007F58473A3F584731B681B6970
:105AD8005B08C7F8E43007F58473A3F584731B6883
:105AE8001B6903F00103002B04D0D7F8E43001331D
:105AF800C7F8E430D7F8A8301B889AB2D7F8E43052
:105B08009BB29B029BB213439AB2D7F8A8301A8073
:105B180034E007F58473A3F584731B685B78012B65
:105B28002CD107F58473A3F582731B68C7F8B430CA
:105B380007F58473A3F582731B68B3F850309BB2E2
:105B48001A46D7F8B4301344C7F8B43007F584734D
:105B5800A3F584731B681B78DA00D7F8B4301344B4
:105B680003F20243C7F8B03007F58473A3F58473D2
:105B78001B681B699AB2D7F8B0301A8007F584738E
:105B8800A3F582731B68C7F8A43007F58473A3F5DF
:105B980084731B685B78002B40F09D8007F5847345
:105BA800A3F582731B68C7F89C3007F58473A3F5C7
:105BB80082731B68B3F850309BB21A46D7F89C30F2
:105BC8001344C7F89C3007F58473A3F584731B68E6
:105BD8001B78DA00D7F89C30134403F20643C7F861
:105BE8009830D7F898301B889BB2C3F309039AB250
:105BF800D7F898301A8007F58473A3F584731B6867
:105C08001B693E2B2BD907F58473A3F584731B6896
:105C18001B695B09C7F8E03007F58473A3F5847343
:105C28001B681B6903F01F03002B04D1D7F8E03071
:105C3800013BC7F8E030D7F898301B889AB2D7F8FC
:105C4800E0309BB29B029BB213439BB26FEA434383
:105C58006FEA53439AB2D7F898301A8069E007F58B
:105C68008473A3F584731B681B69002B0CD1D7F8C8
:105C780098301B889BB26FEA43436FEA53439AB24A
:105C8800D7F898301A8054E007F58473A3F5847325
:105C98001B681B695B08C7F8E03007F58473A3F538
:105CA80084731B681B6903F00103002B04D0D7F829
:105CB800E0300133C7F8E030D7F898301B889AB243
:105CC800D7F8E0309BB29B029BB213439AB2D7F845
:105CD80098301A802DE007F58473A3F584731B6848
:105CE8005B78012B25D107F58473A3F582731B68B4
:105CF800B3F850309BB21A46D7F8A4301344C7F80B
:105D0800A43007F58473A3F584731B681B78DA0045
:105D1800D7F8A430134403F20643C7F8A03007F5B8
:105D28008473A3F584731B681B699AB2D7F8A030F3
:105D38001A8007F58473A3F584731B68DB69002B4D
:105D480000F0188207F58473A3F582731A6807F5C3
:105D58008473A3F584731B681B789B0013441B880A
:105D6800A7F89630B7F8963003F48043002B05D097
:105D7800B7F8963003F04003002B0DD1B7F89630F2
:105D880003F48043002B40F0F581B7F8963003F018
:105D98004003002B40F0EE8107F58473A3F582736E
:105DA8001A6807F58473A3F584731B681B789B0036
:105DB80013441B889BB223F4E04323F07003A7F835
:105DC800943007F58473A3F582731A6807F5847312
:105DD800A3F584731B681B789B001A44B7F89430AA
:105DE80043F07F4343F47F0343F4004343F0C0038D
:105DF8009BB21380BEE107F58473A3F584731B6817
:105E0800DB78012B40F0B48107F58473A3F5847324
:105E18001B689A6907F58473A3F584731B681B696B
:105E28009A4217D907F58473A3F584731B681B6915
:105E3800C7F8043107F58473A3F584731B689A695E
:105E4800D7F80431D21A07F58473A3F584731B6855
:105E58009A610EE007F58473A3F584731B689B6948
:105E6800C7F8043107F58473A3F584731B6800220F
:105E78009A6107F58473A3F584731B685B78002B1C
:105E880040F0858007F58473A3F582731B68C7F813
:105E9800CC3007F58473A3F582731B68B3F85030D0
:105EA8009BB21A46D7F8CC301344C7F8CC3007F564
:105EB8008473A3F584731B681B78DA00D7F8CC3099
:105EC800134403F20243C7F8C830D7F8C8301B8818
:105ED8009BB2C3F309039AB2D7F8C8301A80D7F82F
:105EE80004313E2B23D9D7F804315B09C7F8DC30DD
:105EF800D7F8043103F01F03002B04D1D7F8DC30A6
:105F0800013BC7F8DC30D7F8C8301B889AB2D7F8FD
:105F1800DC309BB29B029BB213439BB26FEA4343B4
:105F28006FEA53439AB2D7F8C8301A8060E0D7F8BE
:105F38000431002B0CD1D7F8C8301B889BB26FEA0C
:105F480043436FEA53439AB2D7F8C8301A804FE0F8
:105F5800D7F804315B08C7F8DC30D7F8043103F010
:105F68000103002B04D0D7F8DC300133C7F8DC304C
:105F7800D7F8C8301B889AB2D7F8DC309BB29B029E
:105F88009BB213439AB2D7F8C8301A8030E007F5AD
:105F98008473A3F584731B685B78012B28D107F5FC
:105FA8008473A3F582731B68C7F8D43007F584732C
:105FB800A3F582731B68B3F850309BB21A46D7F822
:105FC800D4301344C7F8D43007F58473A3F5847329
:105FD8001B681B78DA00D7F8D430134403F2024365
:105FE800C7F8D030D7F804319AB2D7F8D0301A8031
:105FF80007F58473A3F582731B68C7F8C43007F5E7
:106008008473A3F584731B685B78002B40F085804C
:1060180007F58473A3F582731B68C7F8BC3007F5CE
:106028008473A3F582731B68B3F850309BB21A4689
:10603800D7F8BC301344C7F8BC3007F58473A3F510
:1060480084731B681B78DA00D7F8BC30134403F25A
:106058000643C7F8B830D7F8B8301B889BB2C3F3EB
:1060680009039AB2D7F8B8301A80D7F804313E2B12
:1060780023D9D7F804315B09C7F8D830D7F80431E9
:1060880003F01F03002B04D1D7F8D830013BC7F821
:10609800D830D7F8B8301B889AB2D7F8D8309BB226
:1060A8009B029BB213439BB26FEA43436FEA53438D
:1060B8009AB2D7F8B8301A805CE0D7F80431002BD0
:1060C8000CD1D7F8B8301B889BB26FEA43436FEA0C
:1060D80053439AB2D7F8B8301A804BE0D7F8043156
:1060E8005B08C7F8D830D7F8043103F00103002B58
:1060F80004D0D7F8D8300133C7F8D830D7F8B8303B
:106108001B889AB2D7F8D8309BB29B029BB2134334
:106118009AB2D7F8B8301A802CE007F58473A3F543
:1061280084731B685B78012B24D107F58473A3F56E
:1061380082731B68B3F850309BB21A46D7F8C43044
:106148001344C7F8C43007F58473A3F584731B6838
:106158001B78DA00D7F8C430134403F20643C7F8B3
:10616800C030D7F804319AB2D7F8C0301A8001E0AD
:1061780001233AE007F58473A3F582731A6807F5DB
:106188008473A3F584731B681B789B0013441B88D6
:106198009BB223F4804323F07003A7F88A30B7F842
:1061A8008A3083F48053A7F88A30B7F88A3083F4AA
:1061B8000053A7F88A3007F58473A3F582731A6829
:1061C80007F58473A3F584731B681B789B001A4436
:1061D800B7F88A3043F07F4343F47F0343F4004326
:1061E80043F080039BB213800023184607F5847799
:1061F800BD4680BD80B485B000AF786039603B682B
:106208005B78002B20D07A683B681B789B0013448E
:106218001B889BB223F4E04323F04003BB81BB8976
:1062280083F01003BB817A683B681B789B001A4493
:10623800BB8943F07F4343F47F0343F4004343F0B7
:1062480080039BB213801FE07A683B681B789B0031
:1062580013441B889BB223F4804323F07003FB8113
:10626800FB8983F48053FB817A683B681B789B0029
:106278001A44FB8943F07F4343F47F0343F400430C
:1062880043F080039BB21380002318461437BD46A1
:106298005DF8047B704780B487B000AF78603960E0
:1062A8003B681B7B002B40F09D803B685B78002B94
:1062B8004CD07A683B681B789B0013441B883B8250
:1062C8003B8A03F04003002B1BD07A683B681B789D
:1062D8009B0013441B889BB223F4E04323F0700314
:1062E800FB817A683B681B789B001A44FB8943F062
:1062F8007F4343F47F0343F4004343F0C0039BB25E
:1063080013803B68DB78012B6CD07A683B681B787C
:106318009B0013441B889BB223F4E04323F0400303
:10632800BB81BB8983F02003BB817A683B681B78FB
:106338009B001A44BB8943F07F4343F47F0343F433
:10634800004343F080039BB213804BE07A683B68BC
:106358001B789B0013441B88FB82FB8A03F4804351
:10636800002B1BD07A683B681B789B0013441B8862
:106378009BB223F4E04323F07003BB827A683B6846
:106388001B789B001A44BB8A43F07F4343F47F0386
:1063980043F4404343F080039BB213807A683B6820
:1063A8001B789B0013441B889BB223F4804323F083
:1063B80070037B827B8A83F480537B827B8A83F49D
:1063C80000537B827A683B681B789B001A447B8A5F
:1063D80043F07F4343F47F0343F4004343F08003D7
:1063E8009BB21380002318461C37BD465DF8047B1A
:1063F800704780B483B000AF78600B46FB70FB78C1
:10640800002B03D17B688022A3F84C200023184678
:106418000C37BD465DF8047B704780B483B000AF8D
:1064280078607B68B3F858309BB26FEA43436FEAF1
:1064380053439AB27B68A3F85820002318460C37B8
:10644800BD465DF8047B704780B485B000AF7860C6
:106458007B68B3F844309BB2FB60FB68184614377E
:10646800BD465DF8047B704780B48BB000AFF86020
:10647800B96011461A460B46FB801346BB80BB88A1
:1064880001335B08BB61FB687B61BB68FB61FA8811
:106498007B69134403F580633B62BB697B621BE045
:1064A800FB691B787B82FB6901331B781B021AB2DC
:1064B800B7F9123013431BB27B823B6A7A8A1A807F
:1064C8003B6A02333B62FB690133FB61FB690133C1
:1064D800FB617B6A013B7B627B6A002BE0D100BFDA
:1064E80000BF2C37BD465DF8047B704780B48BB085
:1064F80000AFF860B96011461A460B46FB80134698
:10650800BB80BB885B089BB2BB61FB687B61BB68D7
:10651800FB61FA887B69134403F580633B62BB69BE
:106528007B6218E03B6A1B889BB23B613B6A023383
:106538003B623B69DAB2FB691A70FB690133FB61A4
:106548003B691B0ADAB2FB691A70FB690133FB610C
:106558007B6A013B7B627B6A002BE3D1BB8803F03B
:1065680001039BB2002B07D03B6A1B889BB23B619F
:106578003B69DAB2FB691A7000BF2C37BD465DF87B
:10658800047B704780B582B000AF0023FB71032005
:1065980001F070FD0F2000F00DF80346002B02D02B
:1065A8000123FB7101E0FBF739FAFB79184608373C
:1065B800BD4680BD80B584B000AF78600023FB7312
:1065C800164B1B68002B22D0154B1A68134B1B68FF
:1065D8004FF47A71B1FBF3F3B2FBF3F3184601F011
:1065E8007CFD0346002B0FD17B680F2B09D80022B6
:1065F80079684FF0FF3001F048FD0A4A7B68136064
:1066080007E00123FB7304E00123FB7301E001238E
:10661800FB73FB7B18461037BD4680BD6C0000201D
:10662800700000206800002080B400AF054B1A6895
:10663800054B1B681344034A136000BFBD465DF851
:10664800047B7047481F00206C00002080B400AF16
:10665800034B1B681846BD465DF8047B704700BFB6
:10666800481F002080B588B000AF78607B68002B99
:1066780001D10123FEE27B681B6803F00103002BB4
:1066880075D0974B9B6803F00C03BB61944BDB6898
:1066980003F003037B61BB690C2B02D17B69032BDD
:1066A80002D0BB69082B0BD18D4B1B6803F4003358
:1066B800002B5BD07B685B68002B57D10123D9E2A4
:1066C8007B685B68B3F5803F06D1854B1B68844ABD
:1066D80043F4803313601DE07B685B68B3F5A02F3B
:1066E8000CD17F4B1B687E4A43F4802313607C4B9C
:1066F8001B687B4A43F4803313600BE0784B1B68BC
:10670800774A23F480331360754B1B68744A23F46B
:10671800802313607B685B68002B13D0FFF796FF1C
:10672800386108E0FFF792FF02463B69D31A642BF1
:1067380001D903239EE26A4B1B6803F40033002B44
:10674800F0D014E0FFF782FF386108E0FFF77EFF22
:1067580002463B69D31A642B01D903238AE2604BB2
:106768001B6803F40033002BF0D100E000BF7B6806
:106778001B6803F00203002B75D0594B9B6803F08C
:106788000C03BB61564BDB6803F003037B61BB69F9
:106798000C2B02D17B69022B02D0BB69042B1FD1C1
:1067A8004F4B1B6803F48063002B05D07B68DB68C4
:1067B800002B01D101235DE2494B5B6823F0FE42C7
:1067C8007B681B691B06464913434B60454B1B6896
:1067D8001846FFF7EFFE0346002B43D0012349E29A
:1067E8007B68DB68002B23D03D4B1B683C4A43F495
:1067F80080731360FFF72AFF386108E0FFF726FF70
:1068080002463B69D31A022B01D9032332E2344BE7
:106818001B6803F48063002BF0D0314B5B6823F0D6
:10682800FE427B681B691B062D4913434B601AE027
:106838002B4B1B682A4A23F480731360FFF706FF6B
:10684800386108E0FFF702FF02463B69D31A022BC2
:1068580001D903230EE2224B1B6803F48063002B4B
:10686800F0D100E000BF7B681B6803F00803002B31
:1068780041D07B685B69002B1CD0194BD3F894304E
:10688800174A43F00103C2F89430FFF7DFFE38617E
:1068980008E0FFF7DBFE02463B69D31A022B01D959
:1068A8000323E7E10E4BD3F8943003F00203002BE7
:1068B800EFD020E00A4BD3F89430094A23F00103C3
:1068C800C2F89430FFF7C2FE38610DE0FFF7BEFE54
:1068D80002463B69D31A022B06D90323CAE100BF3B
:1068E80000100240680000208C4BD3F8943003F06D
:1068F8000203002BEAD17B681B6803F00403002B1A
:1069080000F0A6800023FB77844B9B6D03F0805337
:10691800002B01D1012300E00023002B0DD07F4B79
:106928009B6D7E4A43F0805393657C4B9B6D03F0CF
:106938008053FB60FB680123FB77794B1B6803F4EA
:106948008073002B18D1764B1B68754A43F480730B
:106958001360FFF77BFE386108E0FFF777FE024619
:106968003B69D31A022B01D9032383E16C4B1B68C3
:1069780003F48073002BF0D07B689B68012B08D14F
:10698800664BD3F89030654A43F00103C2F8903063
:1069980024E07B689B68052B10D1604BD3F89030BE
:1069A8005E4A43F00403C2F890305C4BD3F8903051
:1069B8005A4A43F00103C2F890300FE0574BD3F81E
:1069C8009030564A23F00103C2F89030534BD3F865
:1069D8009030524A23F00403C2F890307B689B68D9
:1069E800002B16D0FFF732FE38610AE0FFF72EFEC3
:1069F80002463B69D31A41F28832934201D90323F4
:106A080038E1464BD3F8903003F00203002BEDD069
:106A180015E0FFF71BFE38610AE0FFF717FE024694
:106A28003B69D31A41F28832934201D9032321E109
:106A38003A4BD3F8903003F00203002BEDD1FB7FE3
:106A4800012B05D1354B9B6D344A23F08053936558
:106A58007B681B6803F02003002B3CD07B689B6994
:106A6800002B1CD02D4BD3F898302C4A43F001034F
:106A7800C2F89830FFF7EAFD386108E0FFF7E6FD55
:106A880002463B69D31A022B01D90323F2E0234BB8
:106A9800D3F8983003F00203002BEFD01BE01F4B14
:106AA800D3F898301D4A23F00103C2F89830FFF755
:106AB800CDFD386108E0FFF7C9FD02463B69D31AEE
:106AC800022B01D90323D5E0144BD3F8983003F0F7
:106AD8000203002BEFD17B68DB69002B00F0C98033
:106AE8000E4B9B6803F00C030C2B00F083807B6833
:106AF800DB69022B5ED1094B1B68084A23F08073BF
:106B08001360FFF7A3FD38610CE0FFF79FFD024615
:106B18003B69D31A022B05D90323ABE000100240CE
:106B280000700040554B1B6803F00073002BECD13C
:106B3800524BDA68524B13407A68116A7A68526A83
:106B4800013A120111437A68926A120211437A6873
:106B5800126B5208013A520511437A68526B520877
:106B6800013A520611437A68D26AD2060A43434967
:106B78001343CB60414B1B68404A43F0807313605A
:106B88003E4BDB683D4A43F08073D360FFF75EFD00
:106B9800386108E0FFF75AFD02463B69D31A022B19
:106BA80001D9032366E0354B1B6803F00073002B03
:106BB800F0D05EE0314B1B68304A23F080731360DD
:106BC800FFF744FD386108E0FFF740FD02463B69E6
:106BD800D31A022B01D903234CE0284B1B6803F07E
:106BE8000073002BF0D1254BDA682449254B13405C
:106BF800CB603EE07B68DB69012B01D1012339E0E2
:106C08001E4BDB687B617B6903F003027B681B6AB0
:106C18009A422CD17B6903F0F0027B685B6A013BE6
:106C28001B019A4223D17B6903F4FE427B689B6A6D
:106C38001B029A421BD17B6903F078427B68DB6AAE
:106C4800DB069A4213D17B6903F4C0027B681B6B95
:106C58005B08013B5B059A4209D17B6903F0C0627E
:106C68007B685B6B5B08013B5B069A4201D00123A2
:106C780000E0002318462037BD4680BD00100240C2
:106C88000C809F01FCFFEEFE80B586B000AF7860F7
:106C9800396000237B617B68002B01D101231EE151
:106CA800914B1B6803F00F033A689A4210D98E4B38
:106CB8001B6823F00F028C493B6813430B608A4B17
:106CC8001B6803F00F033A689A4201D0012306E1DA
:106CD8007B681B6803F00103002B73D07B685B683B
:106CE800032B29D1814B1B6803F00073002B01D1C2
:106CF8000123F4E000F09CF938613B697C4A934237
:106D08003FD97A4B9B6803F0F003002B09D07B68CE
:106D18001B6803F00203002B33D07B689B68002BB1
:106D28002FD1724B9B6823F0F003704A43F0800325
:106D3800936080237B6124E07B685B68022B07D12A
:106D48006A4B1B6803F40033002B09D10123C6E00A
:106D5800664B1B6803F48063002B01D10123BEE05E
:106D680000F0CEF838613B69614A934209D95F4B1C
:106D78009B6823F0F0035D4A43F08003936080230F
:106D88007B615A4B9B6823F003027B685B68574919
:106D980013438B60FFF75AFCF8600AE0FFF756FCD4
:106DA8000246FB68D31A41F28832934201D9032381
:106DB80095E04E4B9B6803F00C027B685B689B0078
:106DC8009A42EBD17B681B6803F00203002B23D0A7
:106DD8007B681B6803F00403002B05D0434B9B68BA
:106DE800424A43F4E06393607B681B6803F008033E
:106DF800002B07D03D4B9B6823F47C533B4A43F45C
:106E0800E0639360394B9B6823F0F0027B689B68D2
:106E1800364913438B6008E07B69802B05D1334BDF
:106E28009B68324A23F0F00393602F4B1B6803F0F2
:106E38000F033A689A421DD22B4B1B6823F00F02AE
:106E480029493B6813430B60FFF700FCF8600AE030
:106E5800FFF7FCFB0246FB68D31A41F288329342E3
:106E680001D903233BE0204B1B6803F00F033A686A
:106E78009A42EDD17B681B6803F00403002B08D00D
:106E88001A4B9B6823F4E0627B68DB68174913435D
:106E98008B607B681B6803F00803002B09D0134B39
:106EA8009B6823F460527B681B69DB000F4913431E
:106EB8008B6000F025F802460C4B9B681B0903F019
:106EC8000F030C49CB5C03F01F0322FA03F30A4AB1
:106ED80013600A4B1B681846FFF76CFB03461846FD
:106EE8001837BD4680BD00BF002002400010024098
:106EF80000B4C40490D60108700000206800002087
:106F080080B487B000AF2C4B9B6803F00C03042BB4
:106F180002D12A4B3B6147E0274B9B6803F00C03E7
:106F2800082B02D1254B3B613EE0234B9B6803F0C5
:106F38000C030C2B36D1204BDB6803F00303FB60FA
:106F48001D4BDB681B0903F00F030133BB60FB68B3
:106F5800032B0CD1194ABB68B2FBF3F3164AD2686B
:106F6800120A02F07F0202FB03F37B610CE0134A72
:106F7800BB68B2FBF3F3104AD268120A02F07F0230
:106F880002FB03F37B6100BF0B4BDB685B0E03F076
:106F9800030301335B007B607A697B68B2FBF3F320
:106FA8003B6101E000233B613B6918461C37BD4645
:106FB8005DF8047B704700BF001002400024F40015
:106FC80080B400AF034B1B681846BD465DF8047BD0
:106FD800704700BF7000002080B500AFFFF7F0FFDA
:106FE8000246064B9B681B0A03F007030449CB5C67
:106FF80003F01F0322FA03F3184680BD0010024075
:10700800A0D6010880B500AFFFF7DAFF0246064BAD
:107018009B68DB0A03F007030449CB5C03F01F03FA
:1070280022FA03F3184680BD00100240A0D60108DA
:1070380080B487B000AF1E4BDB6803F003033B61ED
:107048001B4BDB681B0903F00F030133FB603B6933
:10705800032B0CD1174AFB68B2FBF3F3144AD2682E
:10706800120A02F07F0202FB03F37B610CE0114A73
:10707800FB68B2FBF3F30E4AD268120A02F07F02F1
:1070880002FB03F37B6100BF094BDB685B0E03F077
:10709800030301335B00BB607A69BB68B2FBF3F39F
:1070A8007B607B6818461C37BD465DF8047B7047DB
:1070B800001002400024F40080B586B000AF78606C
:1070C8000023FB740023BB747B681B6803F4002354
:1070D800002B00F0988000237B74434B9B6D03F0DA
:1070E8008053002B0DD1404B9B6D3F4A43F080539A
:1070F80093653D4B9B6D03F08053BB60BB680123D8
:107108007B743A4B1B68394A43F480731360FFF76A
:107118009DFAF86009E0FFF799FA0246FB68D31A6E
:10712800022B02D90323FB7405E0304B1B6803F4E0
:107138008073002BEFD0FB7C002B59D12A4BD3F85E
:10714800903003F440737B617B69002B1ED07B6811
:107158001B6D7A699A4219D0234BD3F8903023F4E7
:1071680040737B61204BD3F890301F4A43F480333F
:10717800C2F890301C4BD3F890301B4A23F480336C
:10718800C2F89030184A7B69C2F890307B6903F0E6
:107198000103002B16D0FFF759FAF8600BE0FFF750
:1071A80055FA0246FB68D31A41F28832934202D953
:1071B8000323FB7406E00C4BD3F8903003F0020372
:1071C800002BECD0FB7C002B0BD1074BD3F8903075
:1071D80023F440727B681B6D03491343C1F8903058
:1071E80008E0FB7CBB7405E0001002400070004022
:1071F800FB7CBB747B7C012B05D1A74B9B6DA64AFE
:1072080023F0805393657B681B6803F00103002B10
:107218000AD0A14BD3F8883023F003027B685B685F
:107228009D491343C1F888307B681B6803F002034B
:10723800002B0AD0984BD3F8883023F00C027B68D7
:107248009B6895491343C1F888307B681B6803F035
:107258000403002B0AD0904BD3F8883023F0300277
:107268007B68DB688C491343C1F888307B681B68EE
:1072780003F00803002B0AD0874BD3F8883023F09B
:10728800C0027B681B6984491343C1F888307B6856
:107298001B6803F01003002B0AD07F4BD3F888300B
:1072A80023F440727B685B697B491343C1F88830DB
:1072B8007B681B6803F02003002B0AD0764BD3F8B9
:1072C800883023F440627B689B6973491343C1F893
:1072D80088307B681B6803F04003002B0AD06E4B94
:1072E800D3F8883023F440527B68DB696A4913433A
:1072F800C1F888307B681B6803F08003002B0AD034
:10730800654BD3F8883023F440427B681B6A624996
:107318001343C1F888307B681B6803F48073002B23
:107328000AD05D4BD3F8883023F440327B685B6A1F
:1073380059491343C1F888307B681B6803F400334C
:10734800002B0AD0544BD3F89C3023F003027B68FF
:107358009B6A51491343C1F89C307B681B6803F44E
:107368000073002B0AD04C4BD3F8883023F440220A
:107378007B68DB6A48491343C1F888307B681B681F
:1073880003F48063002B15D0434BD3F8883023F4E3
:1073980040127B681B6B40491343C1F888307B68F7
:1073A8001B6BB3F5801F05D13B4BDB683A4A43F4AE
:1073B8008013D3607B681B6803F40063002B15D02F
:1073C800354BD3F8883023F440027B685B6B324935
:1073D8001343C1F888307B685B6BB3F5800F05D128
:1073E8002D4BDB682C4A43F48013D3607B681B6801
:1073F80003F48053002B15D0274BD3F8883023F0A3
:1074080040727B689B6B24491343C1F888307B68C2
:107418009B6BB3F1807F05D11F4BDB681E4A43F499
:107428008013D3607B681B6803F40053002B15D0CE
:10743800194BD3F8883023F040627B68DB6B164920
:107448001343C1F888307B68DB6BB3F1006F05D15B
:10745800114BDB68104A43F48013D3607B681B68C8
:1074680003F48043002B19D00B4BD3F8883023F05A
:1074780040627B681B6C08491343C1F888307B68FD
:107488001B6CB3F1006F09D1034BDB68024A43F46C
:107498008013D36002E000BF001002407B681B68C5
:1074A80003F40043002B15D0294BD3F8883023F080
:1074B80040527B685B6C26491343C1F888307B686F
:1074C8005B6CB3F1805F05D1214BDB68204A43F444
:1074D8008033D3607B681B6803F48033002B15D09E
:1074E8001B4BD3F8883023F040427B689B6C1849CB
:1074F8001343C1F888307B689B6CB3F1804F05D18A
:10750800134BDB68124A43F48033D3607B681B68F3
:1075180003F48023002B15D00D4BD3F89C3023F4B3
:1075280040127B68DB6C0A491343C1F89C307B68C6
:10753800DB6CB3F5001F05D1054BDB68044A43F447
:107548008013D360BB7C18461837BD4680BD00BF8A
:107558000010024080B487B000AF78603960002323
:107568007B615AE13B681A6801217B6901FA03F3E0
:107578001340FB60FB68002B00F04C813B685B68A4
:1075880003F00303012B05D03B685B6803F003039A
:10759800022B30D17B689B683B617B695B000322CF
:1075A80002FA03F3DB433A6913403B613B68DA684C
:1075B8007B695B0002FA03F33A6913433B617B681A
:1075C8003A699A607B685B683B6101227B6902FAD1
:1075D80003F3DB433A6913403B613B685B681B0973
:1075E80003F001027B6902FA03F33A6913433B6132
:1075F8007B683A695A603B685B6803F00303032BB6
:1076080017D07B68DB683B617B695B00032202FA69
:1076180003F3DB433A6913403B613B689A687B6933
:107628005B0002FA03F33A6913433B617B683A69EA
:10763800DA603B685B6803F00303022B23D17B69A4
:10764800DA087B68083253F822303B617B6903F023
:1076580007039B000F2202FA03F3DB433A69134046
:107668003B613B681A697B6903F007039B0002FAD8
:1076780003F33A6913433B617B69DA087B68083294
:10768800396943F822107B681B683B617B695B00A2
:10769800032202FA03F3DB433A6913403B613B6878
:1076A8005B6803F003027B695B0002FA03F33A6943
:1076B80013433B617B683A691A603B685B6803F473
:1076C8004033002B00F0A6805B4B1B6E5A4A43F0F8
:1076D80001031366584B1B6E03F00103BB60BB68C4
:1076E800564A7B699B08023352F823303B617B6919
:1076F80003F003039B000F2202FA03F3DB433A690A
:1077080013403B617B68B3F1904F1FD07B684C4AB4
:10771800934219D07B684B4A934213D07B684A4AFC
:1077280093420DD07B68494A934207D07B68484A08
:10773800934201D105230AE0062308E0042306E06A
:10774800032304E0022302E0012300E000237A6916
:1077580002F00302920093403A6913433B613749B0
:107768007B699B0802333A6941F82320394B9B68AF
:107778003B61FB68DB433A6913403B613B685B68EC
:1077880003F48013002B03D03A69FB6813433B6171
:10779800304A3B6993602F4BDB683B61FB68DB43F6
:1077A8003A6913403B613B685B6803F40013002BA4
:1077B80003D03A69FB6813433B61264A3B69D360AF
:1077C800244B5B683B61FB68DB433A6913403B61D0
:1077D8003B685B6803F40033002B03D03A69FB680D
:1077E80013433B611B4A3B6953601A4B1B683B615F
:1077F800FB68DB433A6913403B613B685B6803F411
:107808008033002B03D03A69FB6813433B61114A6C
:107818003B6913607B6901337B613B681A687B694C
:1078280022FA03F3002B7FF49DAE00BF00BF1C3784
:10783800BD465DF8047B704700100240000001401F
:107848000004004800080048000C004800100048E8
:10785800001400480004014080B485B000AF78608F
:107868000B467B807B681A697B881340002B02D00B
:107878000123FB7301E00023FB73FB7B18461437DD
:10788800BD465DF8047B704780B584B000AF786072
:107898007B68002B01D101238DE07B681B681A46A9
:1078A800474B9A420FD87B681B681A46454B1344CE
:1078B800454AA2FB03231B099A007B685A647B682C
:1078C800424A1A640EE07B681B681A46404B134410
:1078D8003D4AA2FB03231B099A007B685A647B6814
:1078E8003C4A1A647B68022283F825207B681B685F
:1078F8001B68FB60FB6823F4FF4323F07003FB6005
:107908007B689A687B68DB681A437B681B691A4343
:107918007B685B691A437B689B691A437B68DB69F0
:107928001A437B681B6A1343FA681343FB607B683E
:107938001B68FA681A60786800F0B6F97B689B687B
:10794800B3F5804F02D17B6800225A607B685A6881
:107958007B689B6CD2B21A607B68DB6C7A68126DAC
:107968005A607B685B68002B10D07B685B68042BCF
:107978000CD8786800F0D6F97B685B6D00221A6035
:107988007B689B6D7A68D26D5A6008E07B6800223C
:107998005A657B6800229A657B680022DA657B68F5
:1079A8000022DA637B68012283F825207B680022A5
:1079B80083F82420002318461037BD4680BD00BF39
:1079C80007040240F8FFFDBFCDCCCCCC000002403C
:1079D800F8FBFDBF0004024080B586B000AFF86038
:1079E800B9607A603B600023FB75FB6893F824302C
:1079F800012B01D1022366E0FB68012283F82420D1
:107A0800FB6893F82530DBB2012B55D1FB680222C5
:107A180083F82520FB680022DA63FB681B681A6874
:107A2800FB681B6822F001021A603B687A68B96833
:107A3800F86800F0FBF8FB681B6B002B08D0FB68AC
:107A48001B681A68FB681B6842F00E021A600FE098
:107A5800FB681B681A68FB681B6822F004021A603E
:107A6800FB681B681A68FB681B6842F00A021A6008
:107A7800FB689B6C1B6803F48033002B07D0FB6802
:107A88009B6C1A68FB689B6C42F480721A60FB68F6
:107A98005B6D002B07D0FB685B6D1A68FB685B6D3C
:107AA80042F480721A60FB681B681A68FB681B68DE
:107AB80042F001021A6005E0FB68002283F82420E6
:107AC8000223FB75FB7D18461837BD4680BD80B57F
:107AD80084B000AF78607B681B6C1B68FB607B68B8
:107AE8001B681B68BB607B685B6C03F01F03042288
:107AF8009A40FB681340002B26D0BB6803F00403B0
:107B0800002B21D07B681B681B6803F02003002B27
:107B180007D17B681B681A687B681B6822F004021F
:107B28001A607B685B6C03F01F027B681B6C042186
:107B380001FA02F25A607B681B6B002B71D07B68DC
:107B48001B6B786898476CE07B685B6C03F01F03DD
:107B580002229A40FB681340002B2ED0BB6803F02A
:107B68000203002B29D07B681B681B6803F02003E5
:107B7800002B0BD17B681B681A687B681B6822F096
:107B88000A021A607B68012283F825207B685B6CF7
:107B980003F01F027B681B6C022101FA02F25A6093
:107BA8007B68002283F824207B68DB6A002B38D0AE
:107BB8007B68DB6A7868984733E07B685B6C03F026
:107BC8001F0308229A40FB681340002B2AD0BB6889
:107BD80003F00803002B25D07B681B681A687B68B4
:107BE8001B6822F00E021A607B685B6C03F01F02B0
:107BF8007B681B6C012101FA02F25A607B68012242
:107C0800DA637B68012283F825207B68002283F8E9
:107C180024207B685B6B002B04D07B685B6B7868E7
:107C2800984700BF00BF1037BD4680BD80B485B0FF
:107C380000AFF860B9607A603B60FB68DB6CFA689B
:107C4800126D5A60FB685B6D002B04D0FB689B6D5E
:107C5800FA68D26D5A60FB685B6C03F01F02FB6820
:107C68001B6C012101FA02F25A60FB681B683A6832
:107C78005A60FB689B68102B08D1FB681B687A6800
:107C88009A60FB681B68BA68DA6007E0FB681B68E3
:107C9800BA689A60FB681B687A68DA6000BF1437B4
:107CA800BD465DF8047B704780B487B000AF78604C
:107CB8007B681B681A46164B9A4202D8154B7B61A3
:107CC80001E0154B7B617B693B617B681B68DBB21C
:107CD800083B124AA2FB03231B09FB607B685B6C11
:107CE8009B089A003B6913441A467B689A647B6830
:107CF8000B4ADA64FB6803F01F0301229A407B6891
:107D08001A6500BF1C37BD465DF8047B704700BF8D
:107D1800070402400008024020080240CDCCCCCC29
:107D28008008024080B485B000AF78607B685B68EB
:107D3800DBB2FB60FA680B4B13449B001A467B6866
:107D48005A657B68084A9A65FB68013B03F01F0384
:107D580001229A407B68DA6500BF1437BD465DF89A
:107D6800047B70473F8200104009024080B485B010
:107D780000AF78607B68002B41D14B4B1B6803F444
:107D8800C063B3F5806F31D1474BD3F88030464A92
:107D980023F48073C2F88030434B1B6823F4C0631C
:107DA800414A43F400731360404B1B68322202FBC4
:107DB80003F33F4AA2FB03239B0C0133FB6002E061
:107DC800FB68013BFB60384B5B6903F48063B3F5E8
:107DD800806F02D1FB68002BF2D1334B5B6903F44F
:107DE8008063B3F5806F58D1032357E02E4BD3F847
:107DF80080302D4A23F48073C2F880304DE07B68D0
:107E0800B3F5007F41D1284B1B6803F4C063B3F579
:107E1800806F31D1244BD3F88030234A43F48073E8
:107E2800C2F88030204B1B6823F4C0631E4A43F419
:107E3800007313601D4B1B68322202FB03F31C4ABC
:107E4800A2FB03239B0C0133FB6002E0FB68013BB0
:107E5800FB60154B5B6903F48063B3F5806F02D157
:107E6800FB68002BF2D1104B5B6903F48063B3F518
:107E7800806F12D1032311E00B4BD3F880300A4AEC
:107E880043F48073C2F8803007E0074B1B6823F483
:107E9800C063054A43F4806313600023184614370F
:107EA800BD465DF8047B70470070004070000020FC
:107EB80083DE1B4380B400AF054B9B68044A43F440
:107EC8008043936000BFBD465DF8047B704700BFE8
:107ED8000070004080B485B000AF78607B6803F024
:107EE8000703FB600C4BDB68BB60BA684FF6FF0307
:107EF8001340BB60FB681A02BB68134343F0BF63BF
:107F080043F40033BB60044ABB68D36000BF143736
:107F1800BD465DF8047B704700ED00E080B400AF1B
:107F2800044BDB681B0A03F007031846BD465DF8DF
:107F3800047B704700ED00E080B483B000AF0346D7
:107F4800FB7197F90730002B0BDBFB7903F01F025D
:107F5800074997F907305B09012000FA02F241F856
:107F6800232000BF0C37BD465DF8047B704700BF77
:107F780000E100E080B483B000AF03463960FB71D4
:107F880097F90730002B0ADB3B68DAB20C4997F9FE
:107F980007301201D2B20B4483F800230AE03B6891
:107FA800DAB20849FB7903F00F03043B1201D2B29D
:107FB8000B441A7600BF0C37BD465DF8047B70474A
:107FC80000E100E000ED00E080B489B000AFF860A7
:107FD800B9607A60FB6803F00703FB61FB69C3F1D2
:107FE8000703042B28BF0423BB61FB690433062B5A
:107FF80002D9FB69033B00E000237B614FF0FF32AD
:10800800BB6902FA03F3DA43BB681A407B699A40FA
:108018004FF0FF317B6901FA03F3D9437B680B40CA
:10802800134318462437BD465DF8047B70470000AB
:1080380080B582B000AF78607B68013BB3F1807F88
:1080480001D301230FE00A4A7B68013B53600F21EB
:108058004FF0FF30FFF78EFF054B00229A60044B6C
:1080680007221A60002318460837BD4680BD00BFA6
:1080780010E000E080B582B000AF78607868FFF764
:1080880029FF00BF0837BD4680BD80B586B000AF68
:108098000346B9607A60FB73FFF740FF78617A683E
:1080A800B9687869FFF790FF024697F90F301146D3
:1080B8001846FFF75FFF00BF1837BD4680BD80B583
:1080C80082B000AF0346FB7197F907301846FFF7F7
:1080D80033FF00BF0837BD4680BD80B582B000AF12
:1080E80078607868FFF7A4FF034618460837BD464E
:1080F80080BD80B483B000AF786039607B689B68CE
:1081080023F47C123B681A437B689A6000BF0C37E3
:10811800BD465DF8047B704780B483B000AF7860DB
:1081280039607B689B6823F0E0723B681A437B6880
:108138009A6000BF0C37BD465DF8047B704780B479
:1081480083B000AF78607B689B6803F0E0731846E3
:108158000C37BD465DF8047B7047000080B487B0DB
:1081680000AFF860B9607A603B60FB6860331A461C
:10817800BB689B0013447B617B691A68084B1340FA
:108188007A6802F0F8413A680A43134343F0004220
:108198007B691A6000BF1C37BD465DF8047B7047D9
:1081A80000F0FF0380B485B000AF786039607B6869
:1081B80060331A463B689B001344FB60FB681B68EE
:1081C80003F0F84318461437BD465DF8047B704742
:1081D80080B487B000AFF860B9607A60FB6860333C
:1081E8001A46BB689B0013447B617B691B6823F0BC
:1081F80000427B681A437B691A6000BF1C37BD4682
:108208005DF8047B704780B487B000AFF860B96050
:108218007A60FB6860331A46BB689B0013447B6135
:108228007B691B6823F080727B681A437B691A603C
:1082380000BF1C37BD465DF8047B704780B487B02B
:1082480000AFF860B9607A60FB6860331A46BB68B3
:108258009B0013447B617B691B6823F000727B6879
:108268001A437B691A6000BF1C37BD465DF8047B62
:10827800704780B483B000AF786039607B685B6911
:1082880023F000423B681A437B685A6100BF0C37F1
:10829800BD465DF8047B704780B483B000AF78605A
:1082A8007B68DB6803F44063002B01D1012300E005
:1082B800002318460C37BD465DF8047B704780B430
:1082C80087B000AFF860B9607A60FB6830331A464F
:1082D800BB681B0A9B0003F00C0313447B617B699A
:1082E8001A68BB6803F01F031F2101FA03F3DB437D
:1082F8001A407B689B0E03F01F01BB6803F01F0345
:1083080001FA03F31A437B691A6000BF1C37BD46A4
:108318005DF8047B704780B487B000AFF860B9603F
:108328007A60FB6814331A46BB685B0E9B0003F047
:10833800040313447B617B691A68BB681B0D03F057
:108348001F03072101FA03F3DB431A40BB681B0D27
:1083580003F01F03796801FA03F31A437B691A6073
:1083680000BF1C37BD465DF8047B704780B485B0FC
:1083780000AFF860B9607A60FB68D3F8B020BB68DA
:10838800C3F31203DB431A407B6803F01803084960
:10839800D940BB680B40C3F312031A43FB68C3F808
:1083A800B02000BF1437BD465DF8047B704700BF9E
:1083B800FFFF070080B483B000AF78607B689B68DC
:1083C80003F01F0318460C37BD465DF8047B704761
:1083D80080B483B000AF78607B689B6823F020434B
:1083E80023F03F037A68936000BF0C37BD465DF801
:1083F800047B704780B483B000AF78607B689B686B
:1084080003F00053B3F1005F01D1012300E0002322
:1084180018460C37BD465DF8047B704780B483B0BE
:1084280000AF78607B689B6823F0104323F03F031C
:1084380043F080527B689A6000BF0C37BD465DF8F8
:10844800047B704780B483B000AF78607B689B681A
:1084580003F08053B3F1805F01D1012300E00023D2
:1084680018460C37BD465DF8047B704780B483B06E
:1084780000AF78607B689B6823F0004323F03F03DC
:1084880043F001027B689A6000BF0C37BD465DF877
:10849800047B704780B483B000AF78607B689B68CA
:1084A80023F0004323F03F0343F002027B689A6005
:1084B80000BF0C37BD465DF8047B704780B483B0BD
:1084C80000AF78607B689B6803F00103012B01D142
:1084D800012300E0002318460C37BD465DF8047BF5
:1084E800704780B483B000AF78607B689B6803F006
:1084F8000203022B01D1012300E0002318460C37A8
:10850800BD465DF8047B704780B483B000AF7860E7
:108518007B689B6823F0004323F03F0343F0040289
:108528007B689A6000BF0C37BD465DF8047B7047D6
:1085380080B483B000AF78607B689B6803F0040365
:10854800042B01D1012300E0002318460C37BD4657
:108558005DF8047B704780B483B000AF78607B68B7
:108568009B6803F00803082B01D1012300E00023D6
:1085780018460C37BD465DF8047B704790B589B046
:1085880000AF78600023FB770023FB607B68002B3B
:1085980001D10123A9E17B685B69002B7B68DB6D56
:1085A800002B09D17868F8F715FD7B6800221A6658
:1085B8007B68002283F858207B681B681846FFF701
:1085C80019FF0346002B04D07B681B681846FFF789
:1085D800FFFE7B681B681846FFF734FF0346002B35
:1085E80015D17B681B681846FFF718FF9C4B1B6862
:1085F8009B099C4AA2FB03239B0901335B00FB6098
:1086080002E0FB68013BFB60FB68002BF9D17B684B
:108618001B681846FFF716FF0346002B0DD17B6831
:10862800DB6D43F010027B68DA657B681B6E43F0F4
:1086380001027B681A660123FB777B681B68184672
:10864800FFF776FF78617B68DB6D03F01003002B82
:1086580040F042817B69002B40F03E817B68DB6DF6
:1086680023F4817343F002027B68DA657B681B6838
:108678001846FFF723FF0346002B41D17B681B6890
:10868800B3F1A04F04D07B681B68774A93420FD19F
:108698004FF0A040FFF712FF04467348FFF70EFFA4
:1086A80003462343002B0CBF01230023DBB212E057
:1086B8006E48FFF703FF04466D48FFF7FFFE0346C9
:1086C8001C436C48FFF7FAFE03462343002B0CBFFC
:1086D80001230023DBB2002B12D07B681B68B3F1A7
:1086E800A04F04D07B681B685F4A934201D1624A5D
:1086F80000E0624A7B685B6819461046FFF7F9FCA0
:108708007B685B7F5A037B68DB6B1A437B68DB689B
:108718001A437B689B681A437B6893F824301B04D0
:108728001343BB617B6893F82430012B06D17B6827
:108738009B6A013B5B04BA691343BB617B68DB6AD4
:10874800002B09D07B68DB6A03F478727B681B6BAB
:108758001343BA691343BB617B681B68DA68484BEB
:1087680013407A681268B9690B43D3607B681B6849
:108778001B6923F040617B685A6B7B681B680A435E
:108788001A617B681B681846FFF7E5FE38617B694C
:10879800002B7FD13B69002B7CD17B681B7F9A0320
:1087A8007B6893F838305B001343BB617B681B68B8
:1087B800DB6823F4804323F002037A681268B969FE
:1087C8000B43D3607B681B69002B17D07B681B6841
:1087D8001A697B681B6842F480321A617B681B68DF
:1087E800D3F8C03023F47F5323F03F037A6811692C
:1087F8007A6812680B43C2F8C03013E07B681B68C4
:108808001A697B681B6822F480321A617B681B68CE
:10881800D3F8C0307A68126823F47F5323F03F03FB
:10882800C2F8C0307B6893F84030012B2AD17B68AE
:108838001B681B6923F4FF6323F004037A68516CF7
:108848007A68926C11437A68D26C11437A68126D17
:108858000A431A437B681B6842F001021A6119E057
:1088680070000020632D3E050001005000040050F8
:10887800000500500006005000030050000700509B
:108888000740F0FF7B681B681A697B681B6822F049
:1088980001021A617B685B69012B0CD17B681B683C
:1088A8001B6B23F00F017B681B6A5A1E7B681B68D1
:1088B8000A431A6307E07B681B681A6B7B681B68AE
:1088C80022F00F021A637B68DB6D23F0030343F089
:1088D80001027B68DA6507E07B68DB6D43F0100214
:1088E8007B68DA650123FB77FB7F18462437BD4692
:1088F80090BD00BF80B586B000AFF860B9607A60FF
:10890800FB681B68B3F1A04F04D0FB681B685A4A88
:10891800934201D1594B00E0594B1846FFF74AFDE5
:108928003861FB681B681846FFF702FE0346002BF8
:1089380040F09B80FB6893F85830012B01D102234B
:1089480096E0FB68012283F85820FB681B684D4AB3
:10895800934208D03B69002B05D03B69052B02D018
:108968003B69092B7AD1F86800F0ECFC0346FB75EB
:10897800FB7D002B6DD1FB68DB6D23F4706323F066
:10898800010343F48072FB68DA65FB681B683A4AA6
:10899800934209D0FB681B683B4A934202D0FB68AC
:1089A8001B6803E0394B01E04FF0A043FA681268F6
:1089B800934202D03B69002B05D1FB68DB6D23F4A1
:1089C8008012FB68DA65FB68DB6D03F48053002BCB
:1089D80006D0FB681B6E23F00602FB681A6602E0ED
:1089E800FB6800221A66FB685B6D294ADA62FB683D
:1089F8005B6D284A1A63FB685B6D274A5A63FB68FC
:108A08001B681C221A60FB68002283F85820FB6848
:108A18001B685A68FB681B6842F010025A60FB68C2
:108A28001B68DA68FB681B6842F00102DA60FB68C1
:108A3800586DFB681B6840331946BA687B68FEF7B7
:108A4800CBFF0346FB75FB681B681846FFF75CFD08
:108A58000DE0FB68002283F8582008E00123FB752D
:108A6800FB68002283F8582001E00223FB75FB7D98
:108A780018461837BD4680BD00010050000300505D
:108A88000007005000060050000500500004005088
:108A9800379501080F9601082B96010880B483B01A
:108AA80000AF786000BF0C37BD465DF8047B7047A7
:108AB80080B483B000AF786000BF0C37BD465DF866
:108AC800047B704780B5B6B000AF7860396000238A
:108AD80087F8D7300023FB607B6893F85830012B68
:108AE80002D1022300F013BC7B68012283F85820CE
:108AF8007B681B681846FFF71BFD0346002B40F0F8
:108B0800F3837B6818683B6859683B681B681A469A
:108B1800FFF7D5FB7B681B681846FFF709FDC7F808
:108B2800D0007B681B681846FFF715FDC7F8CC0016
:108B3800D7F8D030002B40F0D981D7F8CC30002BB3
:108B480040F0D4813B689B68B3F1004F0FD17B683C
:108B580018683B681B6800221946FFF7DCFB7B6836
:108B68001B684FF000411846FFF783FB0EE07B6857
:108B780018683B6819683B689B681A46FFF7CBFB87
:108B88007B681B6800211846FFF773FB3B685A692E
:108B98007B681B68DB68DB0803F003035B0002FAF1
:108BA80003F3C7F8C8303B681B69042B22D07B68E5
:108BB80018683B6819693B681A68D7F8C830FFF726
:108BC800CDFA7B6818683B6819693B689B691A4647
:108BD800FFF719FB7B6818683B6819693B681B7FBE
:108BE800012B02D14FF0007300E000231A46FFF773
:108BF80025FB7BE17B681B6800211846FFF7D2FA4A
:108C08000346C3F31203002B0AD17B681B680021BB
:108C18001846FFF7C7FA03469B0E03F01F021EE033
:108C28007B681B6800211846FFF7BCFA0346C7F8A3
:108C3800BC30D7F8BC3093FAA3F3C7F8B830D7F8EC
:108C4800B830C7F8C030D7F8C030002B01D1202386
:108C580004E0D7F8C030B3FA83F3DBB21A463B68B6
:108C68001B68C3F31203002B05D13B681B689B0EDE
:108C780003F01F0318E03B681B68C7F8B030D7F84B
:108C8800B03093FAA3F3C7F8AC30D7F8AC30C7F8D4
:108C9800B430D7F8B430002B01D1202304E0D7F842
:108CA800B430B3FA83F3DBB29A4206D17B681B680F
:108CB800002200211846FFF78BFA7B681B68012108
:108CC8001846FFF76FFA0346C3F31203002B0AD1C5
:108CD8007B681B6801211846FFF764FA03469B0E60
:108CE80003F01F021EE07B681B6801211846FFF78E
:108CF80059FA0346C7F8A430D7F8A43093FAA3F377
:108D0800C7F8A030D7F8A030C7F8A830D7F8A830EF
:108D1800002B01D1202304E0D7F8A830B3FA83F35D
:108D2800DBB21A463B681B68C3F31203002B05D15C
:108D38003B681B689B0E03F01F0318E03B681B6829
:108D4800C7F89830D7F8983093FAA3F3C7F8943057
:108D5800D7F89430C7F89C30D7F89C30002B01D155
:108D6800202304E0D7F89C30B3FA83F3DBB29A42AD
:108D780006D17B681B68002201211846FFF728FAF4
:108D88007B681B6802211846FFF70CFA0346C3F3F9
:108D98001203002B0AD17B681B6802211846FFF7D3
:108DA80001FA03469B0E03F01F021EE07B681B6856
:108DB80002211846FFF7F6F90346C7F88C30D7F8B2
:108DC8008C3093FAA3F3C7F88830D7F88830C7F8FF
:108DD8009030D7F89030002B01D1202304E0D7F849
:108DE8009030B3FA83F3DBB21A463B681B68C3F3CF
:108DF8001203002B05D13B681B689B0E03F01F0371
:108E080016E03B681B68C7F88030D7F8803093FAC3
:108E1800A3F3FB67FB6FC7F88430D7F88430002BC7
:108E280001D1202304E0D7F88430B3FA83F3DBB20E
:108E38009A4206D17B681B68002202211846FFF778
:108E4800C7F97B681B6803211846FFF7ABF903468F
:108E5800C3F31203002B0AD17B681B680321184651
:108E6800FFF7A0F903469B0E03F01F0217E07B688B
:108E78001B6803211846FFF795F903467B677B6F4C
:108E880093FAA3F33B673B6FBB67BB6F002B01D122
:108E9800202303E0BB6FB3FA83F3DBB21A463B68C7
:108EA8001B68C3F31203002B05D13B681B689B0E9C
:108EB80003F01F0311E03B681B68BB66BB6E93FAA7
:108EC800A3F37B667B6EFB66FB6E002B01D1202330
:108ED80003E0FB6EB3FA83F3DBB29A4206D17B68F8
:108EE8001B68002203211846FFF772F97B681B688C
:108EF8001846FFF7E3FA0346002B40F03D817B68F4
:108F080018683B6819683B68DB681A46FFF72EFA51
:108F18003B68DB68A24A934240F02E817B68186860
:108F28003B681B68C3F31203002B0BD13B681B681B
:108F38009B0E013303F01F03092B94BF0123002369
:108F4800DBB219E03B681B68FB65FB6D93FAA3F382
:108F5800BB65BB6D3B663B6E002B01D1202303E054
:108F68003B6EB3FA83F3DBB2013303F01F03092B23
:108F780094BF01230023DBB2002B79D03B681B6828
:108F8800C3F31203002B07D13B681B689B0E013308
:108F98009B0603F0F84215E03B681B683B653B6D98
:108FA80093FAA3F3FB64FB6C7B657B6D002B01D10B
:108FB800202303E07B6DB3FA83F3DBB201339B0616
:108FC80003F0F8423B681B68C3F31203002B09D176
:108FD8003B681B689B0E013303F01F03012101FA54
:108FE80003F317E03B681B687B647B6C93FAA3F37D
:108FF8003B643B6CBB64BB6C002B01D1202303E0BA
:10900800BB6CB3FA83F3DBB2013303F01F03012116
:1090180001FA03F342EA03013B681B68C3F3120336
:10902800002B0AD13B681B689B0E013303F01F021B
:1090380013465B0013441B0518E03B681B68BB63C1
:10904800BB6B93FAA3F37B637B6BFB63FB6B002B1C
:1090580001D1202303E0FB6BB3FA83F3DBB20133C6
:1090680003F01F0213465B0013441B050B437EE00D
:109078003B681B68C3F31203002B07D13B681B68CE
:109088009B0E01339B0603F0F84215E03B681B6812
:10909800FB62FB6A93FAA3F3BB62BB6A3B633B6B5D
:1090A800002B01D1202303E03B6BB3FA83F3DBB23F
:1090B80001339B0603F0F8423B681B68C3F31203B5
:1090C800002B09D13B681B689B0E013303F01F037B
:1090D800012101FA03F317E03B681B683B623B6A16
:1090E80093FAA3F3FB61FB697B627B6A002B01D1D6
:1090F800202303E07B6AB3FA83F3DBB2013303F086
:109108001F03012101FA03F342EA03013B681B68CC
:10911800C3F31203002B0DD13B681B689B0E013370
:1091280003F01F0213465B0013441E3B1B0543F06C
:1091380000731BE03B681B687B617B6993FAA3F3B0
:109148003B613B69BB61BB69002B01D1202303E074
:10915800BB69B3FA83F3DBB2013303F01F02134692
:109168005B0013441E3B1B0543F000730B433A6836
:1091780092681946FFF7CFF83B681A68094B134005
:10918800002B00F0BE807B681B68B3F1A04F04D0B1
:109198007B681B68044A93420AD1044B09E000BF6C
:1091A80000007F40000008800001005000030050CC
:1091B800594B1846FEF7C3FFC7F8C4003B681B6845
:1091C800564A934204D03B681B68554A93423AD1A9
:1091D800D7F8C43003F40003002B34D17B681B6834
:1091E800B3F1A04F05D07B681B684E4A934240F00C
:1091F80085807B681B68B3F1A04F04D07B681B682F
:10920800494A934201D1494A00E0434AD7F8C43059
:1092180043F4000319461046FEF77EFF444B1B68D3
:109228009B09444AA2FB03239B095A1C13465B0073
:1092380013449B00FB6002E0FB68013BFB60FB689A
:10924800002BF9D15AE03B681B683B4A934225D171
:10925800D7F8C43003F08073002B1FD17B681B68DC
:10926800314A934204D17B681B68344A934247D001
:109278007B681B68B3F1A04F04D07B681B682A4A3F
:10928800934201D1294A00E0234AD7F8C43043F079
:10929800807319461046FEF73FFF31E03B681B68B4
:1092A800274A93422DD1D7F8C43003F48003002B0A
:1092B80027D17B681B681C4A934222D07B681B68B5
:1092C800B3F1A04F04D07B681B68174A934201D1C1
:1092D800164A00E0104AD7F8C43043F48003194610
:1092E8001046FEF719FF0CE07B68DB6D43F02002A7
:1092F8007B68DA65012387F8D73002E000BF00E019
:1093080000BF7B68002283F8582097F8D7301846AA
:10931800D837BD4680BD00BF00070050000021C3FC
:109328001000C090000600500001005000030050DB
:1093380070000020632D3E05000052C70005005054
:10934800000084CB80B584B000AF78600023BB6098
:109358007B681B681846FFF7B1F80346002B76D1E7
:109368007B681B689A683C4B1340002B0DD07B68C8
:10937800DB6D43F010027B68DA657B681B6E43F097
:1093880001027B681A66012362E07B681B68184645
:10939800FFF76CF87B681B68B3F1A04F04D07B68BB
:1093A8001B682E4A934201D12D4B00E02D4B1846E5
:1093B800FEF7C5FE034603F40003002B13D02A4B27
:1093C8001B689B09294AA2FB03239B095A1C1346C5
:1093D8005B0013449B00BB6002E0BB68013BBB60C1
:1093E800BB68002BF9D1FDF731F9F86028E07B68FC
:1093F8001B681846FFF762F80346002B04D17B6808
:109408001B681846FFF732F8FDF720F90246FB689B
:10941800D31A022B14D97B681B681B6803F001035D
:10942800012B0DD07B68DB6D43F010027B68DA6599
:109438007B681B6E43F001027B681A66012307E014
:109448007B681B681B6803F00103012BCFD1002345
:1094580018461037BD4680BD3F000080000100500F
:10946800000300500007005070000020632D3E05E7
:1094780080B584B000AF78607B681B681846FFF73A
:1094880030F8F8607B681B681846FFF717F8034642
:10949800002B47D0FB68002B44D17B681B689B6876
:1094A80003F00D03012B0CD17B681B681846FEF7EF
:1094B800F1FF7B681B6803221A60FDF7C7F8B860E4
:1094C80029E07B68DB6D43F010027B68DA657B6816
:1094D8001B6E43F001027B681A66012323E0FDF747
:1094E800B5F80246BB68D31A022B14D97B681B68EF
:1094F8009B6803F00103002B0DD07B68DB6D43F004
:1095080010027B68DA657B681B6E43F001027B689A
:109518001A66012307E07B681B689B6803F0010358
:10952800002BDCD1002318461037BD4680BD80B51E
:1095380084B000AF78607B689B6AFB60FB68DB6D7A
:1095480003F05003002B4BD1FB68DB6D43F4007232
:10955800FB68DA65FB681B681B6803F00803002BCF
:1095680021D0FB681B681846FEF796FE0346002BC1
:1095780032D0FB681B68DB6803F40053002B2BD147
:10958800FB68DB6D23F48072FB68DA65FB68DB6DD2
:1095980003F48053002B1FD1FB68DB6D43F00102FD
:1095A800FB68DA6518E0FB681B68DB6803F00203F8
:1095B800002B11D1FB68DB6D23F48072FB68DA6540
:1095C800FB68DB6D03F48053002B05D1FB68DB6D72
:1095D80043F00102FB68DA65F868F7F7C7F90EE0AF
:1095E800FB68DB6D03F01003002B03D0F868FFF76E
:1095F8005FFA04E0FB685B6D5B6B7868984700BFB7
:109608001037BD4680BD80B584B000AF78607B68F8
:109618009B6AFB60F868FFF741FA00BF1037BD4648
:1096280080BD80B584B000AF78607B689B6AFB60C2
:10963800FB68DB6D43F04002FB68DA65FB681B6E74
:1096480043F00402FB681A66F868FFF731FA00BFB6
:109658001037BD4680BD80B483B000AF78607B68AA
:109668009B6803F00103012B01D1012300E00023D3
:1096780018460C37BD465DF8047B704780B483B04C
:1096880000AF786039607B689B6823F0404323F023
:109698003F033A6802F08042134343F000427B687C
:1096A8009A6000BF0C37BD465DF8047B704780B4F4
:1096B80083B000AF78607B689B6803F00043B3F128
:1096C800004F01D1012300E0002318460C37BD46A6
:1096D8005DF8047B704780B483B000AF78607B6826
:1096E8009B6803F00403042B01D1012300E000234D
:1096F80018460C37BD465DF8047B704780B584B0CA
:1097080000AF786039600023BB607B6893F85830FD
:10971800012B01D102234DE07B68012283F85820F8
:109728007868FFF7A5FE0346FB73FB7B002B36D159
:109738007B68DB6D23F4885323F0020343F00202B5
:109748007B68DA657B681B6839681846FFF796FFFF
:1097580014E0BB680133BB60BB68184A93420DD95B
:109768007B68DB6D23F0120343F010027B68DA6537
:109778007B68002283F8582001231BE07B681B6864
:109788001846FFF794FF0346002BE2D17B68DB6D98
:1097980023F0030343F001027B68DA6505E07B6888
:1097A800DB6D43F010027B68DA657B68002283F882
:1097B8005820FB7B18461037BD4680BD01DE0400EB
:1097C80090B5A1B000AF78603960002387F87F308A
:1097D8007B6893F85830012B01D10223E7E07B68BE
:1097E800012283F8582000237B660023BB667B6830
:1097F8001B68B3F1A04F02D16F4BBB6009E07B68D7
:109808001B686E4A934202D16D4BBB6001E0002396
:10981800BB60BB68002B0BD17B68DB6D43F020027B
:109828007B68DA657B68002283F858200123BEE054
:10983800BB681846FFF74FFFB8677B681B68184678
:10984800FFF749FF0346002B40F0A080BB6F002BB9
:1098580040F09C807B681B68B3F1A04F04D07B6804
:109868001B68554A934201D1564B00E0564B7B6723
:109878003B681B68002B4BD07B6F9B6823F46042CE
:109888003B6859687B6893F838305B030B431A438D
:109898007B6F9A607B681B68B3F1A04F04D07B682C
:1098A8001B68454A93420FD14FF0A040FFF7D3FE03
:1098B80004464148FFF7CFFE03462343002B0CBF65
:1098C80001230023DBB212E03C48FFF7C4FE044644
:1098D8003B48FFF7C0FE03461C433C48FFF7BBFE6E
:1098E80003462343002B0CBF01230023DBB2002BCC
:1098F80056D07B6F9B6823F4716323F00F033A689B
:1099080011683A6892680A431A437B6F9A6047E085
:109918007B6F9B6823F460427B6F9A607B681B684F
:10992800B3F1A04F04D07B681B68234A93420FD140
:109938004FF0A040FFF78FFE04461F48FFF78BFE4D
:1099480003462343002B0CBF01230023DBB212E0A4
:109958001A48FFF780FE04461948FFF77CFE0346C5
:109968001C431A48FFF777FE03462343002B0CBF1E
:1099780001230023DBB2002B12D07B6F9B6823F4FA
:10998800716323F00F037A6F936009E07B68DB6DE6
:1099980043F020027B68DA65012387F87F3000E016
:1099A80000BF7B68002283F8582097F87F3018465C
:1099B8008437BD4690BD00BF000100500004005030
:1099C800000500500003005000070050000600503A
:1099D80080B582B000AF78607B68002B01D101238D
:1099E8008DE07B6893F84130DBB2002B06D17B68B1
:1099F800002283F840207868F7F762FC7B6824220D
:109A080083F841207B681B681A687B681B6822F012
:109A180001021A607B685A687B681B6822F07062D2
:109A28001A617B681B689A687B681B6822F400428D
:109A38009A607B68DB68012B07D17B689A687B6832
:109A48001B6842F400429A6006E07B689A687B686B
:109A58001B6842F404429A607B68DB68022B08D1D9
:109A68007B681B685A687B681B6842F400625A600E
:109A780007E07B681B685A687B681B6822F40062F1
:109A88005A607B681B685B687A68126843F00073E9
:109A980043F4004353607B681B68DA687B681B6883
:109AA80022F40042DA607B681A697B685B6942EAE3
:109AB80003017B689B691A027B681B680A43DA60AA
:109AC8007B68D9697B681A6A7B681B680A431A60D5
:109AD8007B681B681A687B681B6842F001021A6081
:109AE8007B6800225A647B68202283F841207B68C7
:109AF80000221A637B68002283F84220002318465C
:109B08000837BD4680BD80B483B000AF7860396047
:109B18007B6893F84130DBB2202B38D17B6893F80F
:109B28004030012B01D1022332E07B68012283F807
:109B380040207B68242283F841207B681B681A68D0
:109B48007B681B6822F001021A607B681B681A6830
:109B58007B681B6822F480521A607B681B6819684E
:109B68007B681B683A680A431A607B681B681A6836
:109B78007B681B6842F001021A607B68202283F828
:109B880041207B68002283F84020002300E0022364
:109B980018460C37BD465DF8047B704780B485B025
:109BA80000AF786039607B6893F84130DBB2202BD6
:109BB80039D17B6893F84030012B01D1022333E07F
:109BC8007B68012283F840207B68242283F84120A7
:109BD8007B681B681A687B681B6822F001021A60A0
:109BE8007B681B681B68FB60FB6823F47063FB6081
:109BF8003B681B02FA681343FB607B681B68FA68C2
:109C08001A607B681B681A687B681B6842F001024F
:109C18001A607B68202283F841207B68002283F841
:109C28004020002300E0022318461437BD465DF8A3
:109C3800047B704780B582B000AF78607B68002BEA
:109C480001D1012349E07B6893F83D30DBB2002B5A
:109C580006D17B68002283F83C207868F7F72CFD52
:109C68007B68022283F83D207B681A687B6804338E
:109C78001946104600F03AFC7B68012283F8482018
:109C88007B68012283F83E207B68012283F83F200D
:109C98007B68012283F840207B68012283F84120F9
:109CA8007B68012283F842207B68012283F84320E5
:109CB8007B68012283F844207B68012283F84520D1
:109CC8007B68012283F846207B68012283F84720BD
:109CD8007B68012283F83D20002318460837BD46DB
:109CE80080BD000080B485B000AF78607B6893F8D1
:109CF8003D30DBB2012B01D001234CE07B6802220E
:109D080083F83D207B681B68264A934222D07B68F3
:109D18001B68B3F1804F1DD07B681B68224A9342B1
:109D280018D07B681B68214A934213D07B681B6854
:109D38001F4A93420ED07B681B681E4A934209D083
:109D48007B681B681C4A934204D07B681B681B4ACB
:109D5800934215D17B681B689A68194B1340FB60C6
:109D6800FB68062B15D0FB68B3F5803F11D07B68E4
:109D78001B681A687B681B6842F001021A6008E0D9
:109D88007B681B681A687B681B6842F001021A60CE
:109D980000E000BF002318461437BD465DF8047B79
:109DA800704700BF002C014000040040000800403C
:109DB800000C0040003401400040014000500140C8
:109DC8000700010080B582B000AF78607B68002B87
:109DD80001D1012349E07B6893F83D30DBB2002BC9
:109DE80006D17B68002283F83C20786800F041F8AF
:109DF8007B68022283F83D207B681A687B680433FD
:109E08001946104600F072FB7B68012283F848204F
:109E18007B68012283F83E207B68012283F83F207B
:109E28007B68012283F840207B68012283F8412067
:109E38007B68012283F842207B68012283F8432053
:109E48007B68012283F844207B68012283F845203F
:109E58007B68012283F846207B68012283F847202B
:109E68007B68012283F83D20002318460837BD4649
:109E780080BD80B483B000AF786000BF0C37BD46AA
:109E88005DF8047B7047000080B584B000AF78604F
:109E980039603B68002B09D17B6893F83E30DBB210
:109EA800012B14BF01230023DBB23CE03B68042BE9
:109EB80009D17B6893F83F30DBB2012B14BF012333
:109EC8000023DBB22FE03B68082B09D17B6893F8AD
:109ED8004030DBB2012B14BF01230023DBB222E0A8
:109EE8003B680C2B09D17B6893F84130DBB2012B1E
:109EF80014BF01230023DBB215E03B68102B09D106
:109F08007B6893F84230DBB2012B14BF0123002396
:109F1800DBB208E07B6893F84330DBB2012B14BF57
:109F280001230023DBB2002B01D00123A6E03B680C
:109F3800002B04D17B68022283F83E2023E03B6893
:109F4800042B04D17B68022283F83F201BE03B6886
:109F5800082B04D17B68022283F8402013E03B6879
:109F68000C2B04D17B68022283F841200BE03B686C
:109F7800102B04D17B68022283F8422003E07B681F
:109F8800022283F843207B681B680122396818463F
:109F980000F026FF7B681B683A4A934218D07B681A
:109FA8001B68394A934213D07B681B68374A93422F
:109FB8000ED07B681B68364A934209D07B681B68C1
:109FC800344A934204D07B681B68334A934201D1D8
:109FD800012300E00023002B07D07B681B685A6C24
:109FE8007B681B6842F400425A647B681B68254AF8
:109FF800934222D07B681B68B3F1804F1DD07B68E9
:10A008001B68264A934218D07B681B68244A9342EF
:10A0180013D07B681B68234A93420ED07B681B6869
:10A02800194A934209D07B681B68184A934204D0A6
:10A038007B681B68184A934215D17B681B689A682D
:10A04800194B1340FB60FB68062B15D0FB68B3F572
:10A05800803F11D07B681B681A687B681B6842F0D8
:10A0680001021A6008E07B681B681A687B681B6835
:10A0780042F001021A6000E000BF002318461037C2
:10A08800BD4680BD002C0140003401400040014025
:10A0980000440140004801400050014000040040D5
:10A0A80000080040000C00400700010080B586B0A1
:10A0B80000AFF860B9607A600023FB75FB6893F81D
:10A0C8003C30012B01D10223FFE0FB68012283F819
:10A0D8003C207B68142B00F2F08001A252F823F098
:10A0E8003DA10108C3A20108C3A20108C3A2010837
:10A0F8007DA10108C3A20108C3A20108C3A20108E7
:10A10800BFA10108C3A20108C3A20108C3A2010894
:10A11800FFA10108C3A20108C3A20108C3A2010844
:10A1280041A20108C3A20108C3A20108C3A20108F1
:10A1380081A20108FB681B68B968184600F08AFA12
:10A14800FB681B689A69FB681B6842F008029A6101
:10A15800FB681B689A69FB681B6822F004029A6115
:10A16800FB681B689969BB681A69FB681B680A4326
:10A178009A61A5E0FB681B68B968184600F004FB03
:10A18800FB681B689A69FB681B6842F400629A6165
:10A19800FB681B689A69FB681B6822F480629A61F5
:10A1A800FB681B689969BB681B691A02FB681B6816
:10A1B8000A439A6184E0FB681B68B968184600F096
:10A1C80077FBFB681B68DA69FB681B6842F00802CA
:10A1D800DA61FB681B68DA69FB681B6822F0040215
:10A1E800DA61FB681B68D969BB681A69FB681B6878
:10A1F8000A43DA6164E0FB681B68B968184600F036
:10A20800E9FBFB681B68DA69FB681B6842F40062BB
:10A21800DA61FB681B68DA69FB681B6822F48062F4
:10A22800DA61FB681B68D969BB681B691A02FB689D
:10A238001B680A43DA6143E0FB681B68B968184683
:10A2480000F05CFCFB681B681A6DFB681B6842F039
:10A2580008021A65FB681B681A6DFB681B6822F008
:10A2680004021A65FB681B68196DBB681A69FB68EC
:10A278001B680A431A6523E0FB681B68B96818461F
:10A2880000F0A6FCFB681B681A6DFB681B6842F4AB
:10A2980000621A65FB681B681A6DFB681B6822F46C
:10A2A80080621A65FB681B68196DBB681B691A0216
:10A2B800FB681B680A431A6502E00123FB7500BFAF
:10A2C800FB68002283F83C20FB7D18461837BD4602
:10A2D80080BD00BF80B584B000AF786039600023CE
:10A2E800FB737B6893F83C30012B01D10223EEE02D
:10A2F8007B68012283F83C207B68022283F83D209A
:10A308007B681B689B68BB60BB6823F4441323F01D
:10A318007703BB60BB6823F47F43BB607B681B6823
:10A32800BA689A603B681B686B4A934200F0B98030
:10A33800694A934200F2BE80684A934200F0B180B5
:10A34800664A934200F2B680654A934200F0A980BB
:10A35800634A934200F2AE80624A934200F0A180C1
:10A36800604A934200F2A6805F4A934200F09980C7
:10A378005D4A934200F29E80B3F1101F00F0918075
:10A38800B3F1101F00F29680B3F5801F00F08980AA
:10A39800B3F5801F00F28E80B3F5005F3ED0B3F5B1
:10A3A800005F00F28780B3F5805F00F08680B3F528
:10A3B800805F7FD8702B1AD0702B7BD8602B50D041
:10A3C800602B77D8502B3CD0502B73D8402B58D0CB
:10A3D800402B6FD8302B64D0302B6BD8202B60D01B
:10A3E800202B67D8002B5CD0102B5AD062E07B68FA
:10A3F80018683B6899683B685A683B68DB6800F0F6
:10A40800CFFC7B681B689B68BB60BB6843F0770325
:10A41800BB607B681B68BA689A604FE07B68186805
:10A428003B6899683B685A683B68DB6800F0B8FC91
:10A438007B681B689A687B681B6842F480429A6054
:10A448003CE07B6818683B6859683B68DB681A46DB
:10A4580000F02AFC7B681B685021184600F083FC3A
:10A468002CE07B6818683B6859683B68DB681A46CB
:10A4780000F049FC7B681B686021184600F073FCFB
:10A488001CE07B6818683B6859683B68DB681A46BB
:10A4980000F00AFC7B681B684021184600F063FC4A
:10A4A8000CE07B681A683B681B681946104600F088
:10A4B8005AFC03E00123FB7300E000BF7B68012224
:10A4C80083F83D207B68002283F83C20FB7B1846FC
:10A4D8001037BD4680BD00BF70001000500010004E
:10A4E80040001000300010002000100080B485B03B
:10A4F80000AF786039607B681B68FB607B684C4AFA
:10A50800934217D07B68B3F1804F13D07B68494AD8
:10A5180093420FD07B68484A93420BD07B68474AE6
:10A52800934207D07B68464A934203D07B68454AEA
:10A53800934208D1FB6823F07003FB603B685B68BB
:10A54800FA681343FB607B68394A934223D07B68DF
:10A55800B3F1804F1FD07B68364A93421BD07B688B
:10A56800354A934217D07B68344A934213D07B68AC
:10A57800334A93420FD07B68334A93420BD07B68AF
:10A58800324A934207D07B68314A934203D07B68B2
:10A598002C4A934208D1FB6823F44073FB603B6864
:10A5A800DB68FA681343FB60FB6823F080023B68B2
:10A5B8005B691343FB607B68FA681A603B689A68BA
:10A5C8007B68DA623B681A687B689A627B68184A1B
:10A5D800934213D07B681A4A93420FD07B681A4A79
:10A5E80093420BD07B68194A934207D07B68184A7C
:10A5F800934203D07B68134A934203D13B681A699C
:10A608007B681A637B6801225A617B681B6903F0C7
:10A618000103012B05D17B681B6923F001027B68CC
:10A628001A6100BF1437BD465DF8047B704700BF50
:10A63800002C01400004004000080040000C0040CD
:10A6480000340140005001400040014000440140F6
:10A658000048014080B487B000AF786039607B68FB
:10A668001B6A7B617B681B6A23F001027B681A62A4
:10A678007B685B683B617B689B69FB60FB6823F4D4
:10A68800803323F07003FB60FB6823F00303FB6057
:10A698003B681B68FA681343FB607B6923F002037D
:10A6A8007B613B689B687A6913437B617B68304AAE
:10A6B800934213D07B682F4A93420FD07B682E4A6F
:10A6C80093420BD07B682D4A934207D07B682C4A73
:10A6D800934203D07B682B4A93420CD17B6923F0C9
:10A6E80008037B613B68DB687A6913437B617B699C
:10A6F80023F004037B617B681D4A934213D07B6877
:10A708001C4A93420FD07B681B4A93420BD07B684C
:10A718001A4A934207D07B68194A934203D07B6850
:10A72800184A934211D13B6923F480733B613B691A
:10A7380023F400733B613B685B693A6913433B61EF
:10A748003B689B693A6913433B617B683A695A6085
:10A758007B68FA689A613B685A687B685A637B68C9
:10A768007A691A6200BF1C37BD465DF8047B7047E2
:10A77800002C0140003401400040014000440140E9
:10A78800004801400050014080B487B000AF7860B5
:10A7980039607B681B6A7B617B681B6A23F0100247
:10A7A8007B681A627B685B683B617B689B69FB60BE
:10A7B800FB6823F0807323F4E043FB60FB6823F419
:10A7C8004073FB603B681B681B02FA681343FB601D
:10A7D8007B6923F020037B613B689B681B017A69D6
:10A7E80013437B617B682C4A934207D07B682B4AD2
:10A7F800934203D07B682A4A93420DD17B6923F0A8
:10A8080080037B613B68DB681B017A6913437B61CA
:10A818007B6923F040037B617B681F4A934213D016
:10A828007B681E4A93420FD07B681E4A93420BD026
:10A838007B681D4A934207D07B681C4A934203D029
:10A848007B68174A934213D13B6923F480633B61C9
:10A858003B6923F400633B613B685B699B003A6991
:10A8680013433B613B689B699B003A6913433B6117
:10A878007B683A695A607B68FA689A613B685A68EB
:10A888007B689A637B687A691A6200BF1C37BD4689
:10A898005DF8047B704700BF002C01400034014084
:10A8A8000050014000400140004401400048014080
:10A8B80080B487B000AF786039607B681B6A7B61C1
:10A8C8007B681B6A23F480727B681A627B685B680A
:10A8D8003B617B68DB69FB60FB6823F4803323F012
:10A8E8007003FB60FB6823F00303FB603B681B6895
:10A8F800FA681343FB607B6923F400737B613B6850
:10A908009B681B027A6913437B617B682B4A9342DD
:10A9180007D07B682A4A934203D07B68294A93422E
:10A928000DD17B6923F400637B613B68DB681B0204
:10A938007A6913437B617B6923F480637B617B685D
:10A948001E4A934213D07B681D4A93420FD07B68FE
:10A958001D4A93420BD07B681C4A934207D07B6800
:10A968001B4A934203D07B68164A934213D13B6932
:10A9780023F480533B613B6923F400533B613B68FC
:10A988005B691B013A6913433B613B689B691B0187
:10A998003A6913433B617B683A695A607B68FA6895
:10A9A800DA613B685A687B68DA637B687A691A629D
:10A9B80000BF1C37BD465DF8047B7047002C014082
:10A9C8000034014000500140004001400044014073
:10A9D8000048014080B487B000AF786039607B6878
:10A9E8001B6A7B617B681B6A23F480527B681A624E
:10A9F8007B685B683B617B68DB69FB60FB6823F015
:10AA0800807323F4E043FB60FB6823F44073FB602E
:10AA18003B681B681B02FA681343FB607B6923F4DD
:10AA280000537B613B689B681B037A6913437B6116
:10AA38007B682C4A934207D07B682B4A934203D009
:10AA48007B682A4A93420DD17B6923F400437B61DA
:10AA58003B68DB681B037A6913437B617B6923F4DA
:10AA680080437B617B681F4A934213D07B681E4AF0
:10AA780093420FD07B681E4A93420BD07B681D4AD5
:10AA8800934207D07B681C4A934203D07B68174ADD
:10AA9800934213D13B6923F480433B613B6923F420
:10AAA80000433B613B685B699B013A6913433B6127
:10AAB8003B689B699B013A6913433B617B683A6930
:10AAC8005A607B68FA68DA613B685A687B681A647E
:10AAD8007B687A691A6200BF1C37BD465DF8047B43
:10AAE800704700BF002C0140003401400050014075
:10AAF80000400140004401400048014080B487B054
:10AB080000AF786039607B681B6A3B617B681B6AB1
:10AB180023F480327B681A627B685B687B617B68A0
:10AB28001B6DFB60FB6823F4803323F07003FB602C
:10AB38003B681B68FA681343FB603B6923F40033E6
:10AB48003B613B689B681B043A6913433B617B6824
:10AB5800194A934213D07B68184A93420FD07B68F6
:10AB6800174A93420BD07B68164A934207D07B68FA
:10AB7800154A934203D07B68144A934209D17B69F2
:10AB880023F480337B613B685B691B027A6913435A
:10AB98007B617B687A695A607B68FA681A653B68EA
:10ABA8005A687B689A647B683A691A6200BF1C37E6
:10ABB800BD465DF8047B7047002C0140003401401D
:10ABC800004001400044014000480140005001405D
:10ABD80080B487B000AF786039607B681B6A3B61DE
:10ABE8007B681B6A23F480127B681A627B685B6847
:10ABF8007B617B681B6DFB60FB6823F0807323F42B
:10AC0800E043FB603B681B681B02FA681343FB6068
:10AC18003B6923F400133B613B689B681B053A6959
:10AC280013433B617B681A4A934213D07B68194AE5
:10AC380093420FD07B68184A93420BD07B68174A1F
:10AC4800934207D07B68164A934203D07B68154A23
:10AC5800934209D17B6923F480237B613B685B695C
:10AC68009B027A6913437B617B687A695A607B68C7
:10AC7800FA681A653B685A687B68DA647B683A69DF
:10AC88001A6200BF1C37BD465DF8047B704700BFE1
:10AC9800002C0140003401400040014000440140C4
:10ACA800004801400050014080B487B000AFF86010
:10ACB800B9607A60FB681B6A7B61FB681B6A23F0DA
:10ACC8000102FB681A62FB689B693B613B6923F0E0
:10ACD800F0033B617B681B013A6913433B617B6965
:10ACE80023F00A037B617A69BB6813437B61FB68C5
:10ACF8003A699A61FB687A691A6200BF1C37BD46D7
:10AD08005DF8047B704780B487B000AFF860B96025
:10AD18007A60FB681B6A7B61FB681B6A23F0100280
:10AD2800FB681A62FB689B693B613B6923F47043CB
:10AD38003B617B681B033A6913433B617B6923F0E2
:10AD4800A0037B61BB681B017A6913437B61FB68C5
:10AD58003A699A61FB687A691A6200BF1C37BD4676
:10AD68005DF8047B704780B485B000AF78603960C7
:10AD78007B689B68FB60FB6823F4401323F0700337
:10AD8800FB603A68FB68134343F00703FB607B688A
:10AD9800FA689A6000BF1437BD465DF8047B7047B7
:10ADA80080B487B000AFF860B9607A603B60FB6838
:10ADB8009B687B617B6923F47F437B613B681A0254
:10ADC8007B681A43BB6813437A6913437B61FB684A
:10ADD8007A699A6000BF1C37BD465DF8047B7047EE
:10ADE80080B487B000AFF860B9607A60BB6803F0E0
:10ADF8001F03012202FA03F37B61FB681A6A7B696D
:10AE0800DB431A40FB681A62FB681A6ABB6803F0E6
:10AE18001F03796801FA03F31A43FB681A6200BF3B
:10AE28001C37BD465DF8047B7047000080B485B0D0
:10AE380000AF786039607B6893F83C30012B01D112
:10AE4800022374E07B68012283F83C207B6802229D
:10AE580083F83D207B681B685B68FB607B681B6828
:10AE68009B68BB607B681B68344A934209D07B6847
:10AE78001B68334A934204D07B681B68314A93426B
:10AE880008D1FB6823F47003FB603B685B68FA68D1
:10AE98001343FB60FB6823F0007323F07003FB602F
:10AEA8003B681B68FA681343FB607B681B68FA6899
:10AEB8005A607B681B68214A934222D07B681B68D2
:10AEC800B3F1804F1DD07B681B681F4A934218D08E
:10AED8007B681B681D4A934213D07B681B681C4A19
:10AEE80093420ED07B681B68154A934209D07B6851
:10AEF8001B68184A934204D07B681B68114A934226
:10AF08000CD1BB6823F08003BB603B689B68BA68C0
:10AF18001343BB607B681B68BA689A607B68012230
:10AF280083F83D207B68002283F83C2000231846E4
:10AF38001437BD465DF8047B704700BF002C014004
:10AF48000034014000500140000400400008004067
:10AF5800000C00400040014080B485B000AF78602C
:10AF680039600023FB607B6893F83C30012B01D1EA
:10AF7800022378E07B68012283F83C20FB6823F0F9
:10AF8800FF023B68DB681343FB60FB6823F44072F5
:10AF98003B689B681343FB60FB6823F480623B6853
:10AFA8005B681343FB60FB6823F400623B681B6823
:10AFB8001343FB60FB6823F480523B681B6913430F
:10AFC800FB60FB6823F400523B685B691343FB603A
:10AFD800FB6823F480423B681B6B1343FB60FB68F0
:10AFE80023F470223B689B691B041343FB60FB68D6
:10AFF80023F080523B68DB691343FB607B681B6866
:10B008001C4A934209D07B681B681B4A934204D0B0
:10B018007B681B68194A93421CD1FB6823F47002B1
:10B028003B689B6A1B051343FB60FB6823F0807237
:10B038003B681B6A1343FB60FB6823F000723B68A4
:10B048005B6A1343FB60FB6823F000523B68DB6AD2
:10B058001343FB607B681B68FA685A647B680022AC
:10B0680083F83C20002318461437BD465DF8047B5E
:10B07800704700BF002C01400034014000500140DF
:10B0880080B582B000AF78607B68002B01D10123C6
:10B0980042E07B68D3F88830002B06D17B68002219
:10B0A80083F884207868F6F713FC7B682422C3F8B9
:10B0B80088207B681B681A687B681B6822F001027D
:10B0C8001A607B689B6A002B02D0786800F024FB2A
:10B0D800786800F025F80346012B01D101231BE015
:10B0E8007B681B685A687B681B6822F490425A6028
:10B0F8007B681B689A687B681B6822F02A029A6042
:10B108007B681B681A687B681B6842F001021A603A
:10B11800786800F0A3FB034618460837BD4680BD93
:10B128002DE9B04F8CB000AF7861002387F82A3042
:10B138007B699A687B691B691A437B695B691A4357
:10B148007B69DB691343FB627B691B681A68AA4B3E
:10B1580013407A691268F96A0B4313607B691B68AC
:10B168005B6823F440517B69DA687B691B680A4392
:10B178005A607B699B69FB627B691B689F4A9342A3
:10B1880004D07B691B6AFA6A1343FB627B691B68FC
:10B198009B6823F06E4323F430637A691268F96A76
:10B1A8000B4393607B691B68DB6A23F00F017B69A3
:10B1B8005A6A7B691B680A43DA627B691B68904A92
:10B1C800934225D18F4BD3F8883003F00303032B28
:10B1D8001AD801A252F823F0F1B1010801B201080E
:10B1E800F9B1010809B20108012387F82B3016E1EB
:10B1F800022387F82B3012E1042387F82B300EE165
:10B20800082387F82B300AE1102387F82B3006E152
:10B218007B691B687C4A934238D17A4BD3F88830D3
:10B2280003F00C030C2B2DD801A252F823F000BF19
:10B238006DB201088DB201088DB201088DB2010806
:10B248007DB201088DB201088DB201088DB20108E6
:10B2580075B201088DB201088DB201088DB20108DE
:10B2680085B20108002387F82B30D8E0022387F83D
:10B278002B30D4E0042387F82B30D0E0082387F85C
:10B288002B30CCE0102387F82B30C8E07B691B6893
:10B298005E4A934225D15B4BD3F8883003F03003E4
:10B2A800302B16D0302B18D8202B0AD0202B14D8AE
:10B2B800002B02D0102B08D00FE0002387F82B308A
:10B2C800ADE0022387F82B30A9E0042387F82B3060
:10B2D800A5E0082387F82B30A1E0102387F82B304E
:10B2E8009DE07B691B684A4A934225D1454BD3F8B8
:10B2F800883003F0C003C02B16D0C02B18D8802B81
:10B308000AD0802B14D8002B02D0402B08D00FE095
:10B31800002387F82B3082E0022387F82B307EE069
:10B32800042387F82B307AE0082387F82B3076E05F
:10B33800102387F82B3072E07B691B68354A9342EB
:10B348002AD1304BD3F8883003F44073B3F5407FEB
:10B358001AD0B3F5407F1BD8B3F5007F0CD0B3F5F6
:10B36800007F15D8002B03D0B3F5807F08D00FE0FD
:10B37800002387F82B3052E0022387F82B304EE069
:10B38800042387F82B304AE0082387F82B3046E05F
:10B39800102387F82B3042E07B691B68174A9342D9
:10B3A8003AD1184BD3F8883003F44063B3F5406FB3
:10B3B8001AD0B3F5406F1BD8B3F5006F0CD0B3F5B6
:10B3C800006F15D8002B03D0B3F5806F08D00FE0BD
:10B3D800002387F82B3022E0022387F82B301EE069
:10B3E800042387F82B301AE0082387F82B3016E05F
:10B3F800102387F82B3012E0F369FFCF008000405C
:10B40800003801400010024000440040004800405D
:10B41800004C004000500040102387F82B307B6917
:10B428001B68AE4A934240F0978097F82B30082B60
:10B4380023D801A252F823F065B4010883B40108A7
:10B448006DB4010883B4010873B4010883B401081A
:10B4580083B4010883B401087BB40108FBF7BCFD81
:10B46800786210E09E4B7B620DE0FBF749FD786245
:10B4780009E04FF400437B6205E000237B6201236F
:10B4880087F82A3000BF7B6A002B00F030817B6987
:10B498005B6A944A32F813301A467B6AB3FBF2F3BC
:10B4A800BB617B695A6813465B001344BA699A42C8
:10B4B80005D37B695B681B03BA699A4203D90123E8
:10B4C80087F82A3013E17B6A0022BB60FA607B6947
:10B4D8005B6A844A32F813309BB200223B607A6080
:10B4E800D7E90023D7E90201F4F792FE02460B469A
:10B4F800104619464FF000024FF000030B0243EAD2
:10B508001063020279694968490800200C4605461B
:10B5180012EB040843EB05097B695B6800229A4635
:10B52800934652465B4640464946F4F771FE02464A
:10B538000B4613463B623B6AB3F5407F08D33B6A30
:10B54800B3F5801F04D27B691B683A6ADA60CEE0E3
:10B55800012387F82A30CAE07B69DB69B3F5004F1D
:10B5680066D197F82B30082B27D801A252F823F080
:10B578009DB50108A5B50108ADB50108C3B5010819
:10B58800B3B50108C3B50108C3B50108C3B50108BF
:10B59800BBB50108FBF720FD786214E0FBF732FD2C
:10B5A800786210E04E4B7B620DE0FBF7A9FC7862F5
:10B5B80009E04FF400437B6205E000237B6201232E
:10B5C80087F82A3000BF7B6A002B00F090807B69E7
:10B5D8005B6A444A32F813301A467B6AB3FBF2F3CB
:10B5E8005A007B695B685B081A447B695B68B2FB3D
:10B5F800F3F33B623B6A0F2B16D93B6AB3F5803FE6
:10B6080012D23B6A9BB223F00F03FB833B6A5B08B1
:10B618009BB203F007039AB2FB8B1343FB837B694E
:10B628001B68FA8BDA6062E0012387F82A305EE053
:10B6380097F82B30082B28D801A252F823F000BF26
:10B648006DB6010875B601087DB6010893B6010804
:10B6580083B6010893B6010893B6010893B60108AA
:10B668008BB60108FBF7B8FC786214E0FBF7CAFC5C
:10B67800786210E01A4B7B620DE0FBF741FC7862C0
:10B6880009E04FF400437B6205E000237B6201235D
:10B6980087F82A3000BF7B6A002B28D07B695B6A59
:10B6A800104A32F813301A467B6AB3FBF2F27B6910
:10B6B8005B685B081A447B695B68B2FBF3F33B6227
:10B6C8003B6A0F2B10D93B6AB3F5803F0CD23B6A1B
:10B6D8009AB27B691B68DA6009E000BF008000400D
:10B6E8000024F40068D60108012387F82A307B6912
:10B6F8000122A3F86A207B690122A3F868207B69EC
:10B7080000225A677B6900229A6797F82A30184600
:10B718003037BD46BDE8B08F80B483B000AF7860E5
:10B728007B689B6A03F00803002B0AD07B681B68C0
:10B738005B6823F400417B689A6B7B681B680A434B
:10B748005A607B689B6A03F00103002B0AD07B6870
:10B758001B685B6823F400317B68DA6A7B681B68C6
:10B768000A435A607B689B6A03F00203002B0AD0E5
:10B778007B681B685B6823F480317B681A6B7B6885
:10B788001B680A435A607B689B6A03F00403002B1A
:10B798000AD07B681B685B6823F480217B685A6B3E
:10B7A8007B681B680A435A607B689B6A03F0100336
:10B7B800002B0AD07B681B689B6823F480517B6848
:10B7C800DA6B7B681B680A439A607B689B6A03F0A4
:10B7D8002003002B0AD07B681B689B6823F4005168
:10B7E8007B681A6C7B681B680A439A607B689B6A53
:10B7F80003F04003002B1AD07B681B685B6823F4B6
:10B8080080117B685A6C7B681B680A435A607B68A6
:10B818005B6CB3F5801F0AD17B681B685B6823F4F7
:10B82800C0017B689A6C7B681B680A435A607B6816
:10B838009B6A03F08003002B0AD07B681B685B6857
:10B8480023F400217B68DA6C7B681B680A435A6022
:10B8580000BF0C37BD465DF8047B704780B598B0D3
:10B8680002AF78607B680022C3F89020FAF7EEFEFA
:10B8780078657B681B681B6803F00803082B2FD1C9
:10B888006FF07E4300937B6D00224FF400117868BF
:10B8980000F08EF80346002B22D07B681B68BB6340
:10B8A800BB6B53E8003F7B637B6B23F080033B65F6
:10B8B8007B681B681A463B6D7B643A64396C7A6C0A
:10B8C80041E80023FB63FB6B002BE6D17B68202259
:10B8D800C3F888207B68002283F88420032363E070
:10B8E8007B681B681B6803F00403042B49D16FF0C5
:10B8F8007E4300937B6D00224FF48001786800F04E
:10B9080057F80346002B3CD07B681B687B627B6A38
:10B9180053E8003F3B623B6A23F49073FB647B6807
:10B928001B681A46FB6C3B63FA62F96A3A6B41E89A
:10B938000023BB62BB6A002BE6D17B681B68083317
:10B948003B613B6953E8003FFB60FB6823F0010360
:10B95800BB647B681B680833BA6CFA61BB61B96960
:10B96800FA6941E800237B617B69002BE5D17B689C
:10B978002022C3F88C207B68002283F884200323CC
:10B9880012E07B682022C3F888207B682022C3F855
:10B998008C207B680022DA667B6800221A677B6845
:10B9A800002283F88420002318465837BD4680BDFE
:10B9B80080B584B000AFF860B9603B601346FB7196
:10B9C8004FE0BB69B3F1FF3F4BD0FAF73FFE0246A9
:10B9D8003B68D31ABA699A4202D3BB69002B01D1DA
:10B9E80003234EE0FB681B681B6803F00403002B6D
:10B9F80037D0BB68802B34D0BB68402B31D0FB6874
:10BA08001B68DB6903F00803082B10D1FB681B686F
:10BA180008221A62F86800F038F8FB680822C3F8B0
:10BA28009020FB68002283F88420012329E0FB682A
:10BA38001B68DB6903F40063B3F5006F11D1FB6881
:10BA48001B684FF400621A62F86800F01EF8FB6881
:10BA58002022C3F89020FB68002283F88420032367
:10BA68000FE0FB681B68DA69BB681340BA689A4242
:10BA78000CBF01230023DBB21A46FB799A42A0D0FF
:10BA8800002318461037BD4680BD80B495B000AF7E
:10BA980078607B681B687B637B6B53E8003F3B6384
:10BAA8003B6B23F49073FB647B681B681A46FB6C42
:10BAB8003B64FA63F96B3A6C41E80023BB63BB6BE8
:10BAC800002BE6D17B681B6808333B623B6A53E86E
:10BAD800003FFB61FB6923F0805323F00103BB6443
:10BAE8007B681B680833BA6CFA62BB62B96AFA6A87
:10BAF80041E800237B627B6A002BE3D17B68DB6E25
:10BB0800012B18D17B681B68FB60FB6853E8003F7A
:10BB1800BB60BB6823F010037B647B681B681A4614
:10BB28007B6CBB617A617969BA6941E800233B6142
:10BB38003B69002BE6D17B682022C3F88C207B6808
:10BB48000022DA667B6800225A6700BF5437BD4678
:10BB58005DF8047B704780B485B000AF78607B687F
:10BB680093F88430012B01D1022327E07B6801225E
:10BB780083F884207B682422C3F888207B681B68AC
:10BB88001B68FB607B681B681A687B681B6822F06F
:10BB980001021A60FB6823F00053FB607B680022F7
:10BBA8005A667B681B68FA681A607B682022C3F8AB
:10BBB80088207B68002283F88420002318461437E5
:10BBC800BD465DF8047B704780B584B000AF7860EF
:10BBD80039607B6893F88430012B01D102232DE072
:10BBE8007B68012283F884207B682422C3F888209C
:10BBF8007B681B681B68FB607B681B681A687B682E
:10BC08001B6822F001021A607B681B689B6823F09E
:10BC180060417B681B683A680A439A60786800F05C
:10BC28004FF87B681B68FA681A607B682022C3F8A3
:10BC380088207B68002283F8842000231846103768
:10BC4800BD4680BD80B584B000AF786039607B6840
:10BC580093F88430012B01D102232DE07B68012267
:10BC680083F884207B682422C3F888207B681B68BB
:10BC78001B68FB607B681B681A687B681B6822F07E
:10BC880001021A607B681B689B6823F060617B680F
:10BC98001B683A680A439A60786800F011F87B6874
:10BCA8001B68FA681A607B682022C3F888207B68C2
:10BCB800002283F88420002318461037BD4680BD33
:10BCC80080B485B000AF78607B685B6E002B08D1CC
:10BCD8007B680122A3F86A207B680122A3F8682008
:10BCE80031E00823FB730823BB737B681B689B68E0
:10BCF8005B0EDBB203F007037B737B681B689B68F2
:10BD08005B0FDBB203F007033B73BB7B3A7B114944
:10BD18008A5C02FB03F33A7B0F498A5C93FBF2F3DC
:10BD28009AB27B68A3F86A20FB7B7A7B09498A5C14
:10BD380002FB03F37A7B08498A5C93FBF2F39AB21D
:10BD48007B68A3F8682000BF1437BD465DF8047B04
:10BD5800704700BF80D6010888D6010880B400AFBC
:10BD6800074BD3F88830064A43F47003C2F888308A
:10BD7800034B044A9A6000BFBD465DF8047B7047D8
:10BD880000ED00E00000010880B586B000AFF86063
:10BD9800B9601346FB71FB68002B01D103231FE038
:10BDA800FB680022C3F8B822FB680022C3F8C0224F
:10BDB800FB680022C3F8CC22BB68002B03D0FB68C9
:10BDC800BA68C3F8B422FB68012283F89C22FB6896
:10BDD800FA791A70F868F5F72BFF0346FB75FB7DB7
:10BDE80018461837BD4680BD80B584B000AF78606E
:10BDF80039600023FB813B68002B01D1032316E047
:10BE08007B683A68C3F8B8227B68D3F8B832DB6A33
:10BE1800002B0BD07B68D3F8B832DB6A07F10E022F
:10BE28001046984702467B68C3F8CC220023184680
:10BE38001037BD4680BD80B582B000AF78607868A5
:10BE4800F5F756FF034618460837BD4680BD80B44F
:10BE580083B000AF7860002318460C37BD465DF804
:10BE6800047B704780B584B000AF78600B46FB70E8
:10BE78000323FB737B68D3F8B832002B09D07B68A7
:10BE8800D3F8B8321B68FA781146786898470346A1
:10BE9800FB73FB7B18461037BD4680BD80B582B06A
:10BEA80000AF78600B46FB707B68D3F8B832002B84
:10BEB80007D07B68D3F8B8325B68FA78114678689F
:10BEC8009847002318460837BD4680BD80B584B022
:10BED80000AF786039607B6803F2AA233968184696
:10BEE80000F046FF7B680122C3F894227B68B3F810
:10BEF800B0321A467B68C3F898227B6893F8AA3256
:10BF080003F01F03022B1AD0022B22D8002B02D0D9
:10BF1800012B0AD01DE07B6803F2AA231946786832
:10BF280000F0EEF90346FB7320E07B6803F2AA23D6
:10BF38001946786800F052FA0346FB7316E07B68EE
:10BF480003F2AA231946786800F091FA0346FB73B6
:10BF58000CE07B6893F8AA3223F07F03DBB2194622
:10BF68007868F5F725FF0346FB7300BFFB7B18468F
:10BF78001037BD4680BD80B586B000AFF8600B466F
:10BF88007A60FB72FB7A002B38D1FB6803F5AA7341
:10BF98003B61FB68D3F89432032B4AD13B699A681A
:10BFA8003B69DB689A4213D93B699A683B69DB684D
:10BFB800D21A3B699A603B69DA683B699B6893428D
:10BFC80028BF13461A467968F86800F0C5FF30E0C4
:10BFD800FB6893F89C32DBB2032B0BD1FB68D3F8D8
:10BFE800B8321B69002B05D0FB68D3F8B8321B693F
:10BFF800F8689847F86800F0C0FF1AE0FB6893F803
:10C008009C32DBB2032B14D1FB68D3F8B8329B699E
:10C01800002B0ED0FB68D3F8B8329B69FA7A114628
:10C02800F86898470346FB75FB7D002B01D0FB7D24
:10C0380000E0002318461837BD4680BD80B586B09D
:10C0480000AFF8600B467A60FB72FB7A002B6BD16D
:10C05800FB6814333B61FB68D3F89432022B56D14A
:10C068003B699A683B69DB689A4214D93B699A68CC
:10C078003B69DB68D21A3B699A603B699B681A4640
:10C088007968F86800F03AFF002300220021F86878
:10C09800F5F738FF3BE03B69DA683B699B689A42F1
:10C0A8001CD13B695A683B69DB689A4216D33B69E5
:10C0B8005A68FB68D3F898329A420FD200220021BE
:10C0C800F86800F01BFFFB680022C3F898220023E1
:10C0D80000220021F868F5F715FF18E0FB6893F8CF
:10C0E8009C32DBB2032B0BD1FB68D3F8B832DB6888
:10C0F800002B05D0FB68D3F8B832DB68F86898479E
:10C108008021F868F5F754FEF86800F049FFFB68ED
:10C1180093F8A032012B22D1F868FFF798FEFB684C
:10C12800002283F8A0221AE0FB6893F89C32DBB265
:10C13800032B14D1FB68D3F8B8325B69002B0ED0FF
:10C14800FB68D3F8B8325B69FA7A1146F868984701
:10C158000346FB75FB7D002B01D0FB7D00E000232F
:10C1680018461837BD4680BD80B582B000AF7860EC
:10C178007B68012283F89C227B680022C3F8942202
:10C188007B6800225A607B680022C3F8A4227B687F
:10C19800D3F8B832002B01D103232FE07B68D3F802
:10C1A800BC32002B0FD07B68D3F8B8325B68002B09
:10C1B80009D07B68D3F8B8325B687A685268D2B223
:10C1C8001146786898474023002200217868F5F7DF
:10C1D800AAFD7B680122A3F864217B684022C3F88A
:10C1E80060214023002280217868F5F79CFD7B6858
:10C1F80001229A847B6840221A6200231846083775
:10C20800BD4680BD80B483B000AF78600B46FB703C
:10C218007B68FA781A74002318460C37BD465DF817
:10C22800047B704780B483B000AF78607B6893F874
:10C238009C32DAB27B6883F89D227B68042283F8FB
:10C248009C22002318460C37BD465DF8047B7047D6
:10C2580080B483B000AF78607B6893F89C32DBB21F
:10C26800042B06D17B6893F89D32DAB27B6883F899
:10C278009C22002318460C37BD465DF8047B7047A6
:10C2880080B582B000AF78607B68D3F8B832002BF5
:10C2980001D1032312E07B6893F89C32DBB2032BB5
:10C2A8000BD17B68D3F8B832DB69002B05D07B68EB
:10C2B800D3F8B832DB6978689847002318460837FE
:10C2C800BD4680BD80B487B000AF78607B687B6175
:10C2D8007B691B787B827B6901337B617B691B7877
:10C2E8003B823B8A1B021AB2B7F9123013431BB2C6
:10C2F800FB81FB8918461C37BD465DF8047B7047F7
:10C3080080B584B000AF786039600023FB733B6868
:10C318001B7803F06003402B05D0402B53D8002B2B
:10C328000BD0202B4FD17B68D3F8B8329B68396883
:10C33800786898470346FB734AE03B685B78092BAB
:10C348003BD801A252F823F0A5C30108B9C30108DC
:10C35800C3C30108AFC30108C3C3010883C30108ED
:10C3680079C30108C3C301089BC301088DC3010831
:10C378003968786800F0DEF924E03968786800F0F8
:10C388006DFB1FE03968786800F0ACFB0346FB736F
:10C3980018E03968786800F04BFC13E03968786871
:10C3A80000F07CFC0EE03968786800F0ABFC09E02E
:10C3B8003968786800F0BAFC04E03968786800F0F9
:10C3C80011FD00BF04E03968786800F00BFD00BF7C
:10C3D800FB7B18461037BD4680BD00BF80B584B0D2
:10C3E80000AF786039600023FB733B681B7803F06B
:10C3F8006003402B05D0402B2FD8002B01D0202BD9
:10C408002BD17B6893F89C32DBB2013B022B1DD801
:10C418003B689B88DBB2012B13D87B68D3F8B83212
:10C428009B683968786898470346FB733B68DB88E4
:10C43800002B10D1FB7B002B0DD1786800F09DFDFF
:10C4480009E03968786800F0CDFC04E0396878685C
:10C4580000F0C8FC00E000BF04E03968786800F02C
:10C46800C1FC00BFFB7B18461037BD4680BD80B5B8
:10C4780084B000AF786039600023FB733B689B8809
:10C48800BB733B681B7803F06003402B07D0402B3D
:10C4980000F24581002B0CD0202B40F040817B68B6
:10C4A800D3F8B8329B683968786898470346FB73B5
:10C4B8003AE13B685B78032B07D0032B00F3298113
:10C4C800002B7FD0012B3CD023E17B6893F89C3272
:10C4D800DBB2022B02D0032B16D02CE0BB7B002B47
:10C4E8000DD0BB7B802B0AD0BB7B19467868F5F74B
:10C4F8005FFC80217868F5F75BFC00BF20E03968B5
:10C50800786800F06FFC1BE03B685B88002B0ED15D
:10C51800BB7B002B0BD0BB7B802B08D03B68DB8818
:10C52800002B04D1BB7B19467868F5F741FC786885
:10C5380000F023FD04E03968786800F053FC00BF80
:10C54800ECE07B6893F89C32DBB2022B02D0032B21
:10C5580016D030E0BB7B002B0DD0BB7B802B0AD0E4
:10C56800BB7B19467868F5F723FC80217868F5F7D6
:10C578001FFC00BF25E03968786800F033FC20E034
:10C588003B685B88002B1BD1BB7B03F07F03002B30
:10C5980004D0BB7B19467868F5F729FC786800F069
:10C5A800ECFC7B68D3F8B8329B68396878689847A0
:10C5B8000346FB7304E03968786800F013FC00E078
:10C5C80000BFABE07B6893F89C32DBB2022B02D051
:10C5D800032B32D097E0BB7B002B07D0BB7B802B93
:10C5E80004D03968786800F0FDFB91E097F90E30C7
:10C5F800002B0BDABB7B03F07F0213469B0013442E
:10C608009B0010337A68134404330BE0BB7B03F0C0
:10C618007F0213469B0013449B0003F5A8737A68B6
:10C6280013440433BB60BB6800221A60BB68022253
:10C638001946786800F047FC6AE097F90E30002B3D
:10C6480011DABB7B03F00F02796813469B00134491
:10C658009B000B4424331B88002B17D1396878685A
:10C6680000F0C0FB54E0BB7B03F00F02796813466F
:10C678009B0013449B000B4403F5B2731B88002BEB
:10C6880004D13968786800F0ADFB41E097F90E30C5
:10C69800002B0BDABB7B03F07F0213469B0013448D
:10C6A8009B0010337A68134404330BE0BB7B03F020
:10C6B8007F0213469B0013449B0003F5A8737A6816
:10C6C80013440433BB60BB7B002B02D0BB7B802BA5
:10C6D80003D1BB6800221A600EE0BB7B194678685C
:10C6E800F5F7A4FB0346002B03D0BB6801221A60B0
:10C6F80002E0BB6800221A60BB680222194678680B
:10C7080000F0E1FB04E03968786800F06BFB00BFDB
:10C7180004E03968786800F065FB00BF04E0396818
:10C72800786800F05FFB00BFFB7B18461037BD46FA
:10C7380080BD000080B584B000AF78603960002308
:10C748003B810023FB600023FB723B685B881B0A6C
:10C758009BB2013B0E2B00F2528101A252F823F04A
:10C76800D9C70108F1C7010831C8010807CA01087B
:10C7780007CA0108A7C90108D3C9010807CA0108DF
:10C7880007CA010807CA010807CA010807CA010839
:10C7980007CA010807CA0108A5C701087B68D3F8BA
:10C7A800B432DB69002B0BD07B68D3F8B432DB6979
:10C7B8007A68127C07F1080110469847F86026E16C
:10C7C8003968786800F00EFBFB7A0133FB721EE1D2
:10C7D8007B68D3F8B4321B687A68127C07F10801C9
:10C7E80010469847F86012E17B681B7C002B0DD13E
:10C7F8007B68D3F8B8329B6A07F10802104698475D
:10C80800F860FB68013302221A7000E17B68D3F8F4
:10C81800B832DB6A07F1080210469847F860FB68EF
:10C82800013302221A70F2E03B685B88DBB2052B09
:10C8380000F2AC8001A252F823F000BF5DC80108E5
:10C8480091C80108C5C80108F9C801082DC901081F
:10C8580061C901087B68D3F8B4325B68002B0BD040
:10C868007B68D3F8B4325B687A68127C07F10801F8
:10C8780010469847F86091E03968786800F0B2FA95
:10C88800FB7A0133FB7289E07B68D3F8B4329B688A
:10C89800002B0BD07B68D3F8B4329B687A68127C83
:10C8A80007F1080110469847F86077E0396878681A
:10C8B80000F098FAFB7A0133FB726FE07B68D3F8DB
:10C8C800B432DB68002B0BD07B68D3F8B432DB685A
:10C8D8007A68127C07F1080110469847F8605DE015
:10C8E8003968786800F07EFAFB7A0133FB7255E00C
:10C8F8007B68D3F8B4321B69002B0BD07B68D3F864
:10C90800B4321B697A68127C07F10801104698470F
:10C91800F86043E03968786800F064FAFB7A01331C
:10C92800FB723BE07B68D3F8B4325B69002B0BD019
:10C938007B68D3F8B4325B697A68127C07F1080126
:10C9480010469847F86029E03968786800F04AFA94
:10C95800FB7A0133FB7221E07B68D3F8B4329B6920
:10C96800002B0BD07B68D3F8B4329B697A68127CB1
:10C9780007F1080110469847F8600FE039687868B1
:10C9880000F030FAFB7A0133FB7207E03968786807
:10C9980000F028FAFB7A0133FB7200BF37E07B68AE
:10C9A8001B7C002B09D17B68D3F8B8325B6B07F18D
:10C9B800080210469847F86029E03968786800F05E
:10C9C80011FAFB7A0133FB7221E07B681B7C002B98
:10C9D8000DD17B68D3F8B8321B6B07F108021046FB
:10C9E8009847F860FB68013307221A700FE039682E
:10C9F800786800F0F7F9FB7A0133FB7207E03968D1
:10CA0800786800F0EFF9FB7A0133FB7200BFFB7A1C
:10CA1800002B1ED13B68DB88002B16D03B89002BEE
:10CA28000ED03B68DA883B89934228BF13469BB2F5
:10CA38003B813B891A46F968786800F044FA09E0B6
:10CA48003968786800F0CEF904E0786800F095FA63
:10CA580000E000BF1037BD4680BD00BF80B584B080
:10CA680000AF786039603B689B88002B31D13B6808
:10CA7800DB88002B2DD13B685B887F2B29D83B684E
:10CA88005B88DBB203F07F03FB737B6893F89C320F
:10CA9800DBB2032B04D13968786800F0A3F91DE0F4
:10CAA8007B68FA7B83F89E22FB7B19467868F5F74A
:10CAB800E9F9786800F061FAFB7B002B04D07B6809
:10CAC800022283F89C2209E07B68012283F89C22D9
:10CAD80004E03968786800F085F900BF00BF1037B6
:10CAE800BD4680BD80B584B000AF78603960002352
:10CAF800FB733B685B88DAB24C4B1A704B4B1B7864
:10CB0800012B05D93968786800F06CF9032388E0AF
:10CB18007B6893F89C32DBB2022B02D0032B25D022
:10CB280071E0424B1B78002B1CD0404B1B781A46F7
:10CB38007B685A603D4B1B7819467868FFF792F975
:10CB48000346FB73FB7B002B04D03968786800F040
:10CB580049F965E0786800F010FA7B68032283F8E9
:10CB68009C225DE0786800F008FA59E02F4B1B78AA
:10CB7800002B12D17B68022283F89C222B4B1B7856
:10CB88001A467B685A60294B1B7819467868FFF764
:10CB980085F9786800F0F1F942E0244B1B781A46D1
:10CBA8007B685B689A422AD07B685B68DBB219466F
:10CBB8007868FFF773F91D4B1B781A467B685A6033
:10CBC8001A4B1B7819467868FFF74CF90346FB7334
:10CBD800FB7B002B0FD03968786800F003F97B687D
:10CBE8005B68DBB219467868FFF758F97B68022260
:10CBF80083F89C2214E0786800F0BFF910E07868A8
:10CC080000F0BBF90CE03968786800F0EBF8074BE6
:10CC18001B7819467868FFF741F90323FB7300BFB7
:10CC2800FB7B18461037BD4680BD00BF4C1F002057
:10CC380080B582B000AF786039603B68DB88012B33
:10CC480004D03968786800F0CDF823E07B6893F861
:10CC58009C32DBB2022B02DC002B03DC15E0032B39
:10CC68000BD012E07B6800229A607B6808330122AF
:10CC78001946786800F027F90CE07B680433012234
:10CC88001946786800F01FF904E03968786800F000
:10CC9800A9F800BF00BF0837BD4680BD80B582B087
:10CCA80000AF786039607B6893F89C32DBB2013B57
:10CCB800022B1ED83B68DB88022B04D039687868C1
:10CCC80000F090F81AE07B680122DA607B68D3F8FC
:10CCD800A432002B05D07B68DB6843F002027B6836
:10CCE800DA607B680C3302221946786800F0EBF8AA
:10CCF80004E03968786800F075F800BF00BF0837AD
:10CD0800BD4680BD80B582B000AF786039603B68B1
:10CD18005B88012B06D17B680122C3F8A4227868BE
:10CD280000F02BF900BF0837BD4680BD80B582B042
:10CD380000AF786039607B6893F89C32DBB2013BC6
:10CD4800022B0BD83B685B88012B0CD17B68002237
:10CD5800C3F8A422786800F010F904E0396878680C
:10CD680000F040F800E000BF00BF0837BD4680BDB6
:10CD780080B584B000AF786039603B68FB60FB68C1
:10CD88001A787B681A70FB680133FB60FB681A78B5
:10CD98007B685A70FB680133FB60F868FFF792FA0A
:10CDA80003461A467B685A80FB680133FB60FB68C0
:10CDB8000133FB60F868FFF785FA03461A467B687B
:10CDC8009A80FB680133FB60FB680133FB60F868FD
:10CDD800FFF778FA03461A467B68DA8000BF1037F7
:10CDE800BD4680BD80B582B000AF786039608021D3
:10CDF8007868F4F7DDFF00217868F4F7D9FF00BF01
:10CE08000837BD4680BD80B586B000AFF860B96010
:10CE18007A600023FB75FB68002B36D0FB683B610A
:10CE2800386900F036F8034601339BB25B009AB2CA
:10CE38007B681A80FB7DBA6813447A6812781A7086
:10CE4800FB7D0133FB75FB7DBA68134403221A701E
:10CE5800FB7D0133FB7513E0FB7DBA6813443A6927
:10CE680012781A703B6901333B61FB7D0133FB7516
:10CE7800FB7DBA68134400221A70FB7D0133FB75F1
:10CE88003B691B78002BE7D100E000BF1837BD468F
:10CE980080BD80B485B000AF78600023FB737B68E9
:10CEA800BB6005E0FB7B0133FB73BB680133BB60F0
:10CEB800BB681B78002BF5D1FB7B18461437BD46A1
:10CEC8005DF8047B704780B584B000AFF860B96046
:10CED8007A60FB680222C3F89422FB687A689A6138
:10CEE800FB687A68DA617B68BA680021F868F4F749
:10CEF800E8FF002318461037BD4680BD80B584B0D2
:10CF080000AFF860B9607A607B68BA680021F86899
:10CF1800F4F7D7FF002318461037BD4680BD80B50B
:10CF280084B000AFF860B9607A60FB680322C3F888
:10CF38009422FB687A68C3F85821FB687A68C3F8BA
:10CF48005C217B68BA680021F868F4F7DBFF0023EE
:10CF580018461037BD4680BD80B584B000AFF86074
:10CF6800B9607A607B68BA680021F868F4F7CAFF8C
:10CF7800002318461037BD4680BD80B582B000AF8B
:10CF880078607B680422C3F89422002300220021E1
:10CF98007868F4F796FF002318460837BD4680BD29
:10CFA80080B582B000AF78607B680522C3F8942210
:10CFB8000023002200217868F4F7A4FF0023184614
:10CFC8000837BD4680BD80B584B000AF78600B4699
:10CFD800FB704FF40770F4F7FFFFF860FB68002B55
:10CFE80005D17B680022C3F8BC22022366E07B6877
:10CFF800FA68C3F8BC227B681B7C002B19D14FF45C
:10D008000073022281217868F4F78DFE7B68012283
:10D018001A874FF40073022201217868F4F783FE1F
:10D028007B680122A3F878217B681022A3F84E20A0
:10D0380016E04023022281217868F4F774FE7B68A9
:10D0480001221A874023022201217868F4F76BFE37
:10D058007B680122A3F878217B681022A3F84E2070
:10D068000823032282217868F4F75DFE7B68012299
:10D07800A3F84C207B68D3F8C0321B689847FB683C
:10D088000022C3F81422FB680022C3F818227B6828
:10D098001B7C002B09D1FB68D3F804224FF40073E2
:10D0A80001217868F4F72EFF07E0FB68D3F8042223
:10D0B800402301217868F4F725FF0023184610372C
:10D0C800BD4680BD80B582B000AF78600B46FB706E
:10D0D80081217868F4F74DFE7B6800221A870121C8
:10D0E8007868F4F746FE7B680022A3F8782182214D
:10D0F8007868F4F73EFE7B680022A3F84C207B6832
:10D108000022A3F84E207B68D3F8BC32002B0ED047
:10D118007B68D3F8C0325B6898477B68D3F8BC3229
:10D128001846F4F767FF7B680022C3F8BC22002387
:10D1380018460837BD4680BD80B586B000AF786018
:10D1480039607B68D3F8BC323B6100237B730023D2
:10D158007B810023FB753B69002B01D10323AFE0E2
:10D168003B681B7803F06003002B3FD0202B40F076
:10D178009F803B68DB88002B2ED03B681B785BB216
:10D18800002B16DA7B68D3F8C0329B683A6850786F
:10D1980039693A68D28898473B68DB88072B28BFEB
:10D1A8000723FB813B69FA8919467868FFF78BFEEC
:10D1B80085E03B685A783B6983F800223B68DB8846
:10D1C800DAB23B6983F8012239693B68DB881A4681
:10D1D8007868FFF7A4FE72E07B68D3F8C0329B68DA
:10D1E8003A68507800223968984768E03B685B786D
:10D1F8000B2B52D801A252F823F000BF35D20108F8
:10D20800B1D20108A3D20108A3D20108A3D2010810
:10D21800A3D20108A3D20108A3D20108A3D201080E
:10D22800A3D201085FD2010889D201087B6893F86C
:10D238009C32DBB2032B07D107F10A0302221946FD
:10D248007868FFF740FE32E039687868FFF7CAFD72
:10D258000323FB752BE07B6893F89C32DBB2032B2E
:10D2680007D107F10D03012219467868FFF72BFE55
:10D278001DE039687868FFF7B5FD0323FB7516E0F4
:10D288007B6893F89C32DBB2032B0FD0396878683F
:10D29800FFF7A8FD0323FB7508E039687868FFF7F6
:10D2A800A1FD0323FB7502E000BF08E000BF06E014
:10D2B80039687868FFF796FD0323FB7500BFFB7D8F
:10D2C80018461837BD4680BD80B584B000AF786079
:10D2D8000B46FB707B68D3F8C432FB607B68D3F8DD
:10D2E800BC32002B01D103234FE07B68D3F8BC325A
:10D2F800BB60FA78796813469B0013449B000B4483
:10D3080018331B68002B29D0FA78796813469B00DC
:10D3180013449B000B4418331A68F978F8680B46D5
:10D328009B000B44DB00034420331B68B2FBF3F182
:10D3380001FB03F3D31A002B10D1FA78796813464E
:10D348009B0013449B000B44183300221A60F978A1
:10D35800002300227868F4F7B4FD15E0BB680022CA
:10D36800C3F814227B68D3F8C0321B69002B0BD09A
:10D378007B68D3F8C0321B69BA68D2F80802BA6869
:10D3880002F50471FA789847002318461037BD460D
:10D3980080BD80B584B000AF78600B46FB707B68B9
:10D3A800D3F8BC32FB607B68D3F8BC32002B01D1C8
:10D3B800032315E0FB7819467868F4F7C4FD0246A4
:10D3C800FB68C3F80C227B68D3F8C032DB68FA68C4
:10D3D800D2F80402FA6802F503721146984700234E
:10D3E80018461037BD4680BD80B584B000AF786060
:10D3F8007B68D3F8BC32FB60FB68002B01D10323A8
:10D408001AE07B68D3F8C032002B14D0FB6893F87D
:10D418000032FF2B0FD07B68D3F8C0329B68FA68C4
:10D4280092F80002F968FA6892F801229847FB68B6
:10D43800FF2283F80022002318461037BD4680BD1E
:10D4480080B483B000AF78607B6843221A80034BB6
:10D4580018460C37BD465DF8047B7047FC00002079
:10D4680080B483B000AF78607B6843221A80034B96
:10D4780018460C37BD465DF8047B7047B80000209D
:10D4880080B483B000AF78607B6843221A80034B76
:10D4980018460C37BD465DF8047B704740010020F4
:10D4A80080B483B000AF78607B680A221A80034B8F
:10D4B80018460C37BD465DF8047B704774000020A1
:10D4C80080B483B000AF786039603B68002B01D12D
:10D4D800032304E07B683A68C3F8C0220023184697
:10D4E8000C37BD465DF8047B704780B487B000AF49
:10D4F800F860B9607A60FB68D3F8BC327B617B69FD
:10D50800002B01D1032308E07B69BA68C3F808221D
:10D518007B697A68C3F81022002318461C37BD4679
:10D528005DF8047B704780B485B000AF78603960DF
:10D538007B68D3F8BC32FB60FB68002B01D1032366
:10D5480004E0FB683A68C3F804220023184614373D
:10D55800BD465DF8047B704780B584B000AF786045
:10D568007B68D3F8BC32FB607B68D3F8BC32002BF5
:10D5780001D1032316E07B681B7C002B09D1FB68D3
:10D58800D3F804224FF4007301217868F4F7BAFC49
:10D5980007E0FB68D3F80422402301217868F4F7F8
:10D5A800B1FC002318461037BD4680BD0D4885469E
:10D5B800FEF7D4FB0C480D490D4A002302E0D4586D
:10D5C800C4500433C4188C42F9D30A4A0A4C0023C5
:10D5D80001E013600432A242FBD3F2F799FFF2F79D
:10D5E800BBFFFEE7000002200000002084010020AD
:10D5F800B8D6010884010020501F0020FEE7000073
:10D60800F8B500BFF8BC08BC9E467047F8B500BF27
:08D61800F8BC08BC9E467047F7
:10D6200053544D3332205669727475616C20436FC8
:10D630006D506F727400000053544D6963726F65D2
:10D640006C656374726F6E696373000043444320BA
:10D65000436F6E666967000043444320496E7465FA
:10D6600072666163650000000100020004000600AC
:10D6700008000A000C00100020004000800000019B
:10D68000010101030701000008040204080101016F
:10D690000000000000000000010203040607080962
:08D6A000000000000102030478
:08D6A800A02BFF7F0100000030
:04D6B000FD0101086F
:04D6B400D90101088F
:10D6B800D5200108F9200108592101081D21010878
:10D6C80081210108A5210108E121010800000000CD
:10D6D80012010002020200408304405700020102C6
:10D6E80003010000040309041A03000000000000FD
:10D6F8000000000000000000000000000000000022
:10D7080000000000F52201081D2301082D2301084F
:10D71800E92301081124010810000000010000009D
:10D728000024F4000A060002000000400100000086
:10D73800CFCF0108CDD0010841D101080000000079
:10D74800F1D30108D1D201089BD3010800000000E1
:10D75800000000000000000069D4010849D4010855
:10D7680089D40108A9D4010809024300020100C0B4
:10D77800320904000001020201000524001001051D
:10D788002401000104240202052406000107058281
:10D798000308001009040100020A0000000705013F
:10D7A800020002000705810200020000090243008E
:10D7B800020100C032090400000102020100052430
:10D7C80000100105240100010424020205240600BA
:10D7D800010705820308001009040100020A00007D
:10D7E8000007050102400000070581024000000013
:10D7F80009074300020104C03209040000010202C3
:10D80800010005240010010524010001042402027E
:10D818000524060001070582030800100904010019
:10D82800020A000000070501024000000705810206
:04D8380040000000AC
:040000050801D5B564
:00000001FF
